:020000040800F2
:1000000000000824692A00080121000803210008D3
:100010000521000807210008092100080000000050
:100020000000000000000000000000000B2100089C
:100030000D210008000000000F2100081121000818
:10004000B92A0008B92A0008B92A0008B92A000804
:10005000B92A0008B92A0008B92A0008B92A0008F4
:10006000B92A0008B92A0008B92A0008192100088D
:10007000B92A0008B92A0008B92A0008B92A0008D4
:10008000B92A0008B92A000829210008B92A00085D
:10009000B92A0008B92A0008B92A0008B92A0008B4
:1000A000B92A0008B92A00083921000849210008A6
:1000B000B92A000859210008B92A0008B92A0008FD
:1000C000B92A0008B92A0008B92A0008B92A000884
:1000D000B92A000869210008B92A0008B92A0008CD
:1000E000B92A0008B92A0008000000007921000898
:1000F000B92A0008B92A0008B92A0008B92A000854
:10010000B92A0008B92A0008B92A0008B92A000843
:10011000B92A0008B92A0008B92A0008B92A000833
:10012000B92A0008B92A0008B92A0008B92A000823
:10013000B92A0008B92A0008B92A0008B92A000813
:1001400000000000000000000000000000000000AF
:10015000B92A0008B92A0008B92A0008B92A0008F3
:10016000B92A0008B92A0008B92A0008B92A0008E3
:10017000B92A0008B92A0008B92A0008B92A0008D3
:10018000B92A0008B92A0008B92A0008B92A0008C3
:10019000B92A0008B92A0008B92A0008B92A0008B3
:1001A000B92A0008B92A0008B92A0008B92A0008A3
:1001B000B92A0008B92A0008B92A0008B92A000893
:1001C000B92A0008B92A0008B92A0008B92A000883
:1001D000B92A0008B92A0008B92A0008B92A000873
:1001E000B92A0008B92A0008B92A0008B92A000863
:1001F000B92A0008B92A0008B92A0008B92A000853
:10020000B92A0008B92A0008B92A0008B92A000842
:10021000B92A0008B92A0008B92A0008B92A000832
:10022000B92A0008B92A0008B92A0008000000000D
:10023000B92A0008B92A000800000000B92A0008FD
:10024000B92A0008B92A0008B92A0008B92A000802
:10025000B92A0008B92A0008B92A0008B92A0008F2
:10026000B92A0008B92A0008B92A0008B92A0008E2
:10027000B92A0008B92A0008B92A000800000000BD
:10028000B92A0008B92A0008B92A000800000000AD
:0802900000000000B92A00087B
:1002C00010B5054C237833B9044B13B10448AFF390
:1002D00000800123237010BDC0090024000000002D
:1002E000F005010808B5034B1BB103490348AFF300
:1002F000008008BD00000000C4090024F0050108CA
:1003000080F0004002E000BF81F0004142001FBFCA
:100310005FEA410392EA030F7FEA226C7FEA236CD3
:100320006AD04FEA1262D2EB1363C1BFD2184140C8
:1003300048404140B8BF5B42192B88BF704710F05E
:10034000004F40F4000020F07F4018BF404211F001
:10035000004F41F4000121F07F4118BF494292EA69
:10036000030F3FD0A2F1010241FA03FC10EB0C0095
:10037000C3F1200301FA03F100F0004302D5494222
:1003800060EB4000B0F5000F13D3B0F1807F06D3CF
:1003900040084FEA310102F10102FE2A51D2B1F1C7
:1003A000004F40EBC25008BF20F0010040EA0300BC
:1003B0007047490040EB0000013A28BFB0F5000F3C
:1003C000EDD2B0FA80FCACF1080CB2EB0C0200FAF2
:1003D0000CF0AABF00EBC25052421843BCBFD04041
:1003E0001843704792F0000F81F4000106BF80F4BB
:1003F00000000132013BB5E74FEA41037FEA226C7E
:1004000018BF7FEA236C21D092EA030F04D092F048
:10041000000F08BF0846704790EA010F1CBF00207C
:10042000704712F07F4F04D1400028BF40F00040D9
:10043000704712F100723CBF00F50000704700F0F9
:10044000004343F0FE4040F4000070477FEA226220
:1004500016BF08467FEA23630146420206BF5FEAF1
:10046000412390EA010F40F4800070474FF00003F1
:1004700004E000BF10F0004348BF40425FEA000CB8
:1004800008BF704743F0964301464FF000001CE060
:1004900050EA010208BF70474FF000030AE000BFB6
:1004A00050EA010208BF704711F0004302D54042F4
:1004B00061EB41015FEA010C02BF84460146002066
:1004C00043F0B64308BFA3F18053A3F50003BCFA81
:1004D0008CF2083AA3EBC25310DB01FA02FC63442E
:1004E00000FA02FCC2F12002BCF1004F20FA02F235
:1004F00043EB020008BF20F00100704702F1200228
:1005000001FA02FCC2F1200250EA4C0021FA02F288
:1005100043EB020008BF20EADC7070474FF0FF0C8D
:100520001CEAD0521EBF1CEAD15392EA0C0F93EA88
:100530000C0F6FD01A4480EA010C400218BF5FEA2A
:1005400041211ED04FF0006343EA501043EA51119D
:10055000A0FB01310CF00040B1F5000F3EBF490097
:1005600041EAD3715B0040EA010062F17F02FD2A9B
:100570001DD8B3F1004F40EBC25008BF20F001007E
:10058000704790F0000F0CF0004C08BF49024CEA95
:10059000502040EA51207F3AC2BFD2F1FF0340EA27
:1005A000C250704740F400004FF00003013A5DDC98
:1005B00012F1190FDCBF00F000407047C2F10002D9
:1005C000410021FA02F1C2F1200200FA02FC5FEAC6
:1005D000310040F1000053EA4C0308BF20EADC7010
:1005E000704792F0000F00F0004C02BF400010F482
:1005F000000F013AF9D040EA0C0093F0000F01F02F
:10060000004C02BF490011F4000F013BF9D041EA50
:100610000C018FE70CEAD15392EA0C0F18BF93EA52
:100620000C0F0AD030F0004C18BF31F0004CD8D17C
:1006300080EA010000F00040704790F0000F17BF03
:1006400090F0004F084691F0000F91F0004F14D049
:1006500092EA0C0F01D142020FD193EA0C0F03D1A1
:100660004B0218BF084608D180EA010000F00040A4
:1006700040F0FE4040F40000704740F0FE4040F47F
:10068000400070474FF0FF0C1CEAD0521EBF1CEA1E
:10069000D15392EA0C0F93EA0C0F69D0A2EB03023C
:1006A00080EA010C49024FEA402037D04FF08053D6
:1006B00043EA111143EA10130CF000408B4238BF9B
:1006C0005B0042F17D024FF4000C8B4224BF5B1AA9
:1006D00040EA0C00B3EB510F24BFA3EB510340EAF7
:1006E0005C00B3EB910F24BFA3EB910340EA9C00A5
:1006F000B3EBD10F24BFA3EBD10340EADC001B0115
:1007000018BF5FEA1C1CE0D1FD2A3FF650AF8B42B8
:1007100040EBC25008BF20F0010070470CF0004CC5
:100720004CEA50207F32C2BFD2F1FF0340EAC250F0
:10073000704740F400004FF00003013A37E792F0B1
:10074000000F00F0004C02BF400010F4000F013A0F
:10075000F9D040EA0C0093F0000F01F0004C02BF0A
:10076000490011F4000F013BF9D041EA0C0195E773
:100770000CEAD15392EA0C0F08D142027FF47DAF0C
:1007800093EA0C0F7FF470AF084676E793EA0C0FFC
:1007900004D14B023FF44CAF08466EE730F0004CFA
:1007A00018BF31F0004CCAD130F000427FF45CAF8A
:1007B00031F000437FF43CAF5FE700BF42000ED250
:1007C000B2F1FE4F0BD34FF09E03B3EB126209D48C
:1007D0004FEA002343F0004323FA02F070474FF042
:1007E0000000704712F1610F01D1420202D14FF0B7
:1007F000FF3070474FF00000704700BF53B94AB94F
:10080000002908BF00281CBF4FF0FF314FF0FF3018
:1008100000F074B9ADF1080C6DE904CE00F006F8F3
:10082000DDF804E0DDE9022304B070472DE9F0476C
:10083000089E0D4604468846002B4DD18A429446B8
:1008400068D9B2FA82F252B101FA02F3C2F1200180
:1008500020FA01F10CFA02FC41EA030894404FEA45
:100860001C45210CB8FBF5FE1FFA8CF705FB1E8317
:1008700041EA03430EFB07F199420BD91CEB03033A
:100880000EF1FF3080F01E81994240F21B81AEF1E3
:10089000020E63445B1AA4B2B3FBF5F005FB103300
:1008A00044EA034400FB07F7A7420AD91CEB0404FF
:1008B00000F1FF3380F00881A74240F205816444D3
:1008C0000238E41B40EA0E4000211EB1D440002350
:1008D000C6E90043BDE8F0878B4208D9002E00F03E
:1008E000EE800021C6E900050846BDE8F087B3FAAE
:1008F00083F100294AD1AB4202D3824200F2F9804F
:10090000841A65EB030301209846002EE2D0C6E965
:100910000048DFE702B9FFDEB2FA82F2002A40F0B7
:100920009180A1EB0C054FEA1C471FFA8CFE0121B8
:10093000B5FBF7F307FB1350250C45EA00450EFB0A
:1009400003F0A84208D91CEB050503F1FF3802D2D9
:10095000A84200F2CB8043462D1AA4B2B5FBF7F0B3
:1009600007FB105544EA05440EFB00FEA64508D9D6
:100970001CEB040400F1FF3502D2A64500F2BB8057
:100980002846A4EB0E0440EA03409EE7C1F120078D
:100990008B4022FA07FC4CEA030C20FA07F405FA14
:1009A00001F31C43FD404FEA1C4900FA01F3B5FB7B
:1009B000F9F8200C1FFA8CFE09FB185540EA054592
:1009C00008FB0EF0A84202FA01F20BD91CEB050558
:1009D00008F1FF3A80F08880A84240F28580A8F1B3
:1009E000020865442D1AA4B2B5FBF9F009FB1055B5
:1009F00044EA054500FB0EFEAE4508D91CEB050593
:100A000000F1FF346CD2AE456AD90238654440EA41
:100A10000840A0FB0294A5EB0E05A542C846A646D9
:100A200056D353D05EB1B3EB080265EB0E0505FA61
:100A300007F722FA01F3CD401F43C6E900750021F4
:100A4000BDE8F087C2F1200320FA03F10CFA02FCA2
:100A500025FA03F395400D434FEA1C471FFA8CFE1D
:100A6000B3FBF7F107FB11302B0C43EA004301FB0A
:100A70000EF0984204FA02F408D91CEB030301F1CA
:100A8000FF382FD298422DD9023963441B1AADB2D8
:100A9000B3FBF7F007FB103345EA034500FB0EF309
:100AA000AB4208D91CEB050500F1FF3816D2AB426A
:100AB00014D902386544ED1A40EA014138E731465D
:100AC000304607E78646E5E61846FAE64B45A9D2E2
:100AD000B9EB020864EB0C0E0138A3E74046EAE7E5
:100AE000204694E74146D1E7D0467BE7023B654488
:100AF00032E7084609E76444023842E7704700BF1E
:100B0000844641EA000313F003036DD1403A41D318
:100B100051F8043B40F8043B51F8043B40F8043BD7
:100B200051F8043B40F8043B51F8043B40F8043BC7
:100B300051F8043B40F8043B51F8043B40F8043BB7
:100B400051F8043B40F8043B51F8043B40F8043BA7
:100B500051F8043B40F8043B51F8043B40F8043B97
:100B600051F8043B40F8043B51F8043B40F8043B87
:100B700051F8043B40F8043B51F8043B40F8043B77
:100B800051F8043B40F8043B51F8043B40F8043B67
:100B9000403ABDD2303211D351F8043B40F8043B07
:100BA00051F8043B40F8043B51F8043B40F8043B47
:100BB00051F8043B40F8043B103AEDD20C3205D317
:100BC00051F8043B40F8043B043AF9D2043208D00F
:100BD000D2071CBF11F8013B00F8013B01D30B8881
:100BE00003806046704700BF082A13D38B078DD05F
:100BF00010F003038AD0C3F10403D21ADB071CBF31
:100C000011F8013B00F8013B80D331F8023B20F89A
:100C1000023B7BE7043AD9D3013A11F8013B00F8D3
:100C2000013BF9D20B7803704B7843708B7883705B
:100C30006046704700000000000000000000000057
:100C4000A2EB0300704700BF02780B78012A28BF8F
:100C50009A42F5D16DE9044540EA0104CDE9026705
:100C60006FF0000C4FEA447212B380EA010414F0F2
:100C7000070F6AD100F0070420F0070004F0030515
:100C800021F007014FEAC505F0E8042314F0040F32
:100C9000F1E804670CFA05F462EA040266EA040665
:100CA0000AD063EA0403624667EA0407664603E083
:100CB000F0E80423F1E8046782FA4CF582EA0604BE
:100CC000A4FA8CF46CBB83FA4CF583EA0705A5FA09
:100CD0008CF595B950E9022351E9026782FA4CF587
:100CE00082EA0604A4FA8CF483FA4CF583EA070539
:100CF000A5FA8CF52543DBD09CB92DBAB5FA85F45D
:100D000024F0070427FA04F1DDE9026723FA04F36B
:100D100003F0FF0001F0FF01FDE80445A0EB010036
:100D2000704724BAB4FA84F424F0070426FA04F1D4
:100D3000DDE9026722FA04F202F0FF0001F0FF0190
:100D4000FDE80445A0EB0100704714F0030F3CD10F
:100D500010F0030428D150F8082B51F8083B82FA10
:100D60004CF582EA0305A5FA8CF55DB950F8042C20
:100D700051F8043C82FA4CF582EA0305A5FA8CF599
:100D8000002DE8D02DBAB5FA85F424F0070423FA33
:100D900004F122FA04F202F0FF0001F0FF01FDE885
:100DA0000445A0EB010070474FEAC40420F00300A3
:100DB00050F8082B21F0030151F8083B0CFA04F419
:100DC00062EA040263EA0403C9E710F003041AD0DC
:100DD000A1EB040120F00300E40750F8042B06D037
:100DE0000FD28B785FFAA2F4E41A06D12BB1CB783C
:100DF0005FFAB2F4E41A00D11BB920465DF8104B3B
:100E0000704701F1040150F8042BCC0721F00301D5
:100E100051F8043B48D824D222F07F4482FA4CF5A2
:100E200094EA1325A5FA8CF50AD165B951F8043B6B
:100E300084EA0204B4EB036F0ED150F8042BEBE705
:100E40004FEA132355E035F07F454DD10878FDE892
:100E50000445C0F1000070474FEA126203F0FF033F
:100E600047E002EA1C4482FA4CF594EA1345A5FADD
:100E70008CF50AD165B951F8043B84EA0204B4EB5D
:100E8000034F0CD150F8042BEBE74FEA134330E04B
:100E900015EA1C4528D10B884FEA124229E04FEA97
:100EA000124203EA1C4324E002F0FF0482FA4CF5EC
:100EB00094EA1365A5FA8CF50AD165B951F8043B9B
:100EC00084EA0204B4EB032F09D150F8042BEBE7BA
:100ED0004FEA13630DE015F0FF0F05D10B684FEAE1
:100EE000122223F07F4304E04FF00000FDE80445A8
:100EF000704712BA1BBA82FA4CF482EA0304A4FACD
:100F00008CF5B5FA85F402FA04F203FA04F34FEA19
:100F10001260FDE80445A0EB13607047000000007C
:100F200001F0FF01102A2BDB10F0070F08D010F89A
:100F3000013B013A8B422DD010F0070F42B3F6D19E
:100F4000F0B441EA012141EA014122F007047FF0B7
:100F500000070023F0E80256083C85EA010586EA0E
:100F6000010685FA47F5A3FA87F586FA47F6A5FA4A
:100F700087F68EB9EED1F0BC01F0FF0102F0070256
:100F800032B110F8013B013A83EA010313B1F8D101
:100F90000020704701387047002D06BF35460338E2
:100FA000073815F0010F07D1013015F4807F02BF1B
:100FB000013015F4C03F0130F0BC0138704700BF6C
:100FC00090F800F06DE9024520F007016FF0000C89
:100FD00010F0070491F820F040F049804FF0000431
:100FE0006FF00700D1E9002391F840F000F108000C
:100FF00082FA4CF2A4FA8CF283FA4CF3A2FA8CF344
:101000004BBBD1E9022382FA4CF200F10800A4FAAA
:101010008CF283FA4CF3A2FA8CF3E3B9D1E90423FE
:1010200082FA4CF200F10800A4FA8CF283FA4CF335
:10103000A2FA8CF37BB9D1E9062301F1200182FAEF
:101040004CF200F10800A4FA8CF283FA4CF3A2FAF5
:101050008CF3002BC6D0002A04BF04301A4612BA03
:10106000B2FA82F2FDE8024500EBD2007047D1E906
:10107000002304F00305C4F100004FEAC50514F095
:10108000040F91F840F00CFA05F562EA05021CBF66
:1010900063EA050362464FF00004A9E781F00041CE
:1010A00002E000BF83F0004330B54FEA41044FEA4D
:1010B000430594EA050F08BF90EA020F1FBF54EAE8
:1010C000000C55EA020C7FEA645C7FEA655C00F084
:1010D000E2804FEA5454D4EB5555B8BF6D420CDD55
:1010E0002C4480EA020281EA030382EA000083EAD8
:1010F000010180EA020281EA0303362D88BF30BD78
:1011000011F0004F4FEA01314FF4801C4CEA1131CD
:1011100002D0404261EB410113F0004F4FEA03332C
:101120004CEA133302D0524263EB430394EA050FB7
:1011300000F0A780A4F10104D5F1200E0DDB02FA26
:101140000EFC22FA05F2801841F1000103FA0EF2BA
:10115000801843FA05F359410EE0A5F120050EF180
:10116000200E012A03FA0EFC28BF4CF0020C43FAB1
:1011700005F3C01851EBE37101F0004507D54FF0BE
:10118000000EDCF1000C7EEB00006EEB0101B1F50E
:10119000801F1BD3B1F5001F0CD349085FEA300054
:1011A0004FEA3C0C04F101044FEA445212F5800F5F
:1011B00080F09A80BCF1004F08BF5FEA500C50F1FC
:1011C000000041EB045141EA050130BD5FEA4C0CDF
:1011D000404141EB0101013C28BFB1F5801FE9D23C
:1011E00091F0000F04BF01460020B1FA81F308BF5F
:1011F0002033A3F10B03B3F120020CDA0C3208DD2B
:1012000002F1140CC2F10C0201FA0CF021FA02F105
:101210000CE002F11402D8BFC2F1200C01FA02F175
:1012200020FA0CFCDCBF41EA0C019040E41AA2BF9A
:1012300001EB0451294330BD6FEA04041F3C1CDA62
:101240000C340EDC04F11404C4F1200220FA04F082
:1012500001FA02F340EA030021FA04F345EA03012C
:1012600030BDC4F10C04C4F1200220FA02F001FAEE
:1012700004F340EA0300294630BD21FA04F0294670
:1012800030BD94F0000F83F4801306BF81F4801109
:101290000134013D4EE77FEA645C18BF7FEA655C7C
:1012A00029D094EA050F08BF90EA020F05D054EA4E
:1012B000000C04BF1946104630BD91EA030F1EBF53
:1012C0000021002030BD5FEA545C05D14000494157
:1012D00028BF41F0004130BD14F580043CBF01F54A
:1012E000801130BD01F0004545F0FE4141F4700130
:1012F0004FF0000030BD7FEA645C1ABF194610460B
:101300007FEA655C1CBF0B46024650EA013406BF0B
:1013100052EA033591EA030F41F4002130BD00BFCA
:1013200090F0000F04BF0021704730B54FF4806487
:1013300004F132044FF000054FF0000150E700BF08
:1013400090F0000F04BF0021704730B54FF4806467
:1013500004F1320410F0004548BF40424FF0000154
:101360003EE700BF42004FEAE2014FEA31014FEA97
:1013700002701FBF12F07F4393F07F4F81F06051E6
:10138000704732F07F4208BF704793F07F4F04BF31
:1013900041F40021704730B54FF4607401F000450E
:1013A00021F000411CE700BF50EA010208BF70476E
:1013B00030B54FF000050AE050EA010208BF70475F
:1013C00030B511F0004502D5404261EB41014FF4C8
:1013D000806404F132045FEA915C3FF4D8AE4FF0D0
:1013E00003025FEADC0C18BF03325FEADC0C18BFB3
:1013F000033202EBDC02C2F1200300FA03FC20FA04
:1014000002F001FA03FE40EA0E0021FA02F1144450
:10141000BDE600BF70B54FF0FF0C4CF4E06C1CEA69
:1014200011541DBF1CEA135594EA0C0F95EA0C0FDA
:1014300000F0DEF82C4481EA030621EA4C5123EA4D
:101440004C5350EA013518BF52EA033541F480117C
:1014500043F4801338D0A0FB02CE4FF00005E1FB2F
:1014600002E506F00042E0FB03E54FF00006E1FB79
:1014700003569CF0000F18BF4EF0010EA4F1FF04BC
:10148000B6F5007F64F5407404D25FEA4E0E6D41FC
:1014900046EB060642EAC62141EA55514FEAC5200D
:1014A00040EA5E504FEACE2EB4F1FD0C88BFBCF589
:1014B000E06F1ED8BEF1004F08BF5FEA500E50F13A
:1014C000000041EB045170BD06F0004646EA010100
:1014D00040EA020081EA0301B4EB5C04C2BFD4EB32
:1014E0000C0541EA045170BD41F480114FF0000E2B
:1014F000013C00F3AB8014F1360FDEBF002001F099
:10150000004170BDC4F10004203C35DA0C341BDC12
:1015100004F11404C4F1200500FA05F320FA04F0E4
:1015200001FA05F240EA020001F0004221F0004118
:1015300010EBD37021FA04F642EB06015EEA430E8B
:1015400008BF20EAD37070BDC4F10C04C4F12005BB
:1015500000FA04F320FA05F001FA04F240EA02006E
:1015600001F0004110EBD37041F100015EEA430E3F
:1015700008BF20EAD37070BDC4F1200500FA05F25F
:101580004EEA020E20FA04F301FA05F243EA0203DE
:1015900021FA04F001F0004121FA04F220EA0200ED
:1015A00000EBD3705EEA430E08BF20EAD37070BD33
:1015B00094F0000F0FD101F00046400041EB010113
:1015C00011F4801F08BF013CF7D041EA060195F0F5
:1015D000000F18BF704703F00046520043EB0303AF
:1015E00013F4801F08BF013DF7D043EA060370479C
:1015F00094EA0C0F0CEA135518BF95EA0C0F0CD0A7
:1016000050EA410618BF52EA4306D1D181EA0301EC
:1016100001F000414FF0000070BD50EA410606BFE6
:101620001046194652EA430619D094EA0C0F02D12B
:1016300050EA013613D195EA0C0F05D152EA033670
:101640001CBF104619460AD181EA030101F000418E
:1016500041F0FE4141F470014FF0000070BD41F0D7
:10166000FE4141F4780170BD70B54FF0FF0C4CF4B1
:10167000E06C1CEA11541DBF1CEA135594EA0C0FD0
:1016800095EA0C0F00F0A7F8A4EB050481EA030E1D
:1016900052EA03354FEA013100F088804FEA033304
:1016A0004FF0805545EA131343EA12634FEA0222D2
:1016B00045EA111545EA10654FEA00260EF0004193
:1016C0009D4208BF964244F1FD0404F5407402D2E5
:1016D0005B084FEA3202B61A65EB03055B084FEA76
:1016E00032024FF480104FF4002CB6EB020E75EB73
:1016F000030E22BFB61A754640EA0C005B084FEA9B
:101700003202B6EB020E75EB030E22BFB61A754617
:1017100040EA5C005B084FEA3202B6EB020E75EB62
:10172000030E22BFB61A754640EA9C005B084FEADA
:101730003202B6EB020E75EB030E22BFB61A7546E7
:1017400040EADC0055EA060E18D04FEA051545EAD6
:1017500016754FEA06164FEAC30343EA52734FEA7F
:10176000C2025FEA1C1CC0D111F4801F0BD141EAF8
:1017700000014FF000004FF0004CB6E711F4801F5D
:1017800004BF01430020B4F1FD0C88BFBCF5E06F3D
:101790003FF6AFAEB5EB030C04BFB6EB020C5FEA4D
:1017A000500C50F1000041EB045170BD0EF0004EA2
:1017B0004EEA113114EB5C04C2BFD4EB0C0541EAD4
:1017C000045170BD41F480114FF0000E013C90E6D1
:1017D00045EA060E8DE60CEA135594EA0C0F08BF95
:1017E00095EA0C0F3FF43BAF94EA0C0F0AD150EA94
:1017F00001347FF434AF95EA0C0F7FF425AF104627
:1018000019462CE795EA0C0F06D152EA03353FF44E
:10181000FDAE1046194622E750EA410618BF52EACB
:1018200043067FF4C5AE50EA41047FF40DAF52EA9F
:1018300043057FF4EBAE12E74FF0FF3C06E000BF3C
:101840004FF0010C02E000BF4FF0010C4DF804CD49
:101850004FEA410C7FEA6C5C4FEA430C18BF7FEA09
:101860006C5C1BD001B050EA410C0CBF52EA430C37
:1018700091EA030F02BF90EA020F0020704710F1B7
:10188000000F91EA030F58BF994208BF90422CBF46
:10189000D8176FEAE37040F0010070474FEA410C3F
:1018A0007FEA6C5C02D150EA013C07D14FEA430C5D
:1018B0007FEA6C5CD6D152EA033CD3D05DF8040BCE
:1018C000704700BF8446104662468C461946634600
:1018D00000E000BF01B5FFF7B7FF002848BF10F1D7
:1018E000000F01BD4DF808EDFFF7F4FF0CBF01201C
:1018F00000205DF808FB00BF4DF808EDFFF7EAFF98
:1019000034BF012000205DF808FB00BF4DF808ED52
:10191000FFF7E0FF94BF012000205DF808FB00BF47
:101920004DF808EDFFF7CEFF94BF012000205DF8D1
:1019300008FB00BF4DF808EDFFF7C4FF34BF0120DE
:1019400000205DF808FB00BF4FEA410C7FEA6C5CA9
:1019500002D150EA013C0AD14FEA430C7FEA6C5CA9
:1019600002D152EA033C02D14FF0000070474FF021
:10197000010070474FEA410212F5001215D211D54D
:101980006FF47873B3EB625212D94FEAC12343F07C
:10199000004343EA505311F0004F23FA02F018BFFE
:1019A000404270474FF00000704750EA013005D1C7
:1019B00011F0004008BF6FF0004070474FF000008A
:1019C000704700BF10B58AB00023079308930993AE
:1019D000009301930293039304930593069326487F
:1019E000264A02604FF4802242608360C360042272
:1019F000026103750122427582610377436283624B
:101A0000C3624FF480520263436380F8383001F0C0
:101A1000E3FE38BB0023079307A9174802F014F828
:101A200018BB174B0093062301930023029340F247
:101A3000FF7203920422049205938DF819306946CF
:101A40000D4801F0B1FA98B90B4C6946204601F0F7
:101A5000ABFA204601F086FD0A21204601F09CF8F1
:101A60000AB010BD00F019F9D4E700F016F9D8E774
:101A700000F013F9E8E700BFDC0900240020024071
:101A80000008302E10B5B8B00446002133913491CF
:101A9000359136913791C02202A808F081FD226865
:101AA0001F4B9A4201D038B010BD4FF400220023E2
:101AB000CDE902234FF400332B9302A804F01AFD62
:101AC00058BB184BD3F8D82042F02002C3F8D820D6
:101AD000D3F8D82002F020020092009AD3F8E02038
:101AE00042F00402C3F8E020D3F8E03003F004032E
:101AF0000193019B022333930323349300243594F1
:101B000033A9094803F0B0FC22462146122002F016
:101B10005FF8122002F092F8C5E700F0BEF8D0E7B7
:101B200000200240004402580008025800B583B06B
:101B30000B4BD3F8D82042F00102C3F8D820D3F8D9
:101B4000D83003F001030193019B002211460B20C2
:101B500002F03EF80B2002F071F803B05DF804FBD0
:101B6000004402582DE9F0418AB0002405940694FF
:101B7000079408940994304BD3F8E02042F0800297
:101B8000C3F8E020D3F8E02002F080020092009A2F
:101B9000D3F8E02042F00402C3F8E020D3F8E020BC
:101BA00002F004020192019AD3F8E02042F001020F
:101BB000C3F8E020D3F8E02002F001020292029A7A
:101BC000D3F8E02042F01002C3F8E020D3F8E02080
:101BD00002F010020392039AD3F8E02042F00202CE
:101BE000C3F8E020D3F8E03003F002030493049B31
:101BF000DFF848802246C621404603F049FD104DDB
:101C000022463021284603F043FDC62305930127D1
:101C1000069707940226089605A9404603F024FC7F
:101C20003023059306970794089605A9284603F0E4
:101C30001BFC0AB0BDE8F0810044025800000258C5
:101C40000008025810B584B0002400940194029456
:101C5000039402F015F801238DF800308DF801404F
:101C60004FF01052019212228DF808208DF8094091
:101C70008DF80A4003228DF80B208DF80C408DF86A
:101C80000D308DF80E308DF80F40684602F016F8D2
:101C9000042002F003F804B010BD72B6FEE70000A5
:101CA00000B59FB04C2200210BA808F079FC20223F
:101CB000002103A808F074FC022003F0EFFC0023CD
:101CC00000933A4BDA6A22F00102DA62DB6A03F02F
:101CD00001030093364B9A6942F440429A619B6932
:101CE00003F440430093009B314B9B6913F4005F66
:101CF000FAD0304BD3F8F42042F00202C3F8F420BB
:101D0000D3F8F43003F002030193019B0023029304
:101D1000274B9A6942F440429A619B6903F440431D
:101D20000293224BDA6A42F00102DA62DB6A03F0C4
:101D300001030293029B1E4B9B6913F4005FFAD0D0
:101D400003230B934FF480330C9301230E93402312
:101D50000F930223149315931693F022179218935E
:101D600019931A9308231B9300231C931D930BA80C
:101D700003F0BEFCB0B93F23039303230493002375
:101D80000593082306934023079308934FF480623A
:101D900009920A93042103A804F010F920B91FB096
:101DA0005DF804FBFFF779FFFFF777FF00040058A9
:101DB000004802580044025800B5B1B0C0220021CA
:101DC000684608F0EDFB4FF000420023CDE9002308
:101DD000684604F08FFB10B931B05DF804FBFFF7E3
:101DE0005CFF0000F8B5FFF72DFF794B5B6913F43A
:101DF000003F13D1BFF34F8FBFF36F8F744B00229F
:101E0000C3F85022BFF34F8FBFF36F8F5A6942F46C
:101E100000325A61BFF34F8FBFF36F8F6C4B5B691A
:101E200013F4803F27D16A4B0022C3F88420BFF30C
:101E30004F8FD3F88040C4F34E3000E01846C4F30F
:101E4000C90243F6E07303EA401343EA8273604930
:101E5000C1F860321346013A002BF2D1431E00282C
:101E6000ECD1BFF34F8F4B6943F480334B61BFF329
:101E70004F8FBFF36F8F00F049FEFFF711FFFFF7A1
:101E80009BFFFFF76FFEFFF751FE00F00FFA00F027
:101E900011FC00F0EFFC00F0BFFAFFF793FD00F03B
:101EA00061FA00214B4806F059FD01252F46002418
:101EB000264658E04849494808F0D8FB4849FEF70B
:101EC000C3FE38B10021474B1980C822434808F0AF
:101ED00067FB4DE0404908F0C9FB4349FEF7B4FEFB
:101EE0000028EFD13C4908F0C1FB08F02BFB3F4B29
:101EF00018603F4808F0A6FBE4E73E4A32F81300BA
:101F00003D4951F82320024441F823200133B3F521
:101F1000007FF2DB394B1F6896FBF7F307FB136377
:101F2000002B40D001362F460025354B1A682F4B29
:101F30001B689A4202DD324B00221A60012F14BF47
:101F4000002304F0010373B172B62D4A1368013304
:101F5000136000242B4B1C602B4B1C602B4B1C6014
:101F600062B6012527461F4BB3F90030002BA1DBD9
:101F7000244B1B68B3F5026F00DB0124234B1B6865
:101F8000B3F5007FD1DB002DCFD00023BFE71A4986
:101F900051F82320B2FBF7F21D4820F8132000224D
:101FA00041F823200133B3F5007FF0DB194FFF2305
:101FB0003B707B704FF480621549B81CFEF7A0FDA2
:101FC00040F202423946144806F0ECFEAAE700BF90
:101FD00000ED00E05827002408060108F827002437
:101FE0000C060108C0280024100601084C0A002431
:101FF00014060108681A002460120024000000245E
:10200000F0270024400A0024480A0024440A00243F
:10201000600E0024500A00243C290024022801D824
:102020000120704708B508F091FA092303600020E9
:1020300008BD000010B5013801280AD814464FF039
:10204000FF3392B20748006807F09AFF40B9204674
:1020500010BD08F07BFA092303604FF0FF30F7E76B
:102060000520F5E7601A0024022801D800207047F7
:1020700008B508F06BFA092303604FF0FF3008BD84
:1020800008B508F063FA092303604FF0FF3008BD7C
:1020900008B548B94FF0FF3301220848006807F03F
:1020A000D7FF40B9012008BD08F050FA09230360AA
:1020B0004FF0FF30F7E70520F5E700BF601A002476
:1020C00008B5022804D84FF400534B60002008BD27
:1020D00008F03CFA09230360F8E7000082B0074BE0
:1020E000D3F8F42042F00202C3F8F420D3F8F4301D
:1020F00003F002030193019B02B0704700440258B1
:10210000FEE7FEE7FEE7FEE7FEE770477047704731
:1021100008B500F029FD08BD08B5024802F008FE28
:1021200008BD00BFC428002408B5024800F0D0FD57
:1021300008BD00BFDC09002408B5024805F0AFFF68
:1021400008BD00BFC026002408B5024805F0A7FF5F
:1021500008BD00BFC026002408B5024805F09FFF57
:1021600008BD00BFA427002408B5024806F0DCFE25
:1021700008BD00BF3C29002408B5024805F08FFFC8
:1021800008BD00BF0C2700240120704708B508F0E7
:10219000DDF9162303604FF0FF3008BD08B54FF09E
:1021A000FF31FFF7F3FFFEE710B503460C4A0D4978
:1021B0000D48006840B10C4800680344521A93422D
:1021C00006D8094A136010BD0748084C0460F2E7BE
:1021D00008F0BCF90C2303604FF0FF30F3E700BFB9
:1021E0000000082400040000641A0024202A0024AF
:1021F000244B1B6803F00F03062B06D8214A1368F3
:1022000023F00F0343F0070313601F4B1A6842F0DB
:1022100001021A6000221A6119681C4A0A401A60F9
:10222000184B1B6813F0080F06D0164A136823F0EA
:102230000F0343F007031360134B00229A61DA6126
:102240001A62134999621349D962134919635A638F
:102250009963DA6319645A64196821F4802119605A
:102260001A660E4B1A680E4B1340B3F1005F03D28F
:102270000C4B0122C3F808210B4B43F2D2021A6027
:10228000704700BF00200052004402587FEDF6EA7C
:10229000000202020000FF01800201010010005C48
:1022A0000000FFFF008000510040005200B58DB0DB
:1022B00000230793089309930A930B9304930593C0
:1022C000069300930193029303932448244A0260E7
:1022D0001722426083604FF6FF72C2600361436160
:1022E000836106F02BF850BB1C4806F087F848BB0A
:1022F0000423079350230893002309930B9307A902
:10230000164806F0F3FA00BB0023049305930693E6
:1023100004A9124806F0AEFCD0B9002200920123B5
:1023200001930292039269460C4806F0C9F990B9EC
:1023300000210A4806F0C6FB0DB05DF804FBFFF76C
:10234000ACFCD1E7FFF7A9FCD2E7FFF7A6FCDBE77F
:10235000FFF7A3FCE1E7FFF7A0FCE9E7C0260024B4
:102360000000014000B58DB0002307930893099346
:102370000A930B930493059306930093019302939E
:1023800003932348234A02601722426083604FF67A
:10239000FF72C2600361836105F0D0FF48BB1C4837
:1023A00006F02CF840BB0423079350230893002326
:1023B00009930B9307A9164806F098FAF8B9002379
:1023C0000493069304A9124806F054FCD0B90022E5
:1023D0000092012301930292039269460C4806F091
:1023E0006FF990B900210A4806F06CFB0DB05DF85A
:1023F00004FBFFF752FCD2E7FFF74FFCD3E7FFF7F0
:102400004CFCDCE7FFF749FCE1E7FFF746FCE9E7B6
:10241000A42700240004004000B58DB000230793DA
:10242000089309930A930B930493059306930093DF
:102430000193029303932448244A026017224260C6
:1024400083604FF6FF72C2600361836105F076FF1F
:1024500058BB1D4805F0D2FF50BB042307935023FF
:1024600008930223099300230B9307A9164806F04B
:102470003DFA00BB00230493069304A9124806F01A
:10248000F9FBD8B9022300930123019300220292A1
:10249000039269460C4806F013F990B900210A48E6
:1024A00006F010FB0DB05DF804FBFFF7F6FBD0E77C
:1024B000FFF7F3FBD1E7FFF7F0FBDBE7FFF7EDFBFF
:1024C000E0E7FFF7EAFBE9E70C27002400180040EB
:1024D00000B58DB000230793089309930A930B93DB
:1024E00003684C4A934208D04B4A93423AD04B4A35
:1024F000934262D00DB05DF804FB494BD3F8F02055
:1025000042F00102C3F8F020D3F8F02002F00102FB
:102510000192019AD3F8E02042F01002C3F8E020C3
:10252000D3F8E03003F010030293029B4FF40073E2
:1025300007930223089301230B9307A9394802F05C
:1025400093FF002211461A2001F042FB1A2001F0ED
:1025500075FB002211461B2001F03AFB1B2001F005
:102560006DFBC7E72E4BD3F8E82042F00202C3F818
:10257000E820D3F8E82002F002020392039AD3F88D
:10258000E02042F00402C3F8E020D3F8E03003F08A
:1025900004030493049B40230793022308930B93A3
:1025A00007A9214802F060FF002211461D2001F01A
:1025B0000FFB1D2001F042FB9CE7194BD3F8E820EC
:1025C00042F04002C3F8E820D3F8E82002F04002CD
:1025D0000592059AD3F8E02042F00202C3F8E02009
:1025E000D3F8E03003F002030693069B4FF48043D8
:1025F0000793022308930B9307A90C4802F034FFBA
:10260000002211462B2001F0E3FA2B2001F016FBEB
:1026100070E700BF000001400004004000180040C7
:1026200000440258001002580008025800040258E2
:102630000368B3F1804F00D0704782B0074BD3F8E6
:10264000E82042F00102C3F8E820D3F8E83003F0B4
:1026500001030193019B02B0704700BF0044025880
:1026600000B587B00023019302930393049305936D
:102670000368B3F1804F02D007B05DF804FB0B4B49
:10268000D3F8E02042F00102C3F8E020D3F8E030B4
:1026900003F001030093009B0123019302220292A5
:1026A000059301A9024802F0DFFEE5E70044025865
:1026B0000000025800B58BB00023079308930993DC
:1026C0000093019302930393049305930693184890
:1026D0004FF0804202601722426083606422C26031
:1026E0000361836105F05AFEC8B90023079309937B
:1026F00007A90F4806F0BEFAA0B960230093322361
:1027000001930022029204926946094805F0F0FE06
:1027100058B90748FFF7A4FF0BB05DF804FBFFF7BB
:10272000BCFAE2E7FFF7B9FAE7E7FFF7B6FAF0E736
:102730005827002438B504460268434B9A4204D017
:102740002268424B9A424FD038BD037F012BF7D10C
:102750003F4B1B6833B33E4B1B68012B28D03D4BCE
:102760001A683D4B1B689A4234DA394B1B68012BBF
:1027700004DD374B1B68B3F5C87F1FDB344B1B6888
:10278000B3F5C87F04DB324B1B68B3F5AF6F1BDBBF
:1027900001224021314802F07BFF2D4A13680133AA
:1027A0001360CDE7012204212C4802F071FFD2E72B
:1027B00000220421294802F06BFFD0E701224021CA
:1027C000264802F065FFE8E700224021234802F096
:1027D0005FFFE2E71E4B1B68012BDEDD012240217B
:1027E0001E4802F055FFD8E7237F012BACD11C48CF
:1027F00000F068FA1B4A11681B4B23F8110012689D
:1028000033F812204EF660239A4206D9154B1A6807
:10281000154B4EF6602123F81210124B1A68124C19
:1028200034F81210114A1568090A114841551D68FB
:102830001168013114F815404454116802311160D7
:102840001A6801321A607FE700000140000400406E
:10285000400A0024F02700244C0A002400000258FB
:10286000DC090024440A0024681A0024480A0024D1
:10287000A01E002408B51A481A4B03604FF46123C8
:10288000436000238360C36003610C224261836163
:10289000C36103624362836207F0CAFC98B90021F6
:1028A0000F4807F005FE88B900210D4807F025FE06
:1028B00078B90B4807F0DDFD70B901220A490848D4
:1028C00007F088FD08BDFFF7E8F9E8E7FFF7E5F94D
:1028D000EAE7FFF7E2F9ECE7FFF7DFF9EDE700BF22
:1028E0003C29002400100140F427002430B5B9B081
:1028F0000446002133913491359136913791C022AD
:1029000002A807F04DFE2268304B9A4201D039B040
:1029100030BD01220023CDE9022302A803F0EAFD25
:1029200000284CD12A4BD3F8F02042F01002C3F813
:10293000F020D3F8F02002F010020092009AD3F8B1
:10294000E02042F00102C3F8E020D3F8E03003F0C9
:1029500001030193019B4FF4C0633393022334932B
:102960000025359536930723379333A9194802F08C
:102970007BFD1948194B03602A2343604023836081
:10298000C5604FF480630361456185614FF48073D6
:10299000C3614FF480330362456201F0D3FB88B911
:1029A0000D4BE3679C6300221146252001F010F9CE
:1029B000252001F043F9E06F01F0C4FBA7E7FFF722
:1029C0006CF9AFE7FFF769F9EAE700BF00100140D3
:1029D0000044025800000258C4280024100002409D
:1029E00008B502681A4B9A4200D008BD194A1388EC
:1029F000B2F90020002A09DB13F4804F11D0164AE7
:102A000012780A2A08D0134B00221A800122124998
:102A1000124807F0DFFCE8E7114A1A430D4B1A8011
:102A2000F4E70D4A12780D2A0DD0C3F30D010D48BD
:102A3000425401339BB2074A1380C72BE6D9134691
:102A400000221A80E2E743F48043024A1380DDE764
:102A500000100140C0280024F42700243C29002451
:102A60000080FFFFF8270024DFF834D0FFF7C0FB19
:102A70000C480D490D4A002302E0D458C4500433D9
:102A8000C4188C42F9D30A4A0A4C002301E01360AF
:102A90000432A242FBD307F05FFDFFF7A3F97047B2
:102AA0000000082400000024C0090024680A01086E
:102AB000C00900241C2A0024FEE70000104B1B78EC
:102AC0000BB90120704710B504464FF47A70B0FB83
:102AD000F3F30C4A1068B0FBF3F001F0BDF868B9ED
:102AE0000F2C01D901200AE0002221464FF0FF30CF
:102AF00001F06EF8044B1C60002000E0012010BDC6
:102B00000C000024040000241000002410B5032051
:102B100001F04CF803F046F90F498B69C3F3032326
:102B20000E4AD35C03F01F03D8408B6903F00F03F8
:102B3000D35C03F01F0320FA03F3094A1360094B27
:102B400018600F20FFF7BAFF10B10124204610BD16
:102B50000446FFF7C3FAF9E70044025818060108D3
:102B60000800002404000024034B1B78034A11686A
:102B70000B441360704700BF0C000024D0290024D0
:102B8000014B1868704700BFD0290024014B18681A
:102B9000000C70470010005C2DE9F04104460E4621
:102BA00003684549454A934218BF8B4213D102F549
:102BB0000072976807F01F072569082D12D0052FAE
:102BC00018BF002F09D0092F07D0936813F4404F86
:102BD0002DD1042506E03A4AEBE7DB6813F0010F3C
:102BE0001FD10425FFF7CCFF804623681A682A42CC
:102BF00023D1B6F1FF3FF8D0FFF7C2FFA0EB0800EA
:102C0000B04201D8002EF0D123681B682B42ECD1D2
:102C1000636D43F004036365002384F850300320A0
:102C200045E0636D43F02003636501203FE0636D81
:102C300043F020036365012039E0626D42F40072C5
:102C40006265DA6812F4406F11D1627D7AB91A6850
:102C500012F0080F0BD0626D22F480726265626D13
:102C600012F4805F03D1626D42F001026265134A83
:102C700093420CD01A4693420CD0052F14BF00216A
:102C800001213FB131B9092F04D0D26803E0A2F588
:102C90008072F0E7DA68082D06D012F4804F08D170
:102CA0000C221A60002002E008221A600020BDE811
:102CB000F0810020FBE700BF00200240002102401D
:102CC000006302580368186C70477047704770477C
:102CD000F8B5044603681D685E689649964A9342B3
:102CE00018BF8B4240D1954B9F6807F01F0715F026
:102CF000020F10D016F0020F0DD0636D13F0100FFD
:102D000003D1636D43F400636365204600F09AFECF
:102D1000236802221A6015F0040F02D016F0040F87
:102D200005D115F0080F4FD016F0080F4CD0636D89
:102D300013F0100F03D1636D43F4007363652368D0
:102D4000DA6812F4406F39D17B4A93420ED01A46AA
:102D500093420ED0052F14BF002101214FB141B97C
:102D6000092F06D0D26805E0754BBDE7A2F5807249
:102D7000EEE7DA6812F4005F20D11A6812F0080F4B
:102D80001CD09A6812F0040F10D15A6822F00C027D
:102D90005A60636D23F480736365636D13F4805F21
:102DA0000CD1636D43F00103636507E0636D43F08D
:102DB00010036365A36D43F00103A3652046FFF78D
:102DC00084FF23680C221A6015F0200F02D016F041
:102DD000200F05D115F0400F63D016F0400F60D0E2
:102DE000636D13F0100F03D1636D43F400536365FB
:102DF0002368DA6C12F4C07F19D10121DA6812F469
:102E0000406F16D101204C4A934214D01A46934287
:102E100014D0062F14BF4FF0000C4FF0010C6FB10F
:102E2000BCF1000F0AD1072F08D0D26807E00021BB
:102E3000E4E70020E7E7A2F58072E8E7DA6851B33B
:102E400012F0007F03D030B312F4005F23D1196871
:102E500011F0400F1FD012F4001F1CD19A6812F01D
:102E6000080F10D15A6822F060025A60636D23F493
:102E700080536365636D13F4807F0CD1636D43F001
:102E80000103636507E0636D43F010036365A36DA1
:102E900043F00103A365204600F0D0FD23686022C3
:102EA0001A6015F0800F02D016F0800F36D115F49D
:102EB000807F02D016F4807F44D115F4007F02D0C9
:102EC00016F4007F4AD115F0100F20D016F0100F25
:102ED0001DD0236B6BB1002F4ED023681549164AC5
:102EE000934218BF8B4245D1144B9B6813F4404F5B
:102EF0000AD0636D43F480636365A36D43F00203FE
:102F0000A3652046FFF7E3FE236810221A6015F43C
:102F1000806F02D016F4806F34D1F8BD636D43F436
:102F2000803363652046FFF7D1FE236880221A6054
:102F3000BDE700BF00200240002102400023024004
:102F400000630258636D43F400336365204600F06C
:102F500077FD23684FF480721A60AEE7636D43F427
:102F600080236365204600F06CFD23684FF40072F7
:102F70001A60A8E70B4BB8E72368DB6813F0030F70
:102F8000C2D0B6E7636D43F480436365A36D43F03D
:102F90000803A36523684FF480621A60204600F09E
:102FA0004EFDBAE700630258F0B583B000220192EB
:102FB00090F85020012A00F055820346012280F843
:102FC00050200068826812F0040F09D05A6D42F058
:102FD00020025A650120002283F8502003B0F0BD82
:102FE0000A68C2F31304002C4ED1C2F38462012498
:102FF0009440C2692243C2611D684C683035220A80
:10300000920002F00C02A85804F01F0E1F2404FACC
:103010000EF420EA04000C68C4F3846C0CFA0EFC75
:1030200040EA0C00A8501C68A26812F0040200D00C
:103030000122A06810F0080000D0012002432FD028
:103040001868826812F0010F40F008820A68CD68A3
:10305000D0F8C040C2F3130624EA060405F0180CA9
:10306000B24D25FA0CF52A40C2F313022243C0F8F0
:10307000C020C868AE4A904200F0B0800A68002ABA
:10308000C0F26B810020A6E792FAA2F232B1B2FA46
:1030900082F202F01F0201249440AAE72022F8E7FE
:1030A0000F688D681434780E800000F004002658F4
:1030B000C7F3045E4FF0070C0CFA0EFC26EA0C0C6A
:1030C00005FA0EF54CEA050525509A48006800F00F
:1030D0007040B0F1805F0BD01C68E06810F0100FFA
:1030E00039D14869E468C4F382046400A04006E072
:1030F00048691C68E468C4F382046400A0400D6958
:10310000042D36D01F680E68603757F8254004F04C
:10311000004406F0F8463043204347F8250018687D
:103120000E694C7E012C1ED01546603050F82640AA
:1031300024F000442C4340F826401D680C69087EAA
:10314000012813D0286920F4F04004F01F04A240A5
:1031500002432A6174E74869E468A40804F004049F
:103160006400A040CBE74FF00045DEE74FF400627B
:10317000E8E71868026E02F0F8420C68B2EB846F60
:103180001DD01868426E02F0F8420C68B2EB846FF2
:103190001AD01868826E02F0F8420C68B2EB846FA5
:1031A00017D01868C26E02F0F8420C68B2EB846F58
:1031B0007FF446AFC26E22F00042C26640E7026E64
:1031C00022F000420266DCE7426E22F000424266D4
:1031D000DFE7826E22F000428266E2E71C680A683E
:1031E000C2F31305002D34D1900E013000F01F0002
:1031F00009288CBF00200120002861D0002D37D184
:10320000900E0130800600F0F840002D3CD1960E63
:10321000013606F01F070126BE403043002D41D184
:10322000920E013202F01F0202EB4202120502432B
:1032300088681434550EAD0005F004056659C2F3D4
:1032400004520727974026EA070690403043605112
:1032500014E792FAA2F048B1B0FA80F0013000F021
:103260001F0009288CBF00200120C5E72020F5E7BA
:1032700092FAA2F030B1B0FA80F00130800600F08E
:10328000F840C2E72020F8E792FAA2F646B1B6FA73
:1032900086F6013606F01F06012707FA06F6BCE798
:1032A0002026F6E792FAA2F242B1B2FA82F2013295
:1032B00002F01F0202EB42021205B8E72022F6E7F5
:1032C000CDB9900E0130800600F0F840FDB9960EA1
:1032D000013606F01F070126BE40304365BB920E43
:1032E000013202F01F0202EB42021E3A120542F0C6
:1032F000007202439CE792FAA2F030B1B0FA80F07B
:103300000130800600F0F840E0E72020F8E792FA6C
:10331000A2F646B1B6FA86F6013606F01F06012778
:1033200007FA06F6D9E72026F6E700BFFFFF0F00F1
:103330000000FF470010005C92FAA2F25AB1B2FA04
:1033400082F2013202F01F0202EB42021E3A120523
:1033500042F00072CDE72022F3E719684248434C5F
:10336000A14218BF81420CBF0120002021D1404E54
:10337000B56805F0E077F0B13B48806810F00100D7
:1033800000D00120394CA46814F0010400D00124BD
:1033900020430CBF01200020002859D0354882422C
:1033A00012D03548824231D0344882423FD000208A
:1033B00011E6334EDCE73348806810F0010000D09E
:1033C000012080F00100E7E715F4000FE9D12D4A54
:1033D000914201D00020FEE547F40002B16821F0DF
:1033E000E0710A43B260284A126892092749A1FB9A
:1033F0000212920901325200019202E0019A013A4E
:103400000192019A002AF9D10020E4E515F0807FAD
:10341000CAD11C4A914201D00020DCE547F08072FD
:10342000B16821F0E0710A43B2600020D3E515F4E1
:10343000800F15D1134A914201D00020CBE547F40B
:103440008002B16821F0E0710A43B2600020C2E559
:103450005A6D42F020025A650120BCE50020BAE511
:103460000020B8E50220B9E500200240002102401A
:1034700000230240000084CB000052C70000B8CFF8
:10348000006302580060025804000024632D3E05CA
:1034900038B503689A6812F0010F56D1044699684E
:1034A0002B4A114209D0436D43F010034365836DED
:1034B00043F001038365012048E09968254A0A40EA
:1034C00042F001029A60FFF75BFB05462368224940
:1034D000224A934218BF8B420DD102F500729268C6
:1034E00002F01F021D498B4207D01946994207D0AE
:1034F00032B100202AE01A4AF1E7A1F58071F5E720
:1035000023681A6812F0010F1DD19A6812F0010F9A
:1035100005D199680F4A0A4042F001029A60FFF70C
:103520002FFB401B0228EBD923681B6813F0010F07
:10353000E6D1636D43F010036365A36D43F00103AF
:10354000A365012002E0002000E0002038BD00BF9C
:103550003F000080C0FFFF7F0020024000210240AA
:103560000063025838B5044603683E493E4A934218
:1035700018BF8B4252D102F50072956805F01F0505
:103580009B6813F0040F69D194F85030012B67D079
:10359000012384F850302046FFF77AFF002859D1E4
:1035A000626DA0F60273134043F480736365236871
:1035B0002D4A934234D01A46934200D01DB9626D11
:1035C00022F480126265626D12F4805F2BD0A26DCE
:1035D00022F00602A2651C221A60002384F85030F3
:1035E0002368214A934221D01A46934221D0052DC7
:1035F00014BF00210121E5B1D9B9092D19D0636D9E
:1036000043F480136365D36813F0007F27D0636DA4
:1036100023F4405343F48053636520E0134AACE73E
:10362000A2F58072C8E70022A265D4E7A2F58072F5
:10363000DBE7DA6812F0007F05D0626D22F44052B9
:1036400042F4805262659968094A0A4042F00402D5
:103650009A6004E0002384F8503000E0022038BD76
:103660000220FCE7002002400021024000630258D3
:10367000C0FFFF7F38B5044603684F494F4A934265
:1036800018BF8B4223D14E4B9B6813F4403F14BFAD
:10369000012300234BB302F0DBFD05466368B3F55D
:1036A000003F1CD0B3F5403F1DD0B3F5803F16D08E
:1036B000FFF76CFA41F20303984258D8414B9D4200
:1036C0004FD92268936843F48073936038BD3E4BB2
:1036D0009B6813F4403F14BF01230023DAE71B0C5F
:1036E000B5FBF3F5E4E78508E2E74FF4002000219D
:1036F00003F0A6FF05466368B3F5101F2DD022D84E
:10370000B3F5E01F27D004D9B3F5001FD0D1450988
:10371000CEE7B3F5801F0DD006D9B3F5A01F09D0B1
:10372000B3F5C01F06D0C3E7B3F5002F02D0B3F541
:10373000402F04D19B0C5B00B5FBF3F5B8E7B3F564
:10374000802FF7D0B4E7B3F5201F08D0B3F5301FB2
:10375000AED1050AACE70509AAE78509A8E7C509BE
:10376000A6E72268936823F480739360AEE7174B53
:103770009D4205D82268936823F440739360A5E7BF
:10378000134B9D4207D82268936823F4407343F497
:10379000807393609AE70F4B9D4207D82268936825
:1037A00023F4407343F4007393608FE722689368B7
:1037B00043F44073936089E70020024000210240F7
:1037C00000230240002D31010063025821BCBE00DD
:1037D00041787D0181F0FA0230B583B00023019376
:1037E000002800F010810446436DEBB123689A680D
:1037F00012F0005F03D09968844A0A409A602368F7
:103800009A6812F0805F1CD19968814A0A4042F0A0
:1038100080529A607F4B1B689B097F4AA2FB03235F
:103820009B090133019309E0FEF72CF90023A365FE
:1038300084F85030DAE7019B013B0193019B002B98
:10384000F9D12268936813F0805F40F09C80636D2B
:1038500043F010036365A36D43F00103A3650125E5
:10386000936813F0040300D00123616D11F0100F71
:1038700040F0C180002B40F0BE80636D23F4817363
:1038800043F002036365936813F0010F21D163498C
:10389000634B9A4218BF8A420CBF0122002274D1A6
:1038A0008B6813F0010300D001235D49896811F092
:1038B000010100D001210B430CBF0123002343B1C0
:1038C000002A6BD0574963688A6822F47C1213433C
:1038D0008B60FFF75BF941F20303984202D9A368BA
:1038E000102B5DD0627D236B43EA4233A268134301
:1038F000227F43EA0243227F012A5CD0626A22B11E
:1039000002F47872A16A0A4313432168C868464AE0
:1039100002401343CB6021688B6813F0040300D08E
:1039200001238A6812F0080200D0012213431BD140
:10393000227DE36A43EA8232C8683C4B034013436A
:10394000CB6094F83830012B3AD02268136923F009
:10395000010313612268136923F07043616B0B4309
:1039600013612046FFF786FEE368012B3AD02268F8
:10397000136B23F00F031363636D23F0030343F012
:10398000010363653CE000256AE7294B9B6813F05F
:10399000010300D0012383F0010390E7254992E75A
:1039A000617D226B42EA41321343227F43EA0243A4
:1039B00043F00C039FE7226A013A43EA42439DE742
:1039C000206802691C4B1340E26B511E226C42EAD4
:1039D0000142616C0A43A16C0A43134343F00103A3
:1039E0000361B7E721680B6B23F00F03A269013A6B
:1039F00013430B63C0E7636D43F010036365012558
:103A0000284603B030BD0125FAE700BFC0FFFF5FC5
:103A1000C0FFFF6F04000024632D3E05002002401C
:103A2000002102400023024003C0F0FFFCBFFFFF63
:103A300000600258006302581EF800FC704770478F
:103A4000704770477047000090F85020012A00F03E
:103A5000A18030B49AB00346012280F850200022A1
:103A60001692179200684C4A904242D0002201926E
:103A7000019A002A41D0926812F0040200D001227B
:103A8000846814F0040F76D1002A74D1424C434A62
:103A9000904218BFA04239D102F500720868002890
:103AA0003FD0906820F440404C68204390601868F4
:103AB000394D3A4CA04218BFA84229D1A86810F04D
:103AC000010000D00120354CA46814F0010400D09E
:103AD000012420430CBF01200020002856D0946808
:103AE0002F4820400C6889682143084390600020DB
:103AF00046E002F580720192BAE75A6D42F0200268
:103B00005A65002283F8502001203CE0254AC5E791
:103B10002548806810F0010000D0012080F00100ED
:103B2000DBE7916821F44041916019681A4C1B4809
:103B3000814218BFA14215D1A16811F0010100D046
:103B400001211648806810F0010000D001200143D7
:103B50000CBF01210021D9B1906811490140916049
:103B600000200DE01049896811F0010100D0012109
:103B700081F00101EFE75A6D42F020025A65012001
:103B8000002283F850201AB030BC70470020F7E7BD
:103B90000020F5E70220704700200240002102408B
:103BA000E0F0FFFF00630258006002580649CB684E
:103BB00023F4E0631B041B0C000200F4E0600343E9
:103BC000024A1A43CA60704700ED00E00000FA059F
:103BD00000B5174BDB68C3F30223C3F1070CBCF13C
:103BE000040F28BF4FF0040C03F1040EBEF1060FC2
:103BF00014D9033B4FF0FF3E0EFA0CFC21EA0C01F6
:103C000099400EFA03F322EA03031943002807DB65
:103C10000901C9B2074B19545DF804FB0023E9E719
:103C200000F00F000901C9B2034B1954F4E700BFBB
:103C300000ED00E000E400E014ED00E0002807DB08
:103C400000F01F02400901239340024A42F820304D
:103C5000704700BF00E100E00138B0F1807F0BD277
:103C60004FF0E0235861054AF02182F8231000202C
:103C7000986107221A6170470120704700ED00E04B
:103C8000BFF35F8F044B5A6A22F480325A620022DB
:103C9000C3F89420704700BF00ED00E040F0010041
:103CA000054BC3F894005A6A42F480325A62BFF35B
:103CB0004F8FBFF36F8F704700ED00E04278164BD7
:103CC000C3F898200378FBB14368134AC2F89C30CC
:103CD000017BC37A1B0643EA0173817A43EAC1433D
:103CE000417B43EA8143817B43EA4143C17B43EA11
:103CF0000143417A43EA0123017A43EA410301780F
:103D00000B43C2F8A0307047034B0022C3F89C203D
:103D1000C3F8A020704700BF00ED00E0F0B4876D4D
:103D20000468664E664DAC4218BFB44242D01835A6
:103D3000AC423FD01835AC423CD01835AC4239D0FB
:103D40001835AC4236D01835AC4233D01835AC42B9
:103D500030D005F55675AC422CD01835AC4229D080
:103D60001835AC4226D01835AC4223D01835AC42B9
:103D700020D01835AC421DD01835AC421AD01835B9
:103D8000AC4217D04F4DAC4214D01435AC4211D0D8
:103D90001435AC420ED01435AC420BD01435AC42C5
:103DA00008D01435AC4205D01435AC4202D01435DD
:103DB000AC4207D1446E856E6560C46E14B1046F69
:103DC000456F656004683D4E3D4DAC4218BFB4423E
:103DD00052D01835AC424FD01835AC424CD01835C3
:103DE000AC4249D01835AC4246D01835AC4243D02D
:103DF0001835AC4240D005F55675AC423CD018356C
:103E0000AC4239D01835AC4236D01835AC4233D03C
:103E10001835AC4230D01835AC422DD01835AC42F4
:103E20002AD01835AC4227D0264E274DAC4218BFB9
:103E3000B44211D0254DAC420ED01435AC420BD05B
:103E40001435AC4208D01435AC4205D01435AC4220
:103E500002D01435AC4224D1C46D04F01F050124F6
:103E6000AC407C60046863608368402B20D00368AA
:103E700099600368DA6014E0C46D04F01F0C3F24FD
:103E800004FA0CF4BC6005682C6824F480242C60CF
:103E9000046863608368402B05D0036899600368F9
:103EA000DA60F0BC704703689A600368D960F8E78D
:103EB00003689A600368D960F3E700BF100002400E
:103EC00028000240085402581C540258305402582A
:103ED00003682749274A934218BF8B422FD01832D4
:103EE00093422CD01832934229D01832934226D0D4
:103EF0001832934223D01832934220D01832934282
:103F00001DD002F55672934219D01832934216D042
:103F10001832934213D01832934210D01832934281
:103F20000DD0183293420AD01832934207D018327B
:103F3000934204D023F0FF038365806D704710B473
:103F4000D9B210390C4AA2FB0142C2F302120B4C47
:103F5000A25CC2655F2906D9094A1A40043282650B
:103F6000806D10BC7047064A1A408265F8E700BFB2
:103F70001000024028000240ABAAAAAA28060108A5
:103F800000FCFFFF83699BB9836A012B0AD0022BD7
:103F900002D00BB100207047C36A13F0807F2AD192
:103FA00000207047C36AB3F1C07F26D0002070475D
:103FB000B3F5005F0AD0836A022B26D9032B26D1E2
:103FC000C36A13F0807F24D100207047836A032BDB
:103FD00003D8DFE803F01404140A00207047C36A12
:103FE00013F0807F0DD100207047C36AB3F1C07F0A
:103FF00009D0002070470120704701207047012040
:104000007047012070470120704701207047002051
:10401000704701207047000003682249224A9342FA
:1040200018BF8B4228D01432934225D014329342C9
:1040300022D0143293421FD0143293421CD0143237
:10404000934219D01432934216D0DAB2103A17497B
:10405000A1FB0212120916491944A8291FD9154BB0
:1040600013449B000366144B436602F01F020123B6
:1040700003FA02F282667047DBB2083B0F4AA2FBEA
:1040800003230F4A02EB1312920002660D4A4266A6
:10409000C3F30413012202FA03F383667047083264
:1040A000DDE700BF085402581C540258ABAAAAAA64
:1040B000F0FBFDBF0082001080080240CDCCCCCCCC
:1040C000009600168058025801794A1E072A2CD8FB
:1040D00030B40368154D164CA34218BFAB4218D03C
:1040E0001434A34215D01434A34212D01434A34282
:1040F0000FD01434A3420CD01434A34209D014348A
:10410000A34206D00B4B0B449B00C3660A4B0367CC
:1041100005E00A4B0B449B00C366094B0367012370
:1041200003FA02F2426730BC7047704708540258E5
:104130001C5402583F820010400902403F9600166E
:104140004059025870B50446FEF71AFD002C00F0E5
:10415000B681054623685349534A934218BF8B42A0
:104160000CBF0122002250D030318B424DD018318B
:104170008B424AD018318B4247D018318B4244D001
:1041800018318B4241D018318B423ED001F5567127
:104190008B423AD018318B4237D018318B4234D011
:1041A00018318B4231D018318B422ED018318B42CE
:1041B0002BD018318B4228D018318B4225D03B4967
:1041C0003B4A934218BF8B4200F03181394A9342F7
:1041D00000F02D811432934200F029811432934271
:1041E00000F025811432934200F021811432934271
:1041F00000F01D811432934200F019814023636561
:10420000032384F8353001204AE0022184F8351078
:10421000002184F834107ABB274A93422CD01832FC
:10422000934229D01832934226D01832934223D099
:104230001832934220D0183293421DD002F55672A4
:10424000934219D01832934216D01832934213D0A9
:104250001832934210D0183293420DD01832934244
:104260000AD01832934207D01832934204D01A6809
:1042700022F001021A6003E01A6822F001021A60BB
:1042800023681A6812F0010F18D0FEF779FC431B5F
:10429000052BF5D920236365032384F835300120ED
:1042A00070BD00BF100002402800024008540258B0
:1042B0001C54025830540258400002401A68814889
:1042C0001040A168E2680A4321690A4361690A4310
:1042D000A1690A43E1690A43216A0A430243616A08
:1042E000042900F099807849086878490140B1F1C3
:1042F000005F11D36168A1F12905A1F13F000328F6
:1043000088BF052D06D9A1F14700012802D94F39F0
:10431000032901D842F480121A602668756925F0D5
:104320000705636A1D43042B08D1A36A1D43E36A92
:1043300023B12046FFF726FE002872D17561204682
:10434000FFF7C6FDE36D03F01F023F239340836038
:1043500023685F495F4A934218BF8B4242D01832AC
:1043600093423FD0183293423CD01832934239D016
:104370001832934236D01832934233D018329342D7
:1043800030D002F5567293422CD01832934229D085
:104390001832934226D01832934223D018329342D7
:1043A00020D0183293421DD0183293421AD01832BE
:1043B000934217D0484A934214D01432934211D0FA
:1043C000143293420ED0143293420BD014329342E3
:1043D00008D01432934205D01432934202D01432E2
:1043E000934213D12046FFF717FEA368802B59D0C4
:1043F000236E22791A60636EA26E5A606368013B75
:10440000072B52D90023E3662367636700206065AA
:10441000012384F8353043E7E16A206B01430A4306
:1044200061E740236365012084F8350038E7022204
:1044300084F83520002284F834201A682749114076
:10444000A268402A2CD0802A27D00022E06842EAC5
:10445000D002206942EAD002606942EAD002A06933
:1044600042EAD002E06942EAD002206A42EA10122F
:104470000A431A6022681A4B13441A4AA2FB032308
:104480001B099B00E3652046FFF722FDE26D02F069
:104490001F0101228A4042605AE74FF48042D5E76B
:1044A0001022D3E700236360A2E72046FFF70CFE4B
:1044B000E36E00221A60236F626F5A60A6E7012044
:1044C000EEE600BF3F8010FE0010005C0000FFFF22
:1044D0001000024028000240085402580F00FEFF5E
:1044E000F8ABFDA7CDCCCCCC002800F03E8170B558
:1044F000044690F83400012800F03981012084F846
:10450000340094F83500C0B2012807D04FF400639E
:104510006365002384F83430012070BD022084F8E4
:104520003500002060652068924E934DA84218BF68
:10453000B0422FD01835A8422CD01835A84229D027
:104540001835A84226D01835A84223D01835A842DD
:1045500020D01835A8421DD005F55675A84219D0AF
:104560001835A84216D01835A84213D01835A842DD
:1045700010D01835A8420DD01835A8420AD01835E9
:10458000A84207D01835A84204D0056825F00105D7
:10459000056003E0056825F0010505602046FFF78A
:1045A000BDFB23687349744A934218BF8B4238D0CD
:1045B0001832934235D01832934232D01832934297
:1045C0002FD0183293422CD01832934229D018326F
:1045D000934226D002F55672934222D0183293426B
:1045E0001FD0183293421CD01832934219D018327F
:1045F000934216D01832934213D01832934210D0FF
:10460000183293420DD01A6822F00E0242F00A02CC
:104610001A60236C93B12268136843F0040313609B
:104620000CE01A6822F01E0242F016021A60236C97
:1046300023B12268136843F00803136023684D49CF
:104640004D4A934218BF8B4242D0183293423FD01A
:10465000183293423CD01832934239D018329342E8
:1046600036D01832934233D01832934230D002F50C
:10467000567293422CD01832934229D0183293426A
:1046800026D01832934223D01832934220D01832C9
:1046900093421DD0183293421AD01832934217D049
:1046A000364A934214D01432934211D014329342BA
:1046B0000ED0143293420BD01432934208D01432ED
:1046C000934205D01432934202D0143293420ED159
:1046D000236E1A6812F4803F03D01A6842F4807285
:1046E0001A60E36E1BB11A6842F480721A60236884
:1046F0002049214A934218BF8B4230D0183293424E
:104700002DD0183293422AD01832934227D0183233
:10471000934224D01832934221D0183293421ED0B3
:1047200002F5567293421AD01832934217D01832BB
:10473000934214D01832934211D0183293420ED0C3
:10474000183293420BD01832934208D01832934259
:1047500005D01A6842F001021A600020DDE61A68EE
:1047600042F001021A600020D7E6012070470220C3
:10477000D3E600BF1000024028000240085402584F
:1047800070B50446FEF7FCF9002C00F09181054657
:1047900094F83530DBB2022B06D08023636500230A
:1047A00084F83430012070BD23688C498C4A9342D0
:1047B00018BF8B4230D0183293422DD0183293421A
:1047C0002AD01832934227D01832934224D018327C
:1047D000934221D0183293421ED002F55672934272
:1047E0001AD01832934217D01832934214D018328C
:1047F000934211D0183293420ED0183293420BD00C
:104800001832934208D01832934205D01A6822F029
:104810000E021A60266809E01A6822F01E021A6069
:104820002268536923F080035361266823686B492B
:104830006B4A934218BF8B4242D0183293423FD00A
:10484000183293423CD01832934239D018329342F6
:1048500036D01832934233D01832934230D002F51A
:10486000567293422CD01832934229D01832934278
:1048700026D01832934223D01832934220D01832D7
:1048800093421DD0183293421AD01832934217D057
:10489000544A934214D01432934211D014329342AA
:1048A0000ED0143293420BD01432934208D01432FB
:1048B000934205D01432934202D01432934204D171
:1048C000226E136823F48073136023684349444ABB
:1048D000934218BF8B422FD0183293422CD01832FB
:1048E000934229D01832934226D01832934223D0D3
:1048F0001832934220D0183293421DD002F55672DE
:10490000934219D01832934216D01832934213D0E2
:104910001832934210D0183293420DD0183293427D
:104920000AD01832934207D01832934204D01A6842
:1049300022F001021A6003E01A6822F001021A60F4
:10494000336813F0010F0ED0FEF71AF9431B052B45
:10495000F6D920236365032384F83530002384F8D7
:10496000343001201FE723681C491D4A934218BFB9
:104970008B4239D01832934236D01832934233D01A
:104980001832934230D0183293422DD018329342CD
:104990002AD01832934227D002F55672934223D080
:1049A0001832934220D0183293421DD018329342CD
:1049B0001AD01832934217D01832934214D01832BA
:1049C000934211D0183293420ED0A16DE36D03F0E3
:1049D0001F02012393404B600DE000BF1000024016
:1049E0002800024008540258A16DE36D03F01F0235
:1049F0003F2393408B6023682E492F4A934218BF70
:104A00008B4242D0183293423FD0183293423CD06E
:104A10001832934239D01832934236D0183293422A
:104A200033D01832934230D002F5567293422CD0D4
:104A30001832934229D01832934226D0183293422A
:104A400023D01832934220D0183293421DD018320E
:104A500093421AD01832934217D0184A934214D076
:104A60001432934211D0143293420ED01432934236
:104A70000BD01432934208D01432934205D0143232
:104A8000934202D0143293420BD1636EA26E5A60ED
:104A9000E36E33B11A6822F480721A60236F626F7A
:104AA0005A60012384F83530002084F834007AE617
:104AB000012078E610000240280002400854025805
:104AC000002800F0298108B5024690F83530DBB2A5
:104AD000022B03D080234365012008BD0368904862
:104AE00090498B4218BF83420CBF0121002166D040
:104AF0003030834263D01830834260D01830834214
:104B00005DD0183083425AD01830834257D01830C5
:104B1000834254D000F55670834250D018308342FF
:104B20004DD0183083424AD01830834247D01830D5
:104B3000834244D01830834241D0183083423ED063
:104B4000183083423BD0196821F00E0119601368B8
:104B5000A0F5956073498B4218BF83426AD07249B1
:104B60008B4267D018318B4264D018318B4261D0B0
:104B700018318B425ED018318B425BD018318B429A
:104B800058D001F556718B4254D018318B4251D018
:104B900018318B424ED018318B424BD018318B429A
:104BA00048D018318B4245D018318B4242D0183151
:104BB0008B423FD0196821F0010119603EE00420CA
:104BC00082F8350081BB584A93422DD01832934267
:104BD0002AD01832934227D01832934224D0183268
:104BE000934221D0183293421ED002F5567293425E
:104BF0001AD01832934217D01832934214D0183278
:104C0000934211D0183293420ED0183293420BD0F7
:104C10001832934208D01832934205D01A6822F015
:104C200001021A60002058E71A6822F001021A6097
:104C3000002052E7196821F0010119601368384813
:104C400038498B4218BF834242D018318B423FD043
:104C500018318B423CD018318B4239D018318B42FD
:104C600036D018318B4233D018318B4230D001F519
:104C700056718B422CD018318B4229D018318B427F
:104C800026D018318B4223D018318B4220D01831D6
:104C90008B421DD018318B421AD018318B4217D05D
:104CA00022498B4214D014318B4211D014318B42E3
:104CB0000ED014318B420BD014318B4208D01431FA
:104CC0008B4205D014318B4202D014318B4217D164
:104CD000116E0B6823F480730B60906DD36D03F03D
:104CE0001F0101238B404360536E916E5960D36E58
:104CF00033B1196821F480711960136F516F5960D5
:104D0000012382F83530002382F83430136D2BB143
:104D1000104698470020E0E6012070470020DCE6BE
:104D2000100002402800024040000240085402588F
:104D3000F0B583B00446002301937D4B1D687D4B85
:104D4000A3FB0535AD0A876D3E68D7F800C0036840
:104D500079497A48834218BF8B420CBF012000205A
:104D600061D0774A93425ED0183293425BD01832BA
:104D7000934258D01832934255D01832934252D0B1
:104D8000183293424FD002F5567293424BD01832EC
:104D9000934248D01832934245D01832934242D0C1
:104DA000183293423FD0183293423CD0183293428B
:104DB00039D01832934236D06249634A934218BFC1
:104DC0008B4212D0614A93420FD0143293420CD0DE
:104DD0001432934209D01432934206D014329342D3
:104DE00003D01432934240F061821A68E16D01F001
:104DF0001F010420884010EA0C0F00F0A78212F077
:104E0000040F00F0A382786012F4004F00F05A8281
:104E100012F4803F40F05082A36C002B00F04682D9
:104E20002046984742E2E26D02F01F0108228A40C4
:104E3000324241D070BB424A93422BD01832934247
:104E400028D01832934225D01832934222D01832FB
:104E500093421FD0183293421CD002F556729342EF
:104E600018D01832934215D01832934212D018320B
:104E700093420FD0183293420CD01832934209D08B
:104E80001832934206D01832934203D01A68C2F304
:104E9000C00202E01A68C2F380026AB11A6822F006
:104EA00004021A60E36D03F01F0208239340BB6005
:104EB000636D43F001036365E26D02F01F0226FAA1
:104EC00002F313F0010F47D023681B481B498B42A4
:104ED00018BF83423CD018318B4239D018318B42F5
:104EE00036D018318B4233D018318B4230D0183144
:104EF0008B422DD018318B422AD001F556718B424E
:104F000026D018318B4223D018318B4220D0183153
:104F10008B421DD018318B421AD018318B4217D0DA
:104F200018318B4214D018318B4211D01B6813E01A
:104F300004000024B5814E1B1000024028000240EE
:104F400040000240085402581C5402583054025881
:104F50005B6913F0800F3BD1E36D03F01F03042264
:104F600002FA03F3334240D02268964896498A42B7
:104F700018BF824235D018318A4232D018318A4265
:104F80002FD018318A422CD018318A4229D01831BA
:104F90008A4226D018318A4223D001F556718A42BE
:104FA0001FD018318A421CD018318A4219D01831CA
:104FB0008A4216D018318A4213D018318A4210D052
:104FC00018318A420DD018318A420AD013680CE099
:104FD000012303FA02F2BA60636D43F002036365D2
:104FE000BAE7126812F0020F3DD1E36D03F01F0320
:104FF000102202FA03F333425FD0226871487249EB
:105000008A4218BF824234D018318A4231D01831D6
:105010008A422ED018318A422BD018318A4228D0A9
:1050200018318A4225D018318A4222D001F55671B2
:105030008A421ED018318A421BD018318A4218D0B9
:1050400018318A4215D018318A4212D018318A425A
:105050000FD018318A420CD018318A4209D0126818
:10506000C2F3800208E0BB60636D43F00403636534
:10507000BBE71268C2F3C002FAB1BB6023681A68CA
:1050800012F4802F0DD01B6813F4002F04D1236C71
:105090009BB12046984710E0A36C73B12046984717
:1050A0000BE01A6812F4807F03D11A6822F008021C
:1050B0001A60236C0BB120469847E36D03F01F0381
:1050C000202202FA03F3334200F0928022683D4826
:1050D0003D498A4218BF82422ED018318A422BD0D5
:1050E00018318A4228D018318A4225D018318A4294
:1050F00022D018318A421FD018318A421CD001F5C3
:1051000056718A4218D018318A4215D018318A4215
:1051100012D018318A420FD018318A420CD018317F
:105120008A4209D018318A4206D018318A4203D007
:105130001268C2F3400202E01268C2F30012002AB1
:1051400056D0BB6094F83530DBB2042B0ED0236808
:105150001A6812F4802F39D01B6813F4002F2CD159
:10516000636C002B44D02046984741E022681368C6
:1051700023F0160313602268536923F08003536100
:10518000236CB3B12268136823F008031360E36D46
:1051900003F01F023F239340BB60012384F83530A6
:1051A000002384F83430236D002B7FD020469847AD
:1051B0007CE0A36C002BE5D1E9E7E36BC3B12046AB
:1051C000984715E010000240280002401A6812F4C7
:1051D000807F09D11A6822F010021A60012384F836
:1051E0003530002384F83430E36B0BB12046984708
:1051F000636D002B5AD0636D13F0010F52D004235E
:1052000084F8353023689649964A934218BF8B42FA
:105210002FD0183293422CD01832934229D0183212
:10522000934226D01832934223D01832934220D092
:10523000183293421DD002F55672934219D018329B
:10524000934216D01832934213D01832934210D0A2
:10525000183293420DD0183293420AD0183293423A
:1052600007D01832934204D01A6822F001021A6063
:1052700003E01A6822F001021A60019B01330193D6
:10528000AB4204D823681B6813F0010FF5D12368E3
:105290001B6813F0010F0BD0032384F83530002373
:1052A00084F83430E36C0BB12046984703B0F0BD6E
:1052B000012384F83530F2E7236C002BF6D020462A
:1052C0009847F3E712F0200F3AD123686449654A02
:1052D000934218BF8B422FD0183293422CD01832F1
:1052E000934229D01832934226D01832934223D0C9
:1052F0001832934220D0183293421DD002F55672D4
:10530000934219D01832934216D01832934213D0D8
:105310001832934210D0183293420DD01832934273
:105320000AD01832934207D01832934204D01A6838
:1053300022F004021A6003E01A6822F008021A60E0
:10534000236C002BB2D020469847AFE7022088405C
:1053500010EA0C0F60D012F0020F5DD0786012F4EA
:10536000004F0ED012F4803F05D1636C002B9DD00E
:10537000204698479AE7E36B002B97D02046984742
:1053800094E712F0200F40D123683549354A934203
:1053900018BF8B422FD0183293422CD01832934230
:1053A00029D01832934226D01832934223D0183293
:1053B000934220D0183293421DD002F55672934288
:1053C00019D01832934216D01832934213D01832A3
:1053D000934210D0183293420DD0183293420AD023
:1053E0001832934207D01832934204D01A6822F040
:1053F0000A021A6003E01A6822F014021A600123FC
:1054000084F83530002384F83430E36B002B3FF40C
:105410004DAF2046984749E7082000FA01F111EA0C
:105420000C0F3FF443AF12F0080F3FF43FAF1A6880
:1054300022F00E021A60E36D03F01F03012202FA4C
:1054400003F37B60626584F83520002384F83430F0
:10545000E36C002B3FF42AAF2046984726E700BFB5
:10546000100002402800024070B582B000236EE0B8
:1054700085685E000324B44025EA0405CC68B44086
:105480002C438460446824EA0C0C4C68C4F3001478
:105490009C4044EA0C0444606CE0DD08083550F898
:1054A000256003F007044FEA840C0F2404FA0CF47F
:1054B00026EA040E0C6904FA0CF444EA0E0440F8DF
:1054C00025406FE0092400E0002404FA0EF42C4388
:1054D0000CF1020C6B4D45F82C404FF0B0442568A0
:1054E000D44325EA0206D1F804C01CF4801F01D081
:1054F00042EA05064FF0B0452E606D6804EA0506E5
:10550000D1F804C01CF4001F01D042EA05064FF098
:10551000B0456E60D5F8845004EA0506D1F804C0A1
:105520001CF4003F01D042EA05064FF0B045C5F833
:105530008460D5F880502C404E6816F4803F01D02E
:1055400042EA05044FF0B042C2F8804001330A68D5
:1055500032FA03F400F093804FF0010C0CFA03FCD4
:105560001CEA0202F2D04C6804F00304013C012C56
:105570007FF67EAF4C6804F00304032C0CD0C468A3
:105580005D004FF0030C0CFA05FC24EA0C0C8C684F
:10559000AC4044EA0C04C4604C6804F00304022CE0
:1055A0003FF47BAF04684FEA430E4FF0030C0CFA54
:1055B0000EFC24EA0C0C4C6804F0030404FA0EF40C
:1055C00044EA0C0404604C6814F4403FBED02E4CF6
:1055D000D4F8F45045F00205C4F8F450D4F8F4407F
:1055E00004F002040194019C4FEA930C0CF10205B3
:1055F000244C54F8255003F003044FEA840E0F2482
:1056000004FA0EF425EA0405204CA0423FF45CAFF6
:1056100004F58064A04222D004F58064A04220D02A
:1056200004F58064A0421ED004F58064A0421CD022
:1056300004F58064A0421AD004F58064A04218D01A
:1056400004F58064A04216D004F58064A04214D012
:1056500004F58064A0423FF435AF0A2435E7012405
:1056600033E7022431E703242FE704242DE7052440
:105670002BE7062429E7072427E7082425E702B0BB
:1056800070BD00BF000400580044025800000258DA
:105690000AB181617047090481617047134BDB686F
:1056A00013F0040F07D1114BDB6803F007038342AB
:1056B0001AD00120704710B50C4AD36823F00703B5
:1056C0001843D060FDF75CFA0446084B5B6813F49E
:1056D000005F07D1FDF754FA001BB0F57A7FF4D9CB
:1056E000012000E0002010BD002070470048025853
:1056F000002800F0398338B50446036813F0010F21
:1057000025D0944A136903F03803926A102B15D000
:10571000182B0FD06368B3F5803F3FD0002B53D1D7
:105720008C4B1A6822F480321A601A6822F48022A4
:105730001A6038E002F00302022AEBD1854B1B68A5
:1057400013F4003F03D06368002B00F00F8323683D
:1057500013F0020F00F0A1807E4A1369926A13F0E1
:1057600038035AD0182B55D0E368002B00F0DE80A8
:1057700078490A6822F0190213430B60FDF700FA1A
:105780000546744B1B6813F0040F40F0AD80FDF725
:10579000F7F9401B0228F4D90320EEE26D4A1368A2
:1057A00043F48033136063682BB3FDF7E9F90546D2
:1057B000684B1B6813F4003FC9D1FDF7E1F9401BAA
:1057C0006428F5D90320D8E2B3F5A02F09D0614BA6
:1057D0001A6822F480321A601A6822F480221A6051
:1057E000E1E75C4B1A6842F480221A601A6842F4BE
:1057F00080321A60D7E7FDF7C3F90546554B1B68A1
:1058000013F4003FA3D0FDF7BBF9401B6428F5D982
:105810000320B2E212F0030FA6D14E4B1B6813F027
:10582000040F03D0E368002B00F0A282494A1368FA
:1058300023F01903E1680B431360FDF7A1F9054656
:10584000444B1B6813F0040F06D1FDF799F9401B78
:105850000228F5D9032090E2FDF798F941F20303FD
:10586000984212D82269402A07D03A494B6823F45B
:105870007C3343EA02334B600FE0364A536823F42B
:105880007C3343F40033536007E0324A536823F01B
:10589000FE43216943EA01635360236813F0100F4C
:1058A00000F088802B4A136903F03803926A082BB2
:1058B00056D0182B50D0E369002B00F0B880254A51
:1058C000136843F080031360FDF75AF90546214B36
:1058D0001B6813F4807F40F08880FDF751F9401B6E
:1058E0000228F4D9032048E2FDF750F941F20303FE
:1058F000984212D82269402A07D016494B6823F4EF
:105900007C3343EA02334B60C7E7124A536823F4FF
:105910007C3343F400335360BFE70E4A536823F0EF
:10592000FE43216943EA01635360B6E7094A1368FD
:1059300023F001031360FDF723F90546054B1B68AF
:1059400013F0040FA9D0FDF71BF9401B0228F5D96D
:10595000032012E20044025802F00302012AAAD1F5
:10596000A14B1B6813F4807F03D0E369802B40F0C8
:105970000182FDF70BF941F20303984212D8226A23
:10598000202A07D098494B6823F0F84343EA826302
:105990004B600FE0944A536823F0F84343F0804390
:1059A000536007E0904AD36823F07C53216A43EAAE
:1059B0000163D360236813F0080F60D06369002B84
:1059C00049D0894A536F43F001035367FDF7D8F874
:1059D0000546854B5B6F13F0020F50D1FDF7D0F8F1
:1059E000401B0228F5D90320C7E1FDF7CFF841F2AB
:1059F0000303984212D8226A202A07D07A494B68BA
:105A000023F0F84343EA82634B60D3E7764A536856
:105A100023F0F84343F080435360CBE7724AD368E6
:105A200023F07C53216A43EA0163D360C2E76E4AE4
:105A3000136823F080031360FDF7A2F805466A4B54
:105A40001B6813F4807FB5D0FDF79AF8401B02283D
:105A5000F5D9032091E1644A536F23F001035367A2
:105A6000FDF78EF80546604B5B6F13F0020F06D012
:105A7000FDF786F8401B0228F5D903207DE1236855
:105A800013F0200F29D0A3699BB1574A136843F440
:105A900080531360FDF774F80546534B1B6813F4ED
:105AA000005F1AD1FDF76CF8401B0228F5D90320DE
:105AB00063E14D4A136823F480531360FDF760F8E7
:105AC0000546494B1B6813F4005F06D0FDF758F8F4
:105AD000401B0228F5D903204FE1236813F0040F7F
:105AE00021D1636A002B00F047813F4A126902F01E
:105AF0003802182A00F0EE80022B79D03A4A136857
:105B000023F080731360FDF73BF80446364B1B68A7
:105B100013F0007F00F0DC80FDF732F8001B022854
:105B2000F4D9032029E1314A136843F480731360E8
:105B3000FDF726F805462D4B1B6813F4807F06D130
:105B4000FDF71EF8401B6428F5D9032015E1A36872
:105B5000012B0AD00BBB244B1A6F22F001021A67EB
:105B60001A6F22F004021A6704E01F4A136F43F011
:105B700001031367A36833B3FDF702F805461A4B18
:105B80001B6F13F0020FACD1FCF7FAFF401B41F280
:105B900088339842F3D90320EFE0052B09D0124B4C
:105BA0001A6F22F001021A671A6F22F004021A67B4
:105BB000E0E70D4B1A6F42F004021A671A6F42F0C9
:105BC00001021A67D6E7FCF7DBFF0546064B1B6FA1
:105BD00013F0020F85D0FCF7D3FF401B41F288334E
:105BE0009842F3D90320C8E0004402580048025804
:105BF000694A136823F080731360FCF7C1FF054600
:105C0000654B1B6813F0007F06D0FCF7B9FF401B03
:105C10000228F5D90320B0E05F4B996A5F4A0A4039
:105C2000A16AE06A41EA00110A439A62226B013AD2
:105C3000C2F30802616B0139490289B20A43A16BC0
:105C40000139090401F4FE010A43E16B0139090637
:105C500001F0FE410A431A63DA6A22F00102DA62B5
:105C6000596B4F4A0A40A16C42EAC1025A63DA6A90
:105C700022F00C02216C0A43DA62DA6A22F0020294
:105C8000616C0A43DA62DA6A42F48032DA62DA6A12
:105C900042F40032DA62DA6A42F48022DA62DA6AC4
:105CA00042F00102DA621A6842F080721A60FCF770
:105CB00067FF0446384B1B6813F0007F06D1FCF7E2
:105CC0005FFF001B0228F5D9032056E0002054E0B6
:105CD000002052E0304A916A106B012B4ED001F047
:105CE0000303A26A93424BD1C1F30511E36A9942BF
:105CF00048D1C0F30802236B013B9A4244D1C0F360
:105D00004622636B013B9A4240D1C0F30642A36B2B
:105D1000013B9A423CD1C0F30660E36B013B9842E1
:105D200038D11D4B5B6BC3F3CC03A26C9A4201D1FB
:105D3000002022E0184AD36A23F00103D362FCF763
:105D40001FFF0546FCF71CFFA842FBD0124A516B0F
:105D5000134B0B40A16C43EAC1035363D36A43F076
:105D60000103D362002008E001207047012004E015
:105D7000012002E0012000E0002038BD0120FCE706
:105D80000120FAE70120F8E70120F6E70120F4E717
:105D90000120F2E70120F0E7004402580CFCFFFF6D
:105DA0000700FFFFF8B57E4B1B6903F03803102B8B
:105DB00000F0F280182B10D013B17A4C2046F8BDB9
:105DC000774B1B6813F0200F00F0E880744B1868C5
:105DD000C0F3C100744CC440F0E7714B9D6A05F0FC
:105DE00003059C6AC4F30514D86A00F001005B6BDC
:105DF000C3F3CC0303FB00F0FAF738FB0646002C94
:105E0000DCD0012D76D0022D00F0A4800DB3204609
:105E1000FAF72CFB01466548FAF734FC0446604B60
:105E2000186BC0F30800FAF721FB05464FF06451E8
:105E30003046FAF773FB01462846FAF767FA4FF047
:105E40007E51FAF763FA01462046FAF767FB0446EB
:105E500071E0534B1B6813F0200F29D0504F3B6863
:105E6000C3F3C1035048D840FAF700FB054620466B
:105E7000FAF7FCFA01462846FAF704FC0446386BA8
:105E8000C0F30800FAF7F2FA05464FF064513046C5
:105E9000FAF744FB01462846FAF738FA4FF07E51EC
:105EA000FAF734FA01462046FAF738FB044642E096
:105EB0002046FAF7DBFA01463D48FAF7E3FB0446D1
:105EC000374B186BC0F30800FAF7D0FA05464FF0CD
:105ED00064513046FAF722FB01462846FAF716FAD3
:105EE0004FF07E51FAF712FA01462046FAF716FBF8
:105EF000044620E02046FAF7B9FA01462B48FAF7A3
:105F0000C1FB0446264B186BC0F30800FAF7AEFA43
:105F100005464FF064513046FAF700FB014628462B
:105F2000FAF7F4F94FF07E51FAF7F0F901462046FE
:105F3000FAF7F4FA04461A4B1B6BC3F34623581CBA
:105F4000FAF794FA01462046FAF79CFBFAF736FC7A
:105F5000044633E72046FAF789FA01461548FAF76E
:105F600091FB04460E4B186BC0F30800FAF77EFA5B
:105F700005464FF064513046FAF7D0FA01462846FC
:105F8000FAF7C4F94FF07E51FAF7C0F901462046FE
:105F9000FAF7C4FA0446CEE7074C0FE7024C0DE7C8
:105FA0000044025800093D000090D0030024744AC8
:105FB0000024744C0024F44A00127A00002800F0F7
:105FC000328170B50D4604469B4B1B6803F00F03EE
:105FD0008B420BD2984A136823F00F030B431360D4
:105FE000136803F00F038B4240F01F81236813F006
:105FF000040F0CD02269914B9B6903F070039A4205
:1060000005D98E498B6923F070031A438A6123688E
:1060100013F0080F0CD06269884BDB6903F0700342
:106020009A4205D98549CB6923F070031A43CA61A6
:10603000236813F0100F0CD0A269804BDB6903F4C6
:10604000E0639A4205D97D49CB6923F4E0631A43A2
:10605000CA61236813F0200F0CD0E269774B1B6AEA
:1060600003F070039A4205D974490B6A23F0700358
:106070001A430A62236813F0020F0CD0E2686F4BD8
:106080009B6903F00F039A4205D96C498B6923F091
:106090000F031A438A61236813F0010F41D0674A46
:1060A000936923F47063A1680B4393616368022BC7
:1060B0000AD0032B27D0012B2CD0604A126812F093
:1060C000040F06D10120ADE0126812F4003F00F089
:1060D000AE805A490A6922F0070213430B61FCF7AC
:1060E0004FFD0646554B1B6903F038036268B3EB5E
:1060F000C20F16D0FCF744FD801B41F28833984252
:10610000F0D903208EE04D4A126812F0007FE0D1F2
:10611000012087E0494A126812F4807FD9D101201A
:1061200080E0236813F0020F0CD0E268434B9B69B8
:1061300003F00F039A4205D240498B6923F00F0305
:106140001A438A613C4B1B6803F00F03AB420AD928
:10615000394A136823F00F032B431360136803F0CD
:106160000F03AB4265D1236813F0040F0CD02269F2
:10617000324B9B6903F070039A4205D22F498B6919
:1061800023F070031A438A61236813F0080F0CD0C0
:1061900062692A4BDB6903F070039A4205D22749F2
:1061A000CB6923F070031A43CA61236813F0100F00
:1061B0000CD0A269214BDB6903F4E0639A4205D25B
:1061C0001E49CB6923F4E0631A43CA61236813F0C4
:1061D000200F0CD0E269194B1B6A03F070039A423E
:1061E00005D216490B6A23F070031A430A62FFF7BF
:1061F000D9FD12498B69C3F30323114AD35C03F021
:106200001F03D8408B6903F00F03D35C03F01F0317
:1062100020FA03F30B4A13600B4B18600B4B186802
:10622000FCF74CFC70BD012070470120FAE701200B
:10623000F8E70120F6E700BF0020005200440258B2
:10624000180601080800002404000024100000249F
:1062500008B5FFF7A7FD0B4A9369C3F303230A4967
:10626000CB5C03F01F0320FA03F3926902F00F02E4
:10627000885C00F01F0023FA00F0044A1060044A12
:10628000136008BD004402581806010808000024E5
:106290000400002408B5FFF7DBFF054BDB69C3F3FF
:1062A0000213044AD35C03F01F03D84008BD00BFAB
:1062B000004402581806010808B5FFF7C9FF054B4E
:1062C000DB69C3F30223044AD35C03F01F03D84005
:1062D00008BD00BF0044025818060108404B9B6AE5
:1062E00003F00303032B79D070B505460E463C4AF4
:1062F000136823F080631360FCF742FC0446384BBC
:106300001B6813F0006F06D0FCF73AFC031B022B4E
:10631000F5D9032070BD324B9A6A22F47C32296889
:1063200042EA01329A626A68013AC2F30802A96835
:106330000139490289B20A43E9680139090401F4C3
:10634000FE010A4329690139090601F0FE410A43A9
:106350009A63DA6A22F0C00269690A43DA62DA6A89
:1063600022F02002A9690A43DA62DA6A22F01002F6
:10637000DA62D96B1B4A0A40E96942EAC102DA6370
:10638000DA6A42F01002DA62C6B91A46DB6A43F4EE
:106390000023D362124A136843F080631360FCF752
:1063A000EFFB04460E4B1B6813F0006F14D1FCF793
:1063B000E7FB001B0228F5D90320ABE7012E05D02F
:1063C000074AD36A43F40013D362E3E7044AD36A6B
:1063D00043F48013D362DDE700209BE70120704780
:1063E000004402580700FFFF404B9B6A03F0030381
:1063F000032B79D070B505460E463C4A136823F04E
:1064000080531360FCF7BCFB0446384B1B6813F049
:10641000005F06D0FCF7B4FB031B022BF5D9032069
:1064200070BD324B9A6A22F07C72296842EA0152AE
:106430009A626A68013AC2F30802A96801394902FE
:1064400089B20A43E9680139090401F4FE010A43EB
:1064500029690139090601F0FE410A431A64DA6A22
:1064600022F4406269690A43DA62DA6A22F400724D
:10647000A9690A43DA62DA6A22F48072DA62596C34
:106480001B4A0A40E96942EAC1025A64DA6A42F4E4
:106490008072DA62C6B91A46DB6A43F48003D362BB
:1064A000124A136843F080531360FCF769FB0446FB
:1064B0000E4B1B6813F0005F14D1FCF761FB001B4F
:1064C0000228F5D90320ABE7012E05D0074AD36A8D
:1064D00043F08073D362E3E7044AD36A43F40003D2
:1064E000D362DDE700209BE701207047004402589B
:1064F0000700FFFFF8B50446036813F0006F30D0C3
:10650000836EB3F5001F26D00ED8EBB1B3F5801F14
:1065100007D102210830FFF7E1FE054645B12E46BE
:1065200021E0012635461EE0B3F5401F09D10025C4
:10653000984A136D23F44013A16E0B431365002694
:1065400011E0012635460EE0924AD36A43F4003347
:10655000D3620025ECE702212830FFF745FF05460E
:10656000DCE700263546236813F4807F14D0A36D42
:10657000042B32D8DFE803F003232A080800854AF9
:10658000D36A43F40033D36255BB824A136D23F0C0
:106590000703A16D0B431365236813F4007F31D00B
:1065A000E36D802B4CD020D8002B43D0402B19D149
:1065B000002104F10800FFF791FE05461AE00021D2
:1065C00004F10800FFF78AFE0546DDE7002104F12B
:1065D0002800FFF709FF0546D6E701263546DBE729
:1065E0002E46D9E7012635460CE0C02B02D0B3F584
:1065F000807F1CD15DBB674A136D23F4E073E16DAE
:106600000B431365236813F4806F46D0D4F8A83089
:10661000B3F5800F39D01FD88BB3B3F5001F18D155
:10662000002104F10800FFF759FE05461AE0012693
:106630003546E7E7574AD36A43F40033D362D9E7D4
:10664000002104F12800FFF7CFFE0546D2E72E46D1
:10665000D8E70126354620E0B3F5C00F02D0B3F5E8
:10666000000F09D1C5B94B4A936D23F46003D4F8E8
:10667000A8100B43936510E0012635460DE0454A0E
:10668000D36A43F40033D362ECE7002104F128001D
:10669000FFF7AAFE0546E5E72E46236813F4006FD0
:1066A00024D0D4F8AC30B3F1007F42D00ED8002B08
:1066B00039D0B3F1807F06D1002104F10800FFF743
:1066C0000DFE054608E0012635460FE0B3F1407F98
:1066D00002D0B3F1806F23D1002D31D12D4A936DBB
:1066E00023F0E063D4F8AC100B439365236813F0F8
:1066F000007F2ED0E36C202B40D026D833B1102B56
:1067000020D1244AD36A43F40033D362002D3CD114
:10671000204AD36C23F03003E16C0B43D36418E0C0
:1067200001263546E2E71B4AD36A43F40033D362BD
:10673000D2E7002104F12800FFF756FE0546CBE71B
:106740002E46D3E70126354603E0302BDED0012666
:106750003546236813F4805F2DD0236EB3F5005FB8
:106760004FD019D8002B46D0B3F5805F0FD1002150
:1067700004F10800FFF7B2FD054613E0022104F121
:106780000800FFF7ABFD0546C0E72E46E1E701260E
:10679000354610E000440258B3F5405F02D0B3F52F
:1067A000804F25D1002D33D1774A136D23F4E04378
:1067B000216E0B431365236813F4005F38D0636EBA
:1067C000B3F5003F53D028D843B1B3F5803F21D172
:1067D000012104F10800FFF781FD0546002D4DD190
:1067E000694A136D23F4E023616E0B4313651FE0C8
:1067F00001263546DFE7644AD36A43F40033D362A7
:10680000D0E7002104F12800FFF7EEFD0546C9E7B7
:106810002E46D0E7012635460AE0B3F5802FDDD0BD
:10682000B3F5A02FDAD0B3F5403FD7D001263546D7
:10683000236813F4804F31D0D4F8B030B3F1005F47
:1068400045D020D843B1B3F1805F19D1012104F1C3
:106850000800FFF743FD0546002D3FD14A4A936DDE
:1068600023F0E043D4F8B0100B43936516E0012108
:1068700004F12800FFF7B8FD0546AFE72E46D7E73D
:10688000012635460AE0B3F1804FE5D0B3F1A04FC1
:10689000E2D0B3F1405FDFD001263546236813F420
:1068A000004F09D0236FB3F1805F19D0B3F1005FBF
:1068B00024D0D3B101263546236813F0807F33D02E
:1068C000A36C032B5BD8DFE803F0272253270121B9
:1068D00004F12800FFF788FD0546BDE72E46DDE7F9
:1068E000294AD36A43F40033D36275B9264A136D3B
:1068F00023F04053216F0B431365DDE7012104F1C1
:106900000800FFF7EBFC0546EFE72E46D4E71E4AEA
:10691000D36A43F40033D362A5BB1B4AD36C23F084
:106920000303A16C0B43D364236813F4800F2DD1B0
:10693000236813F0010F00F0A580E36F282B00F20D
:106940009F80DFE803F08D9D9D9D9D9D9D9D879D72
:106950009D9D9D9D9D9D969D9D9D9D9D9D9D8D9D7E
:106960009D9D9D9D9D9D8D9D9D9D9D9D9D9D8D0014
:10697000022104F10800FFF7B1FC0546CCE701262F
:106980003546D1E72E46CFE700440258914A1368B6
:1069900043F480731360FCF7F3F807468D4B1B68D4
:1069A00013F4807F05D1FCF7EBF8C01B6428F5D900
:1069B0000325002D4AD1884B1B6FD4F8B4205340D7
:1069C00013F4407F0CD0844B1A6F22F44072196F7D
:1069D00041F480311967196F21F4803119671A6702
:1069E000D4F8B430B3F5807F15D08DBBD4F8B43073
:1069F00003F44072B2F5407F1ED0774A136923F446
:106A00007C53136174490B6FD4F8B420C2F30B02AA
:106A100013430B678CE7FCF7B3F807466E4B1B6F0D
:106A200013F0020FE1D1FCF7ABF8C01B41F2883341
:106A30009842F3D90325D8E76748026922F47C52CB
:106A4000664901EA131313430361DBE72E466FE740
:106A50002E466DE7012104F10800FFF73FFC0546D3
:106A6000E5B95D4A536D23F03803E16F0B4353657D
:106A700008E0012104F12800FFF7B6FC0546EFE726
:106A800001263546236813F0020F17D0A36F052B9C
:106A900028D8DFE803F00B05200B0B0B2E46F1E79F
:106AA000012104F10800FFF719FC0546EDB94A4A37
:106AB000536D23F00703A16F0B435365236813F055
:106AC000040F23D0D4F89430052B45D8DFE803F029
:106AD000150F3D151515012104F12800FFF784FC61
:106AE0000546E3E701263546E8E72E46E6E70121BD
:106AF00004F10800FFF7F2FB054685BB364A936DAB
:106B000023F00703D4F894100B439365236813F024
:106B1000200F34D0D4F89030B3F1005F4ED023D89A
:106B200043B1B3F1805F1CD1002104F10800FFF7ED
:106B3000D5FB0546002D48D1274A536D23F0E0438D
:106B4000D4F890100B43536519E0012104F128009B
:106B5000FFF74AFC0546D0E701263546D6E72E4624
:106B6000D4E7012635460AE0B3F1804FE2D0B3F115
:106B7000A04FDFD0B3F1405FDCD00126354623685B
:106B800013F0400F37D0D4F89C30B3F5006F53D0DA
:106B900026D843B1B3F5806F19D1002104F1080064
:106BA000FFF79CFB0546002D4DD10B4A936D23F456
:106BB000E053D4F89C100B4393651CE0022104F1D0
:106BC0002800FFF711FC0546B4E72E46D7E701265B
:106BD000354610E00048025800440258CFFFFF003D
:106BE000B3F5805FDFD0B3F5A05FDCD0B3F5406FC5
:106BF000D9D001263546236813F0800F33D0D4F85E
:106C0000A030B3F5804F00F0A38021D843B1B3F595
:106C1000005F1AD1002104F10800FFF75FFB054671
:106C2000002D40F09C80814A936D23F46043D4F89A
:106C3000A0100B43936516E0022104F12800FFF732
:106C4000D3FB0546AFE72E46D5E7012635460AE0D9
:106C5000B3F5004FE4D0B3F5204FE1D0B3F5C04F0A
:106C6000DED001263546236813F0080F0CD0D4F887
:106C70008430B3F5805F74D06C4A536D23F4405375
:106C8000D4F884100B435365236813F0100F0CD015
:106C9000D4F89830B3F5807F6CD0644A936D23F4B8
:106CA0004073D4F898100B439365236813F4002FB6
:106CB0000BD0D4F8A430B3F5803F74D0B3F5003FC7
:106CC00067D0002B5FD001263546236813F4802F50
:106CD0000CD0D4F88830B3F5001F7CD0B3F5401F3A
:106CE0006FD0B3F5801F67D001263546236813F4B3
:106CF000803F08D0236D002B76D0B3F5803F00F0A5
:106D0000818001263546236813F0005F40F08380C0
:106D1000236813F4003F00F08E80D4F88030B3F580
:106D2000807F00F0EC8040F28380B3F5007F03D0D9
:106D3000B3F5407F40F0E180002D40F0E6803B4A13
:106D4000536D23F44073D4F880100B43536572E005
:106D5000022104F12800FFF747FB054660E72E46B5
:106D600081E7022104F12800FFF73EFB002883D0D1
:106D7000012681E7022104F12800FFF735FB0028F6
:106D80008BD0012689E7002104F10800FFF7A6FA5D
:106D900005467DB9254A936D23F44033D4F8A410F9
:106DA0000B43936591E7022104F12800FFF71CFBD8
:106DB0000546EEE72E4688E71C4AD36A43F40033C3
:106DC000D3627DB9194A536D23F44013D4F8881067
:106DD0000B4353658AE7012104F12800FFF704FB08
:106DE0000546EEE72E4681E7104AD36A43F40033A6
:106DF000D36275B90D4AD36C23F48033216D0B43F4
:106E0000D36480E7022104F10800FFF767FA054622
:106E1000EFE72E4677E7022104F12800FFF7E4FAB6
:106E200000283FF475AF012672E700BF0044025806
:106E3000002B81D00126236813F4801F06D04F4A0F
:106E4000136D23F00043616F0B431365236813F048
:106E5000805F07D0494A136923F48043D4F8B810FF
:106E60000B431361236813F4001F06D0434A136DCC
:106E700023F08073E16E0B431365236813F0804F9A
:106E800009D03E4B1A6922F400421A611A69D4F8FB
:106E9000BC100A431A612368002B06DA374AD36C08
:106EA00023F04053616D0B43D364236813F4000F48
:106EB00007D0324A536D23F44003D4F88C100B43AF
:106EC0005365636813F0010F21D1636813F0020F5B
:106ED00026D1636813F0040F2BD1636813F0080FF9
:106EE00030D1636813F0100F35D1636813F0200FB1
:106EF0003AD106B101263046F8BD01269BE71F4A6C
:106F0000D36A43F40033D36216E72E4693E7002199
:106F100004F10800FFF7E2F90028D6D00646D4E7CE
:106F2000012104F10800FFF7D9F90028D1D0064665
:106F3000CFE7022104F10800FFF7D0F90028CCD0F8
:106F40000646CAE7002104F12800FFF74DFA0028A1
:106F5000C7D00646C5E7012104F12800FFF744FA2F
:106F60000028C2D00646C0E7022104F12800FFF73E
:106F70003BFA0028BDD00646BBE700BF00440258DC
:106F800008B5FFF765F9054B1B6AC3F30213044A02
:106F9000D35C03F01F03D84008BD00BF0044025873
:106FA000180601082DE9F0410446864B9D6A9E6A49
:106FB000C6F30536D86AC0F30010DB6BC3F3CC030D
:106FC00003FB00F0F9F752FA002E00F0F58005F00F
:106FD00003050746012D79D0022D00F0CB800DB3BB
:106FE0003046F9F743FA01467748F9F74BFB054677
:106FF000744B986BC0F30800F9F738FA06464FF067
:1070000064513846F9F78AFA01463046F9F77EF9B5
:107010004FF07E51F9F77AF901462846F9F77EFAE2
:10702000054674E0674B1B6813F0200F2CD0DFF887
:107030009481D8F80030C3F3C1036448D840F9F70D
:1070400015FA05463046F9F711FA01462846F9F7D0
:1070500019FB0546D8F83800C0F30800F9F706FA1E
:1070600006464FF064513846F9F758FA0146304663
:10707000F9F74CF94FF07E51F9F748F901462846E7
:10708000F9F74CFA054642E03046F9F7EFF90146C8
:107090004F48F9F7F7FA05464A4B986BC0F30800DA
:1070A000F9F7E4F906464FF064513846F9F736FA35
:1070B00001463046F9F72AF94FF07E51F9F726F9E3
:1070C00001462846F9F72AFA054620E03046F9F746
:1070D000CDF901463C48F9F7D5FA0546394B986B8E
:1070E000C0F30800F9F7C2F906464FF0645138467C
:1070F000F9F714FA01463046F9F708F94FF07E51D6
:10710000F9F704F901462846F9F708FA05462D4E25
:10711000B06BC0F34620F9F7A9F94FF07E51F9F7AB
:10712000F5F801462846F9F7ADFAF9F747FB206074
:10713000B06BC0F30640F9F799F94FF07E51F9F7BB
:10714000E5F801462846F9F79DFAF9F737FB606044
:10715000B06BC0F30660F9F789F94FF07E51F9F78B
:10716000D5F801462846F9F78DFAF9F727FBA06014
:10717000BDE8F0813046F9F779F901461548F9F78D
:1071800081FA05460F4B986BC0F30800F9F76EF9CA
:1071900006464FF064513846F9F7C0F901463046CB
:1071A000F9F7B4F84FF07E51F9F7B0F801462846E8
:1071B000F9F7B4F90546AAE7002323606360A360EA
:1071C000D6E700BF004402580024744A0090D00360
:1071D0000024744C0024F44A2DE9F0410446864B07
:1071E0009D6A9E6AC6F30556D86AC0F300205B6CA0
:1071F000C3F3CC0303FB00F0F9F738F9002E00F0DD
:10720000F58005F003050746012D79D0022D00F029
:10721000CB800DB33046F9F729F901467748F9F7E5
:1072200031FA0546744B186CC0F30800F9F71EF9E3
:1072300006464FF064513846F9F770F9014630467A
:10724000F9F764F84FF07E51F9F760F801462846E7
:10725000F9F764F9054674E0674B1B6813F0200FDB
:107260002CD0DFF89481D8F80030C3F3C103644810
:10727000D840F9F7FBF805463046F9F7F7F801462C
:107280002846F9F7FFF90546D8F84000C0F3080092
:10729000F9F7ECF806464FF064513846F9F73EF935
:1072A00001463046F9F732F84FF07E51F9F72EF8E3
:1072B00001462846F9F732F9054642E03046F9F72B
:1072C000D5F801464F48F9F7DDF905464A4B186CE9
:1072D000C0F30800F9F7CAF806464FF06451384683
:1072E000F9F71CF901463046F9F710F84FF07E51D6
:1072F000F9F70CF801462846F9F710F9054620E0A1
:107300003046F9F7B3F801463C48F9F7BBF90546B2
:10731000394B186CC0F30800F9F7A8F806464FF08F
:1073200064513846F9F7FAF801463046F8F7EEFFAF
:107330004FF07E51F8F7EAFF01462846F9F7EEF8DC
:1073400005462D4E306CC0F34620F9F78FF84FF00C
:107350007E51F8F7DBFF01462846F9F793F9F9F774
:107360002DFA2060306CC0F30640F9F77FF84FF03B
:107370007E51F8F7CBFF01462846F9F783F9F9F774
:107380001DFA6060306CC0F30660F9F76FF84FF0DB
:107390007E51F8F7BBFF01462846F9F773F9F9F774
:1073A0000DFAA060BDE8F0813046F9F75FF80146BC
:1073B0001548F9F767F905460F4B186CC0F308003C
:1073C000F9F754F806464FF064513846F9F7A6F835
:1073D00001463046F8F79AFF4FF07E51F8F796FFD6
:1073E00001462846F9F79AF80546AAE700232360E4
:1073F0006360A360D6E700BF004402580024744ACB
:107400000090D0030024744C0024F44A2DE9F0418C
:107410000446864B9D6A9E6AC6F30516D86A00F03C
:1074200001005B6BC3F3CC0303FB00F0F9F71EF81C
:10743000002E00F0F58005F003050746012D79D0F8
:10744000022D00F0CB800DB33046F9F70FF801465E
:107450007748F9F717F90546744B186BC0F3080025
:10746000F9F704F806464FF064513846F9F756F834
:1074700001463046F8F74AFF4FF07E51F8F746FFD5
:1074800001462846F9F74AF8054674E0674B1B6841
:1074900013F0200F2CD0DFF89481D8F80030C3F31C
:1074A000C1036448D840F8F7E1FF05463046F8F7D5
:1074B000DDFF01462846F9F7E5F80546D8F8300023
:1074C000C0F30800F8F7D2FF06464FF06451384683
:1074D000F9F724F801463046F8F718FF4FF07E51CF
:1074E000F8F714FF01462846F9F718F8054642E078
:1074F0003046F8F7BBFF01464D48F9F7C3F805469B
:107500004A4B186BC0F30800F8F7B0FF06464FF07F
:1075100064513846F9F702F801463046F8F7F6FEAE
:107520004FF07E51F8F7F2FE01462846F8F7F6FFD5
:10753000054620E03046F8F799FF01463E48F9F746
:10754000A1F80546394B186BC0F30800F8F78EFF19
:1075500006464FF064513846F8F7E0FF01463046E2
:10756000F8F7D4FE4FF07E51F8F7D0FE01462846DA
:10757000F8F7D4FF05462D4E306BC0F34620F8F7E0
:1075800075FF4FF07E51F8F7C1FE01462846F9F726
:1075900079F8F9F713F92060306BC0F30640F8F77B
:1075A00065FF4FF07E51F8F7B1FE01462846F9F726
:1075B00069F8F9F703F96060306BC0F30660F8F71B
:1075C00055FF4FF07E51F8F7A1FE01462846F9F726
:1075D00059F8F9F7F3F8A060BDE8F0813046F8F704
:1075E00045FF01461548F9F74DF805460F4B186B56
:1075F000C0F30800F8F73AFF06464FF064513846EA
:10760000F8F78CFF01463046F8F780FE4FF07E51C8
:10761000F8F77CFE01462846F8F780FF0546AAE702
:10762000002323606360A360D6E700BF00440258D4
:107630000024744C0090D0030024744A0024F44ABF
:1076400000B58BB0A0F580730B432ED0A0F500736E
:107650000B437ED0A0F580630B4300F0D480A0F5EF
:1076600000630B4300F02C81A0F580530B4300F026
:107670008B81A0F500530B4300F0E381A0F50023BC
:107680000B4300F02C82A0F580330B4300F06F8297
:10769000A0F580430B4300F09082A0F5004050EA33
:1076A000010300F0D382002001E3954B1B6D03F032
:1076B0000703042B00F2F282DFE803F005101B033E
:1076C00026009048F3E28E4B186810F0007000F02E
:1076D000EE8207A8FFF79AFE0898E8E2884B186840
:1076E00010F0006000F0E38204A8FFF75BFC049850
:1076F000DDE2834B186810F0005000F0D88201A83A
:10770000FFF76AFD0198D2E27D4AD36C03F0405343
:10771000126812F0040F07D033B9794B1B68C3F31A
:10772000C1037948D840C2E2754A126812F4807FDA
:1077300003D0B3F1805F00F0B382714A126812F493
:10774000003F00F0AF82B3F1005F00F0AD82002097
:10775000ADE26B4B1B6D03F4E073802B33D015D976
:10776000C02B00F0A382B3F5807F1FD1644AD36C95
:1077700003F04053126812F0040F2FD073BB604B1C
:107780001B68C3F3C1036048D84090E283B1402B2B
:107790000AD15B4B186810F0006000F0888204A8E2
:1077A000FFF700FC049882E2002080E200207EE2E5
:1077B000534B186810F0007000F0798207A8FFF7AB
:1077C00025FE089873E24E4B186810F0005000F048
:1077D0006E8201A8FFF700FD019868E2484A12682E
:1077E00012F4807F03D0B3F1805F00F06382444ADB
:1077F000126812F4003F00F05F82B3F1005F00F006
:107800005D82002053E23E4B9B6D03F46003B3F5B1
:10781000800F35D016D9B3F5C00F00F05182B3F503
:10782000000F20D1364AD36C03F04053126812F097
:10783000040F30D07BBB324B1B68C3F3C10332480B
:10784000D84034E28BB1B3F5001F0AD12C4B186835
:1078500010F0006000F02B8204A8FFF7A3FB04984F
:1078600025E2002023E2002021E2254B186810F0D9
:10787000007000F01C8207A8FFF7C8FD089816E208
:107880001F4B186810F0005000F0118201A8FFF79C
:10789000A3FC01980BE21A4A126812F4807F03D00D
:1078A000B3F1805F00F00E82154A126812F4003FB7
:1078B00000F00A82B3F1005F00F008820020F6E1D8
:1078C0000F4B9B6D03F0E063B3F1007F3CD01DD9FB
:1078D000B3F1407F00F0FC81B3F1806F27D1084AFB
:1078E000D36C03F04053126812F0040F37D0002B12
:1078F00035D1034B1B68C3F3C1030348D840D6E11D
:10790000004402580080BB000090D0038BB1B3F15B
:10791000807F0AD19A4B186810F0006000F0C78190
:1079200004A8FFF73FFB0498C1E10020BFE100205D
:10793000BDE1934B186810F0007000F0B88107A803
:10794000FFF764FD0898B2E18D4B186810F0005005
:1079500000F0AD8101A8FFF73FFC0198A7E1884A3C
:10796000126812F4807F03D0B3F1805F00F0B2811F
:10797000834A126812F4003F00F0AE81B3F1005F59
:1079800000F0AC81002092E17D4B1B6D03F4E043DD
:10799000B3F5005F35D016D9B3F5405F00F0A08194
:1079A000B3F5804F20D1764AD36C03F04053126870
:1079B00012F0040F30D07BBB714B1B68C3F3C103C3
:1079C0007048D84073E18BB1B3F5805F0AD16C4B3E
:1079D000186810F0006000F06A8104A8FFF7E2FA6E
:1079E000049864E1002062E1002060E1644B1868C3
:1079F00010F0007000F05B8107A8FFF707FD089802
:107A000055E15F4B186810F0005000F0508101A85C
:107A1000FFF7E2FB01984AE1594A126812F4807FAD
:107A200003D0B3F1805F00F05D81554A126812F413
:107A3000003F00F05981B3F1005F00F05781002052
:107A400035E14F4B1B6D03F4E023B3F5403F32D0DB
:107A500016D8B3F5803F23D0B3F5003F0AD1484B89
:107A6000186810F0005000F0228101A8FFF7B4FB65
:107A700002981CE113B9FEF70DFC18E1002016E195
:107A8000B3F5802F23D0B3F5A02F07D13C4B186856
:107A900010F4003000F00B813B4808E1002006E1C3
:107AA000374B186810F0006000F0018104A8FFF760
:107AB00079FA0598FBE0324B186810F0040000F0EA
:107AC000F6801B68C3F3C1032E48D840EFE02C4B6F
:107AD000186810F4807000F0EA802C48E7E0284B2A
:107AE0009B6D03F44033B3F5803F10D0B3F5003FF6
:107AF00018D00BB10020DAE0214B186810F00060BC
:107B000000F0D58004A8FFF74DFA0498CFE01C4B95
:107B1000186810F0005000F0CA8001A8FFF75CFB65
:107B20000398C4E0164AD36C03F04053126812F075
:107B3000040F07D033B9124B1B68C3F3C1031148BC
:107B4000D840B4E00E4A126812F4807F03D0B3F13B
:107B5000805F00F0CD800A4A126812F4003F00F006
:107B6000C980B3F1005F00F0C78000209FE0044BA4
:107B7000DB6C13F480330BD0ABB9002097E000BF6F
:107B8000004402580090D00300127A0000093D0022
:107B90005A4B186810F0007000F0898007A8FFF7B2
:107BA00035FC089883E0554B186810F000607ED0D3
:107BB00004A8FFF7F7F9069879E0504B9B6D03F0A6
:107BC000E043B3F1405F2FD015D8B3F1805F21D0EF
:107BD000B3F1005F09D1494B186810F0005066D02E
:107BE00001A8FFF7F9FA029861E013B9FFF7C8F9A5
:107BF0005DE000205BE0B3F1804F20D0B3F1A04FF7
:107C000006D13E4B186810F4003050D03C484EE08E
:107C100000204CE0394B186810F0006047D004A8F1
:107C2000FFF7C0F9059842E0344B186810F00400E3
:107C30003DD01B68C3F3C1033248D84037E02F4B17
:107C4000186810F4807032D02F4830E02B4B1B6D39
:107C500003F04053B3F1805F0CD0B3F1005F13D059
:107C60000BB1002023E0254B186810F400301ED023
:107C700023481CE0214B186810F0007017D007A8AB
:107C8000FFF7C4FB089812E01C4B186810F0006066
:107C90000DD004A8FFF786F9059808E0002006E05B
:107CA000194804E0002002E0154800E017480BB036
:107CB0005DF804FB1448FAE70020F8E71048F6E7FF
:107CC0001248F4E71048F2E70020F0E70C48EEE72E
:107CD0000E48ECE70C48EAE70020E8E70848E6E74A
:107CE0000A48E4E70848E2E70020E0E70448DEE766
:107CF0000548DCE70020DAE70148D8E700440258ED
:107D000000127A000090D00300093D000080BB0003
:107D1000F0B4036A23F001030362036A46688469CE
:107D20001F4A22400D68154323F002038C68234349
:107D30001C4A1D4CA04218BF90420CBF01220022D9
:107D40000CD004F58044A04214BF00240124174F36
:107D5000B84203D014B9164CA04205D123F0080351
:107D6000CC68234323F004035AB9124A904214BF4B
:107D7000002201220D4CA04203D012B90C4A9042BD
:107D800007D126F4407C4A6942EA0C0C8E6946EA27
:107D90000C06466085614A6842630362F0BC704726
:107DA0008CFFFEFF00000140000401400040014044
:107DB000004801400044014070B4036A23F480731A
:107DC0000362036A4568C4691A4A22400E68164372
:107DD00023F400738A6843EA0223174A174CA0422F
:107DE00018BF90420CBF0122002206D123F4006389
:107DF000CC6843EA042323F480635AB9104A9042C2
:107E000014BF002201220F4CA04203D012B90E4A27
:107E1000904207D125F4405C4A694CEA021C8D6906
:107E20004CEA05154560C6614A68C263036270BCCE
:107E3000704700BF8CFFFEFF0000014000040140BE
:107E400000440140004001400048014070B4036A12
:107E500023F480530362036A4468C569144A2A40C4
:107E60000D6842EA052223F400538D6843EA053386
:107E7000104E114DA84218BFB0420DD005F58045F7
:107E8000A84214BF0025012506F58046B04203D064
:107E900015B90A4DA84204D124F480444D6944EA3E
:107EA00085144460C2614A680264036270BC704712
:107EB000FF8CFFFE0000014000040140004801402B
:107EC00070B4036A23F480330362036A4268456D29
:107ED000144C2C400D682C4323F400338D6843EA86
:107EE0000543114E114DA84218BFB0420DD005F503
:107EF0008045A84214BF0025012506F58046B04202
:107F000003D015B90A4DA84204D122F480324D693C
:107F100042EA0522426044654A688265036270BC99
:107F2000704700BF8FFFFEFF0000014000040140CA
:107F30000048014070B4036A23F480130362036AAB
:107F40004468456D144A2A400D6842EA052223F42C
:107F500000138D6843EA0553104E114DA84218BF17
:107F6000B0420DD005F58045A84214BF002501257B
:107F700006F58046B04203D015B90A4DA84204D197
:107F800024F480244D6944EA8524446042654A68AB
:107F9000C265036270BC7047FF8FFFFE00000140A6
:107FA000000401400048014010B4036A046A24F050
:107FB00001040462846924F0F00C4CEA021223F0FC
:107FC0000A030B438261036210BC704730B4046A39
:107FD00024F0100404628469056A24F4407C4CEAAD
:107FE000022C2CF4704C1B039BB243EA0C0325F0CB
:107FF000A005090101F0A00129438361016230BCA1
:10800000704710B4046A24F0100404628469036A9F
:1080100024F4704C4CEA023223F0A00343EA01132B
:108020008261036210BC704730B4046A24F4807427
:108030000462C469056A24F0030C4CEA020C2CF0BB
:10804000F00C1B01DBB243EA0C0325F420650902A6
:1080500001F420612943C361016230BC704730B430
:10806000046A24F480540462C469056A24F4407CE0
:108070004CEA022C2CF4704C1B039BB243EA0C0319
:1080800025F42045090301F420412943C36101621D
:1080900030BC70477047704770477047704710B5E5
:1080A000044603681A6912F0020F11D0DA6812F060
:1080B000020F0DD06FF002021A61012303770368EB
:1080C0009B6913F0030F79D0FAF734FB0023237771
:1080D00023681A6912F0040F12D0DA6812F0040F44
:1080E0000ED06FF004021A610223237723689B6984
:1080F00013F4407F68D02046FAF71CFB0023237757
:1081000023681A6912F0080F12D0DA6812F0080F0B
:108110000ED06FF008021A61042323772368DB690D
:1081200013F0030F57D02046FAF704FB0023237700
:1081300023681A6912F0100F12D0DA6812F0100FCB
:108140000ED06FF010021A61082323772368DB69D1
:1081500013F4407F46D02046FAF7ECFA0023237749
:1081600023681A6912F0010F03D0DA6812F0010FC8
:108170003FD123681A6912F0800F03D0DA6812F039
:10818000800F3DD123681A6912F4807F03D0DA682A
:1081900012F0800F3BD123681A6912F0400F03D010
:1081A000DA6812F0400F39D123681A6912F0200FF3
:1081B00003D0DA6812F0200F37D110BDFFF76CFF43
:1081C0002046FFF76AFF81E72046FFF765FF20465C
:1081D000FFF763FF92E72046FFF75EFF2046FFF7B9
:1081E0005CFFA3E72046FFF757FF2046FFF755FF48
:1081F000B4E76FF001021A612046FFF74CFFB8E7C1
:108200006FF080021A61204600F085FDBAE76FF436
:1082100080721A61204600F07FFDBCE76FF04002DB
:108220001A612046FFF73AFFBEE76FF020021A619D
:10823000204600F06FFDC0E730B50368394A904230
:1082400014BF4FF0000E4FF0010EB0F1804F14BF7D
:1082500072464EF00102AAB9334CA04214BF00246A
:108260000124324DA8420DD064B904F1804404F5D4
:108270008234A04214BF0024012405F50065A84201
:1082800000D01CB123F070034C68234312BB264A74
:10829000904214BF00220122244CA0421AD0CAB935
:1082A00002F1804202F58232904214BF0022012284
:1082B00004F50064A0420DD062B91D4A904214BF7B
:1082C0000022012204F59A34A04203D012B9194ABF
:1082D000904204D123F4407CCB6843EA0C0323F0A2
:1082E00080034A69134303608A68C2620A68826233
:1082F000114A904214BF73464EF0010363B90C4B10
:10830000984214BF0023012302F57052904203D01B
:1083100013B9084B984201D10B69036301234361F0
:1083200030BD00BF000001400008004000040040D4
:1083300000440140004801400004014060B310B512
:10834000044690F83D3013B3022384F83D302146B3
:1083500051F8040BFFF770FF012384F8483084F8CC
:108360003E3084F83F3084F8403084F8413084F85F
:10837000423084F8433084F8443084F8453084F83F
:10838000463084F8473084F83D30002010BD80F836
:108390003C30FAF79DF8D7E70120704760B310B57D
:1083A000044690F83D3013B3022384F83D30214653
:1083B00051F8040BFFF740FF012384F8483084F89C
:1083C0003E3084F83F3084F8403084F8413084F8FF
:1083D000423084F8433084F8443084F8453084F8DF
:1083E000463084F8473084F83D30002010BD80F8D6
:1083F0003C30FAF71DF9D7E70120704760B310B59C
:10840000044690F83D3013B3022384F83D302146F2
:1084100051F8040BFFF710FF012384F8483084F86B
:108420003E3084F83F3084F8403084F8413084F89E
:10843000423084F8433084F8443084F8453084F87E
:10844000463084F8473084F83D30002010BD80F875
:108450003C30FFF71FFED7E70120704770B4036A76
:1084600023F010030362036A456884691A4A2240B4
:108470000E6842EA062623F020038A6843EA0213C4
:10848000164A174CA04218BF90420CBF012200228E
:1084900006D123F08003CC6843EA041323F04003A1
:1084A0005AB9104A904214BF002201220E4CA04239
:1084B00003D012B90D4A904207D125F4406C4A69A5
:1084C0004CEA820C8D694CEA8505456086614A68F4
:1084D0008263036270BC7047FF8CFFFE00000140A6
:1084E00000040140004401400040014000480140B8
:1084F00038B590F83C30012B00F0958004460D46CD
:10850000012380F83C30142A00F28880DFE802F072
:108510000B8686861F86868634868686488686866D
:108520005D86868671000068FFF7F2FB226893691A
:1085300043F0080393612268936923F00403936175
:108540002268936929690B439361002067E0006802
:10855000FFF784FF2268936943F400639361226804
:10856000936923F48063936122689369296943EADC
:1085700001239361002052E00068FFF71DFC226890
:10858000D36943F00803D3612268D36923F004035D
:10859000D3612268D36929690B43D36100203EE08F
:1085A0000068FFF753FC2268D36943F40063D3618A
:1085B0002268D36923F48063D3612268D36929696F
:1085C00043EA0123D361002029E00068FFF778FC2B
:1085D0002268536D43F0080353652268536D23F0FE
:1085E000040353652268536D29690B4353650020CA
:1085F00015E00068FFF79EFC2268536D43F40063AA
:1086000053652268536D23F4806353652268536D6C
:10861000296943EA01235365002000E0012000237B
:1086200084F83C3038BD0220FCE7000070B494466A
:10863000046A24F0010404628469066A1D4DB0F1E5
:10864000804F18BFA84223D01B4A904214BF00227B
:108650000122A5F57C45A8421AD0CAB902F1804290
:1086600002F58232904214BF0022012205F5006516
:10867000A8420DD062B9114A904214BF00220122D3
:1086800005F54065A84203D012B944F0010203E0A9
:1086900024F0030242EA0C0222F0F0021B01DBB2DA
:1086A000134326F00A0201F00A01114383610162BB
:1086B00070BC7047000001400008004000400140CD
:1086C00038B590F83C30012B5AD004460D460123B2
:1086D00080F83C3052B1042A1AD0082A2BD00C2A38
:1086E0003BD00120002384F83C3038BDCB684A6879
:1086F00009680068FFF79AFF2268936923F00C036A
:10870000936122689369A9680B4393610020E9E7AC
:10871000CB684A6809680068FFF758FC22689369CB
:1087200023F44063936122689369A96843EA0123B3
:1087300093610020D6E7CB684A6809680068FFF7B4
:1087400073FC2268D36923F00C03D3612268D369D8
:10875000A9680B43D3610020C4E7CB684A68096865
:108760000068FFF77CFC2268D36923F44063D3617F
:108770002268D369A96843EA0123D3610020B1E7E5
:108780000220B2E710B4846824F47F4C42EA03224A
:108790000A4342EA0C02826010BC704710B50468BC
:1087A000A3684C4A1A404B6813434B4A1A400B6863
:1087B0001343A3604B68602B68D01CD8402B50D06B
:1087C00008D9502B15D10A6989680068FFF7ECFBBE
:1087D000002035E0202B60D003D9302B07D00120BA
:1087E0002EE0002B5BD0102B5BD1002028E0002076
:1087F00026E0012024E0702B2BD001D201201FE0C5
:10880000364A93424FD008D9B3F5001F57D018D934
:10881000334A934259D1002012E0303A934244D077
:1088200007D9304A934246D01032934245D10020B6
:1088300006E0B3F5801F3AD0B3F1101F39D1002004
:1088400010BD294A93423CD0103293423BD10020C4
:10885000F6E70B698A68C9680068FFF793FF002094
:10886000EEE70B68052B32D003681C6A1A6A22F007
:1088700001021A620268936923F0F003096943EA6E
:108880000113936103681C620020D9E70A698968B3
:108890000068FFF7B6FB0020D2E70020D0E70020F9
:1088A000CEE70120CCE70020CAE70020C8E700207F
:1088B000C6E70120C4E70020C2E70120C0E700208E
:1088C000BEE70020BCE70120BAE70120B8E701209D
:1088D000B6E700BF8FFFCFFFF8FFFEFF500010008C
:1088E00010002000300010006000100090F83C30B4
:1088F000012B22D010B50446012380F83C3002231E
:1089000080F83D30FFF74AFF80B92268D36823F032
:108910004003D3602268D36823F48043D3600123EB
:1089200084F83D30002384F83C3010BD012084F8E9
:108930003D00002384F83C30F7E70220704701F047
:108940001F01012303FA01FC036A23EA0C030362FB
:10895000036A02FA01F10B430362704710B5044643
:10896000084600294ED194F83E30DBB2013B18BFD7
:108970000123002B40F09B8000286ED1022384F855
:108980003E30012201462068FFF7D9FF23684A499B
:108990004A4A934218BF8B420BD002F57052934261
:1089A00007D002F58062934203D002F580629342C1
:1089B00003D15A6C42F400425A6423683E4AB3F130
:1089C000804F18BF934264D0A2F57C42934260D09E
:1089D00002F5806293425CD002F58062934258D0E7
:1089E00002F57842934254D0A2F56C42934250D0A3
:1089F00002F5943293424CD01A6842F001021A6098
:108A0000002055E004290CD0082911D00C2916D0DB
:108A100010291BD094F84330DBB2013B18BF01236F
:108A2000A7E794F83F30DBB2013B18BF0123A0E772
:108A300094F84030DBB2013B18BF012399E794F86A
:108A40004130DBB2013B18BF012392E794F842307A
:108A5000DBB2013B18BF01238BE7042809D00828AB
:108A60000BD00C280DD010280FD0022384F84330EF
:108A700087E7022384F83F3083E7022384F84030FD
:108A80007FE7022384F841307BE7022384F84230F9
:108A900077E799680A4A0A40062A18BFB2F5803F6C
:108AA00007D01A6842F001021A60002000E001209D
:108AB00010BD0020FCE700BF0000014000040140A1
:108AC0000700010010B504460B4611BB90F83E109C
:108AD000C9B2002B39D194F84420D2B2012A08BF80
:108AE000012940F0BD80002B3FD1022284F83E20B6
:108AF000002B56D1022284F844200C2B00F2B280C5
:108B0000DFE803F05FB0B0B08EB0B0B094B0B0B0FA
:108B10009A00042909D008290BD00C290DD010295E
:108B20000FD090F84310C9B2D3E790F83F10C9B204
:108B3000CFE790F84010C9B2CBE790F84110C9B226
:108B4000C7E790F84210C9B2C3E7042B05D0082B41
:108B500007D094F84720D2B2C0E794F84520D2B2AB
:108B6000BCE794F84620D2B2B8E7042B09D0082B12
:108B70000BD00C2B0DD0102B0FD0022284F84320E9
:108B8000B6E7022284F83F20B2E7022284F84020B0
:108B9000AEE7022284F84120AAE7022284F84220AC
:108BA000A6E7042B05D0082B07D0022284F8472023
:108BB000A3E7022284F845209FE7022284F846209A
:108BC0009BE72168CA6842F00202CA600122194686
:108BD0002068FFF7B4FE2368244AB3F1804F18BF22
:108BE00093422FD0A2F57C4293422BD002F58062B3
:108BF000934227D002F58062934223D002F5784257
:108C000093421FD0A2F56C4293421BD002F59432DE
:108C1000934217D01A6842F001021A60002022E045
:108C20002168CA6842F00402CA60CFE72168CA68B6
:108C300042F00802CA60C9E72168CA6842F010021F
:108C4000CA60C3E799680A4A0A40062A18BFB2F503
:108C5000803F09D01A6842F001021A60002002E049
:108C6000012000E0012010BD0020FCE700000140D1
:108C70000700010090F83C30012B45D070B401236F
:108C800080F83C30022380F83D3003685A689C68C5
:108C90001E4E1F4DAB4218BFB34203D122F47002E7
:108CA0004D682A4322F070020D682A435A60036817
:108CB000164AB3F1804F18BF934217D0A2F57C42F9
:108CC000934213D002F5806293420FD002F5806286
:108CD00093420BD002F57842934207D0A2F56C4242
:108CE000934203D002F59432934204D124F08004DD
:108CF0008A6814439C60012380F83D30002380F88B
:108D00003C30184670BC704702207047000001409C
:108D100000040140704770477047026852E8003F06
:108D200023F0C00342E800310029F6D1026802F1C5
:108D3000080353E8003F23F40003083242E80031FF
:108D40000029F3D12023C0F888307047026852E828
:108D5000003F23F4907342E800310029F6D1026805
:108D600002F1080353E8001F0D4B0B40083242E8A4
:108D700000310029F3D1C36E012B06D02023C0F8A7
:108D80008C300023C36643677047026852E8003F97
:108D900023F0100342E800310029F6D1EEE700BFCE
:108DA000FEFFFFEF1346D0F88820202A3DD110B5F2
:108DB0000446002B18BF002939D00165A0F85430B3
:108DC000A0F856300022C0F890202122C0F8882058
:108DD000C26FCAB11749D163C26F17491164C26F1C
:108DE0001649D164C26F0021116502682832016DF5
:108DF000C06FFBF779FB38B11023C4F89030202303
:108E0000C4F8883001200FE0236840221A622268EB
:108E100002F1080353E8003F43F08003083242E8C0
:108E200000310029F3D1002010BD0220704701203D
:108E3000FAE700BF438E0008AF8E0008BB8E000823
:108E4000704708B50346806BDB69B3F5807F18D0A7
:108E50000023A0F85630026802F1080353E8003FEF
:108E600023F08003083242E800310029F3D1026880
:108E700052E8003F43F0400342E800310029F6D1B8
:108E800008BDFFF7DDFFFBE708B5026852E8003FC9
:108E900023F0400342E800310029F6D12023C0F836
:108EA000883000238367FFF7CBFF08BD704708B504
:108EB000806BFFF7FBFF08BD704738B5846BD4F8B3
:108EC0008820D4F88C5023689B6813F0800F01D061
:108ED000212A10D023689B6813F0400F01D0222D67
:108EE00010D0D4F8903043F01003C4F890302046EE
:108EF000FFF7E2FF38BD0023A4F856302046FFF705
:108F00000CFFE7E70023A4F85E302046FFF71EFFC2
:108F1000E7E708B5806B0023A0F85E30A0F8563074
:108F2000FFF7CAFF08BD704770B504460168CB69FA
:108F300008688D6840F60F021A4008D113F0200F20
:108F400005D010F0200F34D115F0805F31D12AB157
:108F50008B4A2A4033D18B4E304230D1E26E012A07
:108F600000F0C68013F4801F03D015F4800F40F08A
:108F70009B8113F0800F07D010F0800F40F09B8191
:108F800015F4000F40F0978113F0400F03D010F05C
:108F9000400F40F0978113F4000F03D010F0804F82
:108FA00040F0948113F0807F02D00028C0F29281BB
:108FB00070BD636F002BFBD020469847F8E713F095
:108FC000010F09D010F4807F06D001260E62D4F87C
:108FD00090103143C4F8901013F0020F0BD015F02D
:108FE000010F08D0216802260E62D4F8901041F0DB
:108FF0000401C4F8901013F0040F0BD015F0010F0A
:1090000008D0216804260E62D4F8901041F00201C5
:10901000C4F8901013F0080F0BD010F0200F00D1FF
:109020003AB1226808211162D4F890200A43C4F8AA
:10903000902013F4006F0CD010F0806F09D02268DC
:109040004FF400611162D4F8902042F02002C4F87D
:109050009020D4F89020002AAAD013F0200F09D035
:1090600010F0200F02D115F0805F03D0636F0BB1B9
:1090700020469847D4F8902023689B6813F0400F4F
:1090800002D112F0280F2CD02046FFF75FFE236894
:109090009B6813F0400F20D0226802F1080353E8C8
:1090A000003F23F04003083242E800310029F3D1A9
:1090B000D4F880306BB1344A1A65D4F88000FBF7DD
:1090C000FFFC00283FF474AFD4F88000036D98478C
:1090D0006EE72046FFF7F0FE6AE72046FFF7ECFE5A
:1090E00066E72046FFF7E8FE0023C4F890305FE70C
:1090F00013F0100F3FF436AF10F0100F3FF432AF03
:1091000010230B6223689B6813F0400F00F09280DD
:10911000D4F8802013681D481D498B4218BF834234
:1091200038D018318B4235D018318B4232D01831BB
:109130008B422FD018318B422CD018318B4229D042
:1091400018318B4226D001F556718B4222D018314E
:109150008B421FD018318B421CD018318B4219D052
:1091600018318B4216D018318B4213D018318B42F4
:1091700010D018318B420DD05B689BB20CE000BF61
:109180000100001020010004138F000810000240AD
:10919000280002405B689BB2002B3FF409AFB4F893
:1091A0005C1099427FF604AFA4F85E30D369B3F542
:1091B000807F32D0226852E8003F23F4807342E877
:1091C00000310029F6D1226802F1080353E8003F7C
:1091D00023F00103083242E800310029F3D122686C
:1091E00002F1080353E8003F23F04003083242E84D
:1091F00000310029F3D12023C4F88C300023E3662A
:10920000226852E8003F23F0100342E800310029B1
:10921000F6D1D4F88000FBF7B3FA02232367B4F841
:109220005C10B4F85E309BB2C91A89B22046FFF7D1
:109230007AFEBDE6B4F85C10B4F85E309BB2C91A91
:1092400089B2B4F85E309BB2002B3FF4B1AE002976
:109250003FF4AEAE226852E8003F23F4907342E838
:1092600000300028F6D1226802F1080353E8000F0D
:109270001A4B0340083242E800300028F3D1202383
:10928000C4F88C300023E3666367226852E8003F2D
:1092900023F0100342E800300028F6D102232367B0
:1092A0002046FFF740FE83E64FF480130B62204612
:1092B00001F0DCF87CE6A36F002B3FF479AE20468A
:1092C000984775E62046FFF7DFFD71E6204601F07E
:1092D000CFF86DE6204601F0CAF869E6FEFFFFEF21
:1092E00008B5B0F86030D0F88C20222A05D002688A
:1092F000936943F00803936108BD0268516ADBB2C9
:10930000826D0B401370836D01338365B0F85E305E
:109310009BB2013B9BB2A0F85E30B0F85E309BB2CE
:10932000002BE9D1026852E8003F23F4907342E831
:1093300000310029F6D1026802F1080353E8003F2A
:1093400023F00103083242E800310029F3D1202341
:10935000C0F88C300023436703670368164A9342C2
:109360000CD05B6813F4000F08D0026852E8003F8D
:1093700023F0806342E800310029F6D1C36E012B4F
:1093800016D10023C366026852E8003F23F01003A1
:1093900042E800310029F6D10368DA6912F0100FB3
:1093A00001D010221A62B0F85C10FFF7BCFDA3E7F1
:1093B000F9F716FBA0E700BF000C005808B5B0F89D
:1093C0006020D0F88C30222B05D00268936943F0DE
:1093D0000803936108BD03685B6A816D13400B80CD
:1093E000836D02338365B0F85E309BB2013B9BB264
:1093F000A0F85E30B0F85E309BB2002BEAD1026874
:1094000052E8003F23F4907342E800310029F6D17E
:10941000026802F1080353E8003F23F00103083219
:1094200042E800310029F3D12023C0F88C3000231A
:10943000436703670368164A93420CD05B6813F4D2
:10944000000F08D0026852E8003F23F0806342E832
:1094500000310029F6D1C36E012B16D10023C3665B
:10946000026852E8003F23F0100342E8003100296F
:10947000F6D10368DA6912F0100F01D010221A62D7
:10948000B0F85C10FFF74FFDA4E7F9F7A9FAA1E7E0
:10949000000C00582DE9F843B0F860600368DD69FE
:1094A000D3F80090D3F80880D0F88C20222A05D079
:1094B0009A6942F008029A61BDE8F8830446B0F860
:1094C000687008E0D4F89030002B4CD1B4F85E30CE
:1094D0009BB2002B4ED0002F00F0988015F0200F8B
:1094E00000F094802368596AF3B2A26D0B401370A8
:1094F000A36D0133A365B4F85E309BB2013B9BB210
:10950000A4F85E302368DD6915F0070FDED015F092
:10951000010F09D019F4807F06D001221A62D4F815
:1095200090301343C4F8903015F0020F0BD018F0B0
:10953000010F08D0236802221A62D4F8903043F059
:109540000403C4F8903015F0040FBBD018F0010FDD
:10955000B8D0236804221A62D4F8903043F0020392
:10956000C4F89030AEE72046FFF7A6FC0023C4F80D
:109570009030ABE7226852E8003F23F4807342E862
:1095800000310029F6D1226802F1080353E8001FD8
:10959000304B0B40083242E800310029F3D1202340
:1095A000C4F88C3000236367236723682A4A9342F8
:1095B00003D05B6813F4000F06D1E36E012B0DD0CE
:1095C0002046F9F70DFA86E7226852E8003F23F0BB
:1095D000806342E800310029F6D1EEE70023E3661C
:1095E000226852E8003F23F0100342E800310029CE
:1095F000F6D12368DA6912F0100F01D010221A6236
:10960000B4F85C102046FFF78EFC64E7B4F85E30D7
:109610009BB2002B3FF450AFB4F868209A427FF61B
:109620004BAF226802F1080353E8003F23F0805358
:10963000083242E800310029F3D1084B6367226801
:1096400052E8003F43F0200342E800310029F6D100
:1096500032E700BFFEFFFFEF000C0058E192000868
:109660002DE9F843B0F860600368DD69D3F8009035
:10967000D3F80880D0F88C20222A05D09A6942F0CD
:1096800008029A61BDE8F8830446B0F8687008E003
:10969000D4F89030002B4BD1B4F85E309BB2002B45
:1096A0004DD0002F00F0978015F0200F00F0938030
:1096B00023685B6AA26D33401380A36D0233A365F8
:1096C000B4F85E309BB2013B9BB2A4F85E302368D5
:1096D000DD6915F0070FDFD015F0010F09D019F47F
:1096E000807F06D001221A62D4F890301343C4F868
:1096F000903015F0020F0BD018F0010F08D023683E
:1097000002221A62D4F8903043F00403C4F8903077
:1097100015F0040FBCD018F0010FB9D02368042253
:109720001A62D4F8903043F00203C4F89030AFE7E7
:109730002046FFF7C1FB0023C4F89030ACE7226855
:1097400052E8003F23F4807342E800310029F6D14B
:10975000226802F1080353E8001F304B0B40083227
:1097600042E800310029F3D12023C4F88C300023D3
:109770006367236723682A4A934203D05B6813F424
:10978000000F06D1E36E012B0DD02046F9F728F922
:1097900087E7226852E8003F23F0806342E8003107
:1097A0000029F6D1EEE70023E366226852E8003F85
:1097B00023F0100342E800310029F6D12368DA696A
:1097C00012F0100F01D010221A62B4F85C1020467B
:1097D000FFF7A9FB65E7B4F85E309BB2002B3FF4BE
:1097E00051AFB4F868209A427FF64CAF226802F17C
:1097F000080353E8003F23F08053083242E8003169
:109800000029F3D1074B6367226852E8003F43F019
:10981000200342E800310029F6D133E7FEFFFFEFD5
:10982000000C0058BD93000870B586B0044601686E
:1098300083680269134342691343C269134308688A
:10984000884A024013430B602268536823F4405354
:10985000E1680B435360A1692268834B9A4201D0AF
:10986000236A19439068814B03400B43936022683D
:10987000D36A23F00F03616A0B43D36222687C4BE7
:109880009A4221D07B4B9A4200F08C807A4B9A42CC
:1098900000F0A280794B9A4200F0B580784B9A4252
:1098A00000F0C880774B9A4200F0F480764B9A42E1
:1098B00000F01981754B9A4200F02C816A4B9A4254
:1098C00000F03F81802333E0714B5B6D03F0380380
:1098D000282B65D8DFE813F02900640064006400D9
:1098E00064006400640064004D016400640064006E
:1098F00064006400640064002B0064006400640081
:1099000064006400640064005E006400640064003D
:10991000640064006400640060006400640064002B
:1099200064006400640064006200012300E0082316
:109930004D498A4200F02F81E069B0F5004F00F0F8
:10994000AF81202B00F20782202B00F25182DFE84A
:1099500013F01E0224024F024F0227024F024F0251
:109960004F022C024F024F024F024F024F024F0292
:109970004F0231024F024F024F024F024F024F027D
:109980004F024F024F024F024F024F024F024F024F
:109990004F023D021023CBE72023C9E74023C7E74E
:1099A0008023C5E73A4B5B6D03F00703052B11D805
:1099B000DFE813F00600E10008000A000C000E00CA
:1099C0000023B5E70823B3E71023B1E72023AFE76F
:1099D0004023ADE78023ABE72D4B5B6D03F007031E
:1099E000052B0ED8DFE803F003C90507090B002398
:1099F0009EE708239CE710239AE7202398E740235B
:109A000096E7802394E7224B5B6D03F00703052B59
:109A10000ED8DFE803F003B40507090B002387E73E
:109A2000082385E7102383E7202381E740237FE78E
:109A300080237DE7164B5B6D03F00703052B0ED8E3
:109A4000DFE803F0039F0507090B002370E70823F5
:109A50006EE710236CE720236AE7402368E7802342
:109A600066E700BFF369FFCF000C0058FFF4FF1159
:109A7000001001400044004000480040004C0040FD
:109A8000005000400014014000780040007C00407D
:109A9000004402587D4B5B6D03F03803282B20D81F
:109AA000DFE803F0151F1F1F1F1F1F1F711F1F1F40
:109AB0001F1F1F1F171F1F1F1F1F1F1F191F1F1FC4
:109AC0001F1F1F1F1B1F1F1F1F1F1F1F1D000123E5
:109AD0002EE708232CE710232AE7202328E740233A
:109AE00026E7802324E7694B5B6D03F00703052B12
:109AF0000ED8DFE803F0034A0507090B002317E738
:109B0000082315E7102313E7202311E740230FE76D
:109B100080230DE75D4B5B6D03F00703052B0ED82B
:109B2000DFE803F003350507090B002300E70823EE
:109B3000FEE61023FCE62023FAE64023F8E6802325
:109B4000F6E603F50E339B6D03F00703052B0ED8E5
:109B5000DFE803F0031F0507090B0223E8E60823EB
:109B6000E6E61023E4E62023E2E64023E0E6802355
:109B7000DEE60423DCE60423DAE60423D8E6042345
:109B8000D6E60423D4E60423D2E60423D0E6042355
:109B9000CEE60423CCE6202B27D8022BC0F01A8176
:109BA000023B1E2B00F21881DFE813F05000160173
:109BB00056001601160116015B001601160116016A
:109BC0001601160116011601600016011601160194
:109BD00016011601160116011601160116011601CD
:109BE00016011601160116016C00402B2CD14FF402
:109BF0000040626A264B33F81220B0FBF2F365682E
:109C000005EB4501994200F2E980B3EB053F00F214
:109C1000E780002633463146F6F7F0FD090241EAB7
:109C2000106100026B08C0182A46334641F100015A
:109C3000F6F7E4FDA0F54072164B9A4200F2D2808E
:109C40002368D8603046D4E00120D2E0FDF798F9CF
:109C50000028CED10020CCE003A8FDF7A3F904989A
:109C6000F6E76846FDF7B8FA0198F1E7074B1B687D
:109C700013F0200F08D0054B1B68C3F3C10306483F
:109C8000D840E5E70548B4E70348B2E70044025886
:109C900030060108FFFC0F000090D00300093D00D2
:109CA000202B15D8202B00F29F80DFE803F03137FE
:109CB0009D9D3A9D9D9D3F9D9D9D9D9D9D9D449DEE
:109CC0009D9D9D9D9D9D9D9D9D9D9D9D9D9D5000AE
:109CD000402B1BD1626A4D4B33F81230B0FBF3F0CE
:109CE0006268530803EB4000B0FBF2F0A0F11002F1
:109CF0004FF6EF739A4279D883B223F00F03C0F383
:109D0000420018432368D860002072E0012070E010
:109D1000FCF7C0FA0028DDD100206AE0FCF7CCFA9D
:109D2000F8E703A8FDF73EF90498F3E76846FDF766
:109D300053FA0198EEE7364B1B6813F0200F08D05A
:109D4000334B1B68C3F3C1033248D840E2E73248C3
:109D5000C0E73048BEE7402B17D14FF40040626A9D
:109D60002A4B33F81230B0FBF3F0636800EB53007A
:109D7000B0FBF3F0A0F110024FF6EF739A4242D815
:109D8000236880B2D860002033E0012031E0FCF786
:109D900081FA0028E3D100202BE0FCF78DFAF8E7E8
:109DA00003A8FDF7FFF80498F3E76846FDF714FAF7
:109DB0000198EEE7164B1B6813F0200F08D0144BE8
:109DC0001B68C3F3C1031348D840E2E71248C6E753
:109DD0001048C4E701200CE001200AE0012008E05F
:109DE000012006E0012004E0012002E0012000E063
:109DF00001200123A4F86A30A4F8683000236367C7
:109E0000A36706B070BD0120F3E700BF300601086C
:109E1000004402580090D00300093D00836A13F00B
:109E2000010F06D00268536823F40033C16A0B4364
:109E30005360836A13F0020F06D00268536823F45C
:109E40008033016B0B435360836A13F0040F06D019
:109E50000268536823F48023416B0B435360836A89
:109E600013F0080F06D00268536823F40043816B97
:109E70000B435360836A13F0100F06D00268936897
:109E800023F48053C16B0B439360836A13F0200F5C
:109E900006D00268936823F40053016C0B4393606F
:109EA000836A13F0400F0AD00268536823F48013CA
:109EB000416C0B435360436CB3F5801F0BD0836A36
:109EC00013F0800F06D00268536823F40023C16C9E
:109ED0000B43536070470268536823F4C003816CDE
:109EE0000B435360EBE72DE9F84305460F46164652
:109EF0009946DDF820802C68E46937EA04030CBF3A
:109F00004FF0010C4FF0000CB44532D1B8F1FF3FD7
:109F1000F1D0F8F735FEA0EB090040452CD8B8F198
:109F2000000F2BD02B681A6812F0040FE3D0DA6907
:109F300012F0080F11D1DA6912F4006FDBD04FF480
:109F400000621A622846FEF701FF2023C5F8903010
:109F5000002385F8843003200CE008241C62284686
:109F6000FEF7F4FEC5F89040002385F88430012008
:109F700000E00020BDE8F8830320FBE70320F9E7B9
:109F80002DE9F04182B01E46D0F88830202B5BD1FD
:109F900004460D469046002A18BF002901D1012031
:109FA00053E00023C0F890302123C0F88830F8F740
:109FB000E7FD0746A4F85480A4F85680A368B3F5DB
:109FC000805F02D04FF0000816E0236943B34FF0E2
:109FD000000811E02023C4F88830032035E038F869
:109FE000023B2268C3F308039362B4F8562092B28E
:109FF000013A92B2A4F85620B4F856309BB293B10D
:10A0000000963B46002280212046FFF76CFF002887
:10A01000E0D1002DE3D015F8012B23689A62E4E724
:10A02000A8460025E8E700963B460022402120464E
:10A03000FFF759FF18B92023C4F8883005E0202322
:10A04000C4F88830032000E0022002B0BDE8F081AF
:10A050002DE9F04383B01E46D0F88C30202B7ED102
:10A0600004460D469046002A18BF002901D1012060
:10A0700076E00023C0F890302222C0F88C20C3661E
:10A08000F8F77EFD0746A4F85C80A4F85E80A3681C
:10A09000B3F5805F06D0A3B9226972B9FF22A4F894
:10A0A000602014E0226922B940F2FF12A4F8602077
:10A0B0000DE0FF22A4F8602009E07F22A4F86020D0
:10A0C00005E0B3F1805F0AD00022A4F86020B4F864
:10A0D0006080B3F5805F0CD04FF0000924E0226966
:10A0E0001AB97F22A4F86020F1E73F22A4F860208B
:10A0F000EDE7236913B14FF0000915E0A9460025EB
:10A1000012E02023C4F88C30032029E023685A6A27
:10A110005FFA88F3134005F8013BB4F85E2092B271
:10A12000013A92B2A4F85E20B4F85E309BB28BB1D3
:10A1300000963B46002220212046FFF7D4FE00284F
:10A14000DFD1002DE2D123685B6A08EA030329F816
:10A15000023BE2E72023C4F88C30002000E002201C
:10A1600003B0BDE8F08330B583B004460023C0F8E7
:10A170009030F8F705FD05462268126812F0080FC6
:10A1800010D123681B6813F0040F28D12023C4F8D2
:10A190008830C4F88C300020E066206784F88400A2
:10A1A00003B030BD6FF07E430093034600224FF4AE
:10A1B00000112046FFF797FE0028E2D0226852E8FF
:10A1C000003F23F0800342E800310029F6D120232C
:10A1D000C4F88830002384F884300320E0E76FF06F
:10A1E0007E4300932B4600224FF480012046FFF768
:10A1F0007AFE0028CAD0226852E8003F23F4907308
:10A2000042E800310029F6D1226802F1080353E840
:10A21000003F23F00103083242E800310029F3D166
:10A220002023C4F88C30002384F884300320B7E75F
:10A2300078B310B50446D0F888300BB32423C4F8A3
:10A2400088302268136823F0010313602046FFF76B
:10A25000EBFA012813D0A36ABBB92268536823F430
:10A26000904353602268936823F02A039360226826
:10A27000136843F0010313602046FFF774FF10BD1D
:10A2800080F88430F8F732FBD8E72046FFF7C6FDA8
:10A29000E3E701207047000010B48165A0F85C205E
:10A2A000A0F85E20002343678368B3F5805F06D083
:10A2B000A3B9036973B9FF23A0F8603014E0036900
:10A2C00023B940F2FF13A0F860300DE0FF23A0F89F
:10A2D000603009E07F23A0F8603005E0B3F1805FD3
:10A2E0002DD00023A0F860300023C0F89030222346
:10A2F000C0F88C30016801F1080353E8003F43F0D7
:10A300000103083141E80034002CF3D1436EB3F16E
:10A31000005F1ED08368B3F5805F42D0294B43674E
:10A320000369002B43D0026852E8003F43F4907366
:10A3300042E800310029F6D1002010BC70470369C3
:10A340001BB97F23A0F86030CEE73F23A0F8603030
:10A35000CAE7B0F868309342DCD88368B3F5805F11
:10A3600019D0194B4367036943B1026852E8003FB3
:10A3700043F4807342E800310029F6D1026802F10B
:10A38000080353E8003F43F08053083242E80031AD
:10A390000029F3D1D0E70369002BE2D10B4B4367CF
:10A3A000E1E70369002BB9D1094B4367B8E70268BD
:10A3B00052E8003F43F0200342E800310029F6D183
:10A3C000BAE700BFE1920008959400086196000882
:10A3D000BD93000838B5D0F88C30202B19D1002A55
:10A3E00018BF002917D00023C36603680B4CA34293
:10A3F0000CD05B6813F4000F08D0046854E8003FE9
:10A4000043F0806344E80035002DF6D1FFF744FFA8
:10A4100000E0022038BD0120FCE700BF000C00581E
:10A42000436E2BB90123A0F86A30A0F8683070475A
:10A4300030B403689A68C2F342629968490F094DC3
:10A440006B5C1B01084C615C93FBF1F3A0F86A3074
:10A45000AB5C1B01A25C93FBF2F3A0F8683030BC4C
:10A46000704700BF50060108480601087047704752
:10A47000704790F88430012B18D0012380F8843085
:10A480002423C0F8883003681A68196821F0010194
:10A49000196022F000520023436601680A602022FE
:10A4A000C0F8882080F88430184670470220704732
:10A4B00038B590F88430012B1DD00446012380F874
:10A4C00084302423C0F8883003681D681A6822F09D
:10A4D00001021A600268936823F060431943916097
:10A4E000FFF79EFF23681D602023C4F888300020FA
:10A4F00084F8840038BD0220FCE738B590F8843039
:10A50000012B1DD00446012380F884302423C0F899
:10A51000883003681D681A6822F001021A60026818
:10A52000936823F0606319439160FFF779FF236814
:10A530001D602023C4F88830002084F8840038BDD2
:10A540000220FCE70A22002100F05AB9014B1868EA
:10A55000704700BF1400002470B50D4E0D4D761BE2
:10A56000B61006D0002455F8043B01349847A642A3
:10A57000F9D1094E094D761B06F03AF8B61006D00F
:10A58000002455F8043B01349847A642F9D170BD28
:10A590005C0A01085C0A0108640A01085C0A0108F7
:10A5A000830730B548D0541E002A3FD0CAB20346B4
:10A5B00001E0013C3AD303F8012B9D07F9D1032CAC
:10A5C0002DD9CDB245EA05250F2C45EA054536D9EA
:10A5D000A4F1100222F00F0C03F1200EE6444FEA22
:10A5E000121C03F1100242E9045542E902551032EF
:10A5F0007245F8D10CF1010214F00C0F03EB0212BA
:10A6000004F00F0C13D0ACF1040323F00303043364
:10A61000134442F8045B9342FBD10CF003042CB1C9
:10A62000CAB21C4403F8012B9C42FBD130BD6446E6
:10A630001346002CF4D1F9E703461446BFE71A4647
:10A64000A446E0E70FB400B5074983B004AB08683F
:10A6500053F8042B8168019300F0E8F803B05DF82B
:10A6600004EB04B0704700BF14000024024A1268D3
:10A6700001235C3200F002B814000024F0B4074655
:10A6800010B33E468C4616F8010B01E0A04216D0EE
:10A690001CF8014B002CF9D1D8B116F8015B0C461F
:10A6A00001E0002BF9D014F8013B9D42F9D14DB1E6
:10A6B000002306F8013C16603846F0BC70475BB1D9
:10A6C0003746DEE72E46F6E71768002FD9D1384621
:10A6D000F3E7F0BC10607047166038463B70ECE75B
:10A6E0002DE9F04F814645488E4675461EF801CB50
:10A6F00010F80C4014F00804F7D1BCF12D0FE3461C
:10A7000054D0BCF12B0F08BF9EF800B06FF000488A
:10A7100008BF05F1020E1BB1102B4FD01F4604E0FD
:10A72000BBF1300F55D00A231F460025B8FBF7F6C2
:10A73000284607FB168A07E0864215D329D007FB77
:10A7400000C001251EF801BBABF1300CBCF1090FB4
:10A7500006D9ABF1410CBCF1190F08D8ABF1370C9D
:10A7600063450DDD002DE7DA4FF0FF35EAE7ABF189
:10A77000610CBCF1190F03D8ABF1570C6345F1DC48
:10A78000002D0BDB04B140420AB195BB1160BDE85E
:10A79000F08FE245D3DA4FF0FF35D3E72223C9F833
:10A7A00000301AB30EF1FF314046EFE79EF800B0DB
:10A7B0004FF0004805F1020E0124ACE7BBF1300F69
:10A7C000ACD19EF8000000F0DF00582807D01F46EB
:10A7D000ABE79EF8003003F0DF03582B0BD11027B6
:10A7E0009EF801B03B460EF1020E9EE74046BDE8E2
:10A7F000F08F8046D6E708231F4696E7C10601087A
:10A80000012A09D0242A134606D8074A844610682C
:10A810000A466146FFF764BF10B5FFF797FE16239F
:10A820000360002010BD00BF140000242DE9F04F8C
:10A83000D5B01C46079191460546099003F0F4F8FF
:10A840000268179210460E94F6F7BAFB16901DB1E7
:10A85000AB6B002B00F02A82079A536EDD0740F1A4
:10A860003881B2F90C2091B28F0409D4079B42F4CD
:10A8700000529A8191B21A465B6E23F400535366DC
:10A880000E0740F1CB80079B1B69002B00F0C680B0
:10A8900001F01A030A2B00F0CF8000242BAB4D46A9
:10A8A000CDE92944CDE91944CDE91B4412942893FC
:10A8B0009846189400230B940024CDE914342B7887
:10A8C000002B00F09D81AA4604E01AF8013F002BFE
:10A8D00000F0C780252BF8D1BAEB050640F0C58003
:10A8E0009AF80030002B00F08B8100234FF0FF32EC
:10A8F0009AF801608DF883300A930AF1010A0892F0
:10A900001F462B244FF020090AF1010AA6F120036B
:10A910005A2B00F2ED80DFE813F0EB02EB00EB00C6
:10A92000E602EB00EB00EB006A00EB00EB005C02E0
:10A930008002EB0067028A02EB0085025B005B008D
:10A940005B005B005B005B005B005B005B00EB009F
:10A95000EB00EB00EB00EB00EB00EB007A01EB000F
:10A96000F801D2017A017A017A01EB00EB00EB00E9
:10A97000EB00E102EB00EB002D02EB00EB00EB0043
:10A980000202EB00A402EB00EB008307EB00EB00FC
:10A99000EB00EB00EB00EB00EB00EB007A01EB00CF
:10A9A000F801D4017A017A017A01C702D401CD01FC
:10A9B000EB00D402EB006C022F02B502CD01EB00DC
:10A9C00002027E008007EB00EB006107EB007E00D7
:10A9D000A6F1300300221AF8016B02EB820203EBAE
:10A9E0004202A6F13003092BF5D90A928EE7DDF871
:10A9F00024B0584603F018F843681B931846F6F73E
:10AA0000DFFA1C900646584603F00EF88368199347
:10AA1000002E40F0CD869AF8006075E7079D0998F2
:10AA2000294601F0ADFC002841F01C83A98901F002
:10AA30001A030A2B7FF431AF079AB2F90E30002BBC
:10AA4000FFF62BAF536ED80702D4890541F13B8145
:10AA50000799099823464A4655B0BDE8F04F01F0E2
:10AA60004FBCBAEB050600F0CB802A9B33442A93F7
:10AA7000299B0133072BC8E90056299305DC08F10F
:10AA800008080B9B33440B932AE70799099828AAD7
:10AA900003F0AAFF80B90DF1AC08F2E70799099815
:10AAA00028AA03F0A1FF002800F09B800D9B1BB19A
:10AAB0000998194602F08EFE079A536ED90740F1A5
:10AAC000EA8093895B0601F1D9820B9855B0BDE805
:10AAD000F08F079BB3F90C20900591B23FF5C4AEFF
:10AAE0001D46986D02F0A8FFB5F90C2091B2BBE6A7
:10AAF000002E00F0858000228DF8EC608DF8832018
:10AB00000123CDE90C32069308920F921392109212
:10AB10003BAD17F0020302D006990231069117F0FF
:10AB2000840B07D10A990698A1EB0009B9F1000F2F
:10AB300000F370832A9C8AB1299A0DF183010132B6
:10AB40000134C8F80010072A4FF001012A94299215
:10AB5000C8F8041000F3B68308F1080883B1299BF4
:10AB600021AA01330234C8F80020072B4FF002025B
:10AB70002A942993C8F8042000F3B28308F1080846
:10AB8000BBF1800F00F06982089B0C9AA3EB020BCB
:10AB9000BBF1000F00F3AA82FB0500F100820C9BC1
:10ABA000C8F804301C44299BC8F800500133072B17
:10ABB0002A94299300F3228308F10808780705D521
:10ABC0000A9B069A9D1A002D00F39683DDE90A235D
:10ABD00006998A42ACBF9B185B180B93002C7FF43C
:10ABE0005DAF002329930D9B1BB10D99099802F0CD
:10ABF000F1FD0DF1AC0855462B78002B7FF463AEC8
:10AC00002A9B002B41F0D3810023299354E70E9B0C
:10AC1000073323F00702F2E80234CDE91434DDE90A
:10AC2000143424F000440E92994618462146B54B40
:10AC30004FF0FF32F6F788FE002840F0EF84B14B6A
:10AC4000484621464FF0FF32F6F760FE002840F0FC
:10AC5000E584DDE9140100220023F6F74DFE00280B
:10AC600040F067879DF88320A74DA84B27F0800709
:10AC70000321472EC8BF1D4600230D9306910C915A
:10AC800008930F9313931093002A3FF442AF069B4F
:10AC9000013306933DE7079B9B899A053FF512AF69
:10ACA000079CA06D02F0CAFEA3890BE7099802F089
:10ACB00099FCD1E59AF8006047F0200724E647F0B8
:10ACC0001007BA060E9B40F13B84073323F00703BD
:10ACD0001A465B6852F8084B0E929946002BC0F258
:10ACE0004C84089B013300F0D88254EA090327F012
:10ACF000800B40F0D382089B002B40F0D4825F464B
:10AD0000002308930C9354AD1DE10E9B002253F8D1
:10AD1000041B8DF883208DF8EC100E93F0E60E9C4A
:10AD2000089B54F8045B4FF000098DF88390002DC8
:10AD300000F093855A1C00F051861A464946284671
:10AD4000F6F7EEF80D90002801F00E810D9BCDF87E
:10AD500020905B1B0C930E9423EAE3739DF88320F1
:10AD60000693CDF83490CDF83C90CDF84C90CDF8CA
:10AD7000409089E747F0100717F0200900F0D283D0
:10AD80000E9B073323F00703D3F8049053F8084BC6
:10AD90000E9327F4806B002300228DF88320089AFD
:10ADA000511C00F0B88054EA09012BF0800740F0F4
:10ADB000B180002A40F0F685002BA1D11BF00103E1
:10ADC0000C9300F0148430238DF84F310DF24F15A1
:10ADD000B9E00E9B53F8042B0A92002A80F2DA8322
:10ADE0000A9A0E9352420A929AF8006047F00407BA
:10ADF0008AE5BD0600F1D184FC0600F1D88578060D
:10AE000000F1A586B90540F1D2850E9B0B9953F848
:10AE1000042B0E9311705546EEE69AF800608DF8FB
:10AE2000834071E59AF8006047F080076CE5524670
:10AE300012F8016B2A2E01F03F82A6F13003092B94
:10AE4000924698BF002201F2BC801AF8016B02EB17
:10AE5000820203EB4202A6F13003092BF5D90892D6
:10AE600054E547F0100B1BF0200900F076830E9B91
:10AE7000073323F00703D3F8049053F8084B0E93DD
:10AE8000012389E70E9B53F8044B0E933023782659
:10AE90008DF884301E4B189347F0020B8DF88560B7
:10AEA0004FF00009022377E79AF80060682E03BF8D
:10AEB0009AF8016047F400770AF1010A47F0400769
:10AEC00022E59AF800606C2E03BF9AF8016047F003
:10AED00020070AF1010A47F0100715E59AF800600B
:10AEE00047F0080710E59AF8006047F001070BE506
:10AEF0009DF88330002B7FF48EAD9AF800608DF8BA
:10AF0000839001E5FFFFEF7F5C0601086006010802
:10AF10006C060108BB46012B00F0C081022B54AD2A
:10AF200020D1189A04F00F032409D35C05F8013DE1
:10AF300044EA09744FEA191954EA0903F2D154ABEF
:10AF40005B1B5F460C9308990C989DF88320814207
:10AF50004FF00003B8BF01460D9306910F93139372
:10AF6000109391E604F00703E40844EA49744FEAB9
:10AF7000D909303354EA09012A4605F8013DF1D1D7
:10AF80001BF0010FDBD0302BD9D03023023A05F86B
:10AF9000013C54AB9B1A5F460C931546D3E7652ED4
:10AFA00040F3E680DDE9140100220023F6F79AFC65
:10AFB000002800F0DC81299BBF4AC8F8002001333B
:10AFC00001340122072B2A942993C8F8042000F3A6
:10AFD000CC8408F10808229B129A934280F2D68210
:10AFE000169B179A1C44C8E90023299B2A94013315
:10AFF000072B299300F3248408F10808129B5D1E97
:10B00000002D7FF7DBAD102D299BDFF8B09240F3C8
:10B01000BD8449462246B946DDF824B0079C102677
:10B020000F4605E008F10808103D102D40F3AA84F2
:10B0300001331032072BC8E90076CDE92932F1DD62
:10B0400028AA2146584603F0CFFC00287FF42EADF5
:10B05000DDE929320DF1AC08E6E70A9B069AA3EB7D
:10B06000020BBBF1000F7FF78FADBBF1100F299AD8
:10B07000DFF848922CDD1D9621464E46079CDDF8F0
:10B080002490102306E0ABF1100BBBF1100F08F178
:10B0900008081ADD01321031072AC8E90063CDE93A
:10B0A0002921F0DD28AA214648460DF1AC0803F01D
:10B0B0009BFC00287FF4FAACABF1100BBBF1100F36
:10B0C000DDE929214FF01003E4DCB1461D9E0C465A
:10B0D00001325C44072ACDE92924C8F80090C8F859
:10B0E00004B000F3A08308F108084DE5BBF1100F90
:10B0F000299ADFF8C8912DDD41462046A8464C46E6
:10B10000079DDDF82490102306E0ABF1100BBBF196
:10B11000100F01F1080119DD01321030072AC1E9D1
:10B120000043CDE92920F0DD28AA2946484603F04E
:10B130005BFC00287FF4BAACABF1100BBBF1100F35
:10B14000DDE929202BA94FF01003E5DC4546A14697
:10B150008846044601325C44072ACDE92924C8F810
:10B160000090C8F804B000F3D08108F1080813E596
:10B17000129B012B40F38081299EC8F800500136B4
:10B1800001340123072E2A942996C8F8043000F3CD
:10B190007C8308F10808169B179A01361C44072E79
:10B1A000C8E90023CDE9296400F37C8308F108088D
:10B1B000DDE9140100220023F6F794FB002840F09B
:10B1C0007881129B0136013B01351C44072EC8F8DB
:10B1D00000502996C8F804302A9400F35D8108F1E4
:10B1E00008081A9BC8F8043001361C44072E24AB0B
:10B1F000CDE92964C8F800307FF7DEAC07990998DB
:10B2000028AA03F0F1FB00287FF450AC2A9C0DF132
:10B21000AC08D3E4B9F1100FDDE929212BDDCDE92C
:10B220001D3B1F96DDF824B04E461024A946079D0D
:10B2300004E0103E102E08F1080817DD0132204B03
:10B240001031072AC8E90034CDE92921F1DD28AA07
:10B25000294658460DF1AC0803F0C6FB00287FF4E0
:10B2600025AC103E102EDDE92921E7DCDDE91D3B90
:10B270004D46B1461F9EC8F80490013209EB010407
:10B28000072A0F49C8F80010CDE9292400F351839B
:10B290009DF8832008F108084DE4BB460A2C79F19B
:10B2A000000380F00C83303401238DF84F415F465A
:10B2B0000C930DF24F1546E69C060108B0060108F6
:10B2C000A0060108079909981D9328AA03F08CFB92
:10B2D00000287FF4EBAB2A9C1D9B0DF1AC083DE4EC
:10B2E0000799099828AA03F07FFB00287FF4DEABBA
:10B2F0002A9C0DF1AC0843E4102D299B21DD099F08
:10B30000DDF81C90102604E0103D102D08F108080F
:10B3100017DD0133BB4A1034072BC8E90026CDE9FD
:10B320002934F1DD28AA494638460DF1AC0803F06E
:10B330005BFB00287FF4BAAB103D102DDDE929340A
:10B34000E7DC0133AF4AC8F804502C44072BCDE9A1
:10B350002934C8F800207FF739AC0799099828AA42
:10B3600003F042FB00287FF4A1AB2A9C2EE4229933
:10B37000002940F31481DDF84090129B9945A8BF45
:10B380009946B9F1000F0BDD299B01334C44072B83
:10B39000C8E900592A94299300F39A8508F108080E
:10B3A000109EB9F1000FA8BFA6EB0906002E00F30E
:10B3B0004683DDF840B07905AB4400F1CE84229B92
:10B3C000129A934202DBFA0740F1B883169A179952
:10B3D0001444C8E90012299A2A940132072A2992B2
:10B3E00000F3838508F10808129AAE18A6EB0B0645
:10B3F000D51AAE42A8BF2E46002E0DDD299BC8F8F7
:10B4000000B001333444072BC8F804602A94299310
:10B4100000F3F18508F10808002EA8BFAD1B002D30
:10B420007FF7CCAB102D299BDFF8DC9140F3AE8287
:10B4300049462246B946DDF824B0079C10260F463F
:10B4400005E008F10808103D102D40F39B82013300
:10B450001032072BC8E90076CDE92932F1DD28AAA0
:10B460002146584603F0C0FA00287FF41FABDDE9FF
:10B4700029320DF1AC08E6E7FE073FF57DAE299EC7
:10B48000C8F80050013601340123072E2A9429966A
:10B49000C8F804307FF7A3AE0799099828AA03F0EB
:10B4A000A3FA00287FF402ABDDE929640DF1AC08B2
:10B4B00097E6129B5D1E002D7FF793AE102DDFF8EF
:10B4C000489140F37F8222460897099C079F4FF0DE
:10B4D000100B05E008F10808103D102D40F37082B4
:10B4E00001361032072EC8E9009BCDE92962F1DD53
:10B4F00028AA3946204603F077FA00287FF4D6AA16
:10B50000DDE929620DF1AC08E6E70799099828AA58
:10B5100003F06AFA00287FF4C9AA2A9C0DF1AC084E
:10B52000FFF73ABB17F0100372D117F0400200F09A
:10B53000BD820E9A52F8044B0E929946A4B228E4AA
:10B5400053F8044B0E93FB0656D47D0651D544F3B5
:10B55000C0394B4624B2FFF7C1BB1BF0100340F0CB
:10B5600036811BF0400200F092820E9A52F8044B92
:10B570000E929946A4B201230EE42D2364428DF865
:10B58000833069EB4909BB46012308E4F8077FF5DE
:10B5900015AB25E59AF800600E93FFF7B5B9299B26
:10B5A0001A4AC8F80020013301340122072B2A94DB
:10B5B0002993C8F8042000F3708408F108080029D2
:10B5C00040F01E82129A07F0010313433FF4F6AADB
:10B5D000169B1799E218C8E90013299B2A92013398
:10B5E000072B299300F3618308F1080819E254AD91
:10B5F000A9E4B80500F1B4824FEAE4794B46FFF7BD
:10B600006DBB00BFA0060108B00601089C0601083A
:10B610000E9B53F8044B0E93FFF7BBBBDDE91401FF
:10B6200002460B46F6F790F9002840F0A085612EFF
:10B6300000F05085412E00F09982089B013326F0DE
:10B640002003069300F08F85472B00F07985DDE914
:10B65000141247F480730F931346002BC0F2ED854C
:10B660000C9300231D938B460D93069B462B00F0F5
:10B670004A84452B00F04F850899019126A9049131
:10B6800023A9039122A9029102210C9B0998009100
:10B690005A4600F081FF069B472B054640F01C866A
:10B6A00017F0010FB9460F9F40F0D984269B5B1B12
:10B6B0001293069B472B00F01883069B462B00F045
:10B6C0005F84229B1093109B069A013B412A229390
:10B6D00000F0AA85F2B20021002BB8BF109B8DF8B4
:10B6E0009020BABFC3F101032D222B22092B8DF824
:10B6F000912040F363850DF19F04BD4F2246104613
:10B7000087FB0321DA17C2EBA10202EB8201A3EB54
:10B710004101303100F8011C19466329134600F13C
:10B72000FF32ECDC3033D9B2831E9C4202F8011C9C
:10B7300040F2CE8513460DF1920201E013F8011B91
:10B7400002F8011B9C42F9D10DF1A1030DF1920207
:10B750001B1A134424AA9B1A1A93129B1A9A012BA0
:10B760001A440C9240F372850C9B169A13440C9366
:10B770000C9A002329F4806722EAE27247F480776A
:10B780000F930692139310931D9B002B40F0DE82C3
:10B790009DF883200893FFF777BA0E9B0B9853F818
:10B7A000041B0E93C217C1E900025546FFF724BAE5
:10B7B000199B002B3FF42FA9199B1B78002B3FF4FA
:10B7C0002AA99AF8006047F48067FFF79DB80E9B9E
:10B7D00053F8044B0E930123FFF7DEBA854B189301
:10B7E00017F0200949D00E9B073323F00703D3F845
:10B7F000049053F8084B0E93F80709D554EA09034F
:10B8000006D030238DF8856047F002078DF884302C
:10B8100027F4806B0223FFF7BFBABB46FFF723BBB9
:10B82000754B1893DCE70799099828AA03F0DCF810
:10B8300000287FF43BA92A9C0DF1AC08FFF7A4B9BE
:10B840000799099828AA03F0CFF800287FF42EA9B9
:10B850002A9C0DF1AC08FFF7D1BB062B294628BF67
:10B86000062308950D952A460693644D0E940C9375
:10B870000F9113911091FFF707BA17F0100369D0D9
:10B880000E9B53F8044B0E93B6E70799099828AA24
:10B8900003F0AAF800287FF409A9DDE929640DF175
:10B8A000AC0878E40799099828AA03F09DF80028C5
:10B8B0007FF4FCA8DDE929640DF1AC0878E40BF411
:10B8C00080630022CDE90CA80696DDF8648054AFB1
:10B8D00016469A460CE00023204649460A22F4F711
:10B8E0008DFF0A2C79F100031BD3044689462F46AD
:10B8F00020460A2200234946F4F780FF30327D1E9D
:10B90000013607F8012CBAF1000FE4D098F80030A6
:10B910009E42E0D1FF2EDED00A2C79F1000380F0A8
:10B92000F480CDF864801296DDE90CA8069EFFF73E
:10B9300006BB079909981D9328AA03F055F800281B
:10B940007FF4B4A89DF883202A9C1D9B0DF1AC08C0
:10B95000FFF7F1B817F0400200F0B6800E9A52F8E7
:10B96000044B0E929946A4B246E70799099828AA73
:10B9700003F03AF800287FF499A82A9C0DF1AC084E
:10B98000FFF729BB14463A464F46914601332C44F3
:10B99000072BC8F80090C8F80450CDE929347FF788
:10B9A0000BA92BE4012BBB467FF4B8AA7BE40E9BCA
:10B9B0000B9953F8042B554611600E93FFF71CB9F1
:10B9C000089F144601362C44072ECDE92964C8F897
:10B9D0000090C8F804507FF702AC5DE52846CDF82A
:10B9E00020900E94F5F7ECFA03460C90FFF7B4B9EB
:10B9F000676666666C060108800601089406010801
:10BA0000169B1798E218C8E90003299B2A92013374
:10BA1000072B299300F3498108F108080029C0F297
:10BA2000FA821299C8F8005001338C18072BCDE91F
:10BA30002934C8F804107FF7BFA8FFF7DFBB102E2A
:10BA4000299BDFF8C09252DD484642462146A8466F
:10BA5000B946099C079D4FF0100B074603E00832DA
:10BA6000103E102E3DDD01331031072BC2E9007B63
:10BA7000CDE92931F3DD28AA2946204602F0B4FF9A
:10BA800000287FF413A8DDE929312BAAE8E70E9BF3
:10BA90001BF4007914BF53F8044B53F8044B0E9376
:10BAA0001CBF9146E4B20123FFF776B90E9B17F451
:10BAB000007914BF53F8044B53F8044B0E931CBF8A
:10BAC0009146E4B2FFF765B90E9B17F4007914BFF5
:10BAD00053F8044B53F8044B0E931CBF9146E4B249
:10BAE0008AE6454690463A460C464F469146013313
:10BAF0003444072BCDE92934C8F80090C8F8046015
:10BB000000F3E68008F1080853E41C9B1B99ED1A2A
:10BB10001A46284602F0FAFE98F801300BB108F1F7
:10BB20000108204649460A2200230026F4F766FE53
:10BB3000DBE62D228DF88320FFF796B8129AAE1817
:10BB4000A6EB0B06D51AAE42A8BF2E4664E40E9BA8
:10BB50000B9953F8042B0E9311805546FFF74CB800
:10BB600044F3C0194B4664B2FFF7B8B830238DF8E0
:10BB7000843058238DF88530089B632B47F00204EE
:10BB800000F39B8200230D933BADDDE9141247F4D3
:10BB900081730F931346002B2746C0F220820C932B
:10BBA00026F02003069300238B461D93612E00F0A0
:10BBB000ED82412E7FF459AD22AA0C99584602F02D
:10BBC00015FE00224FF07F53F5F724FC02460B468A
:10BBD000CDE9102300220023F5F784FE08B10123EC
:10BBE0002293494B0C93089BCDE912A6CDE91E7810
:10BBF000DDF830A0DDE9106703F1FF39AB461095A1
:10BC000006E00022002309F1FF39F5F76BFEE8B9E1
:10BC10003E4B002230463946F5F7FCFB0F46064600
:10BC2000F5F7A8FE0446F5F78BFB0B4602463946AE
:10BC30003046F5F737FA1AF80430B9F1FF3FD84625
:10BC40004D460BF8013B06460F46DAD130463946E1
:10BC50002F4BDDF848A0139ECDF848800022A9465E
:10BC6000DDF87C80109D1E9FCDE91001F5F762FE86
:10BC7000002840F03482DDE91001254B0022F5F761
:10BC800031FE10B1E10700F12A824B46002B06DBA2
:10BC900001335B4430220BF8012B5B45FBD1ABEB4E
:10BCA0000503B94612930F9F03E50799099828AA3F
:10BCB00002F09AFE00287EF4F9AEDDE929322299DD
:10BCC0000DF1AC08AAE6906D01F0B8FEFEF7C0BE1B
:10BCD0000799099828AA02F087FE00287EF4E6AEAC
:10BCE0002A9C0DF1AC08FFF764BB229B1093DA1C71
:10BCF00002DB089A93420DDD023E26F020030693F4
:10BD0000E1E400BFB00601088006010800003040F1
:10BD10000000E03F109B129A9342C0F2568119F046
:10BD2000010F00F08782169A13440C9319F4806F68
:10BD300003D0109B002B00F350820C9B23EAE3738B
:10BD40000693672600230F9313931DE52D220023EE
:10BD50008DF883200893FEF79ABF129BCDF830A090
:10BD60004246DDF84C801097EB1808935E46199F09
:10BD7000DDF87090DDF824A0DDF81CB00F9B139562
:10BD80002146B8F1000F2ED0002B6BD1013F08F1F6
:10BD9000FF381B9BC2E90039299B01334944072B1B
:10BDA0002A91299362DC0832089B38789B1B8342D6
:10BDB000A8BF0346002B1C460ADD29980130194410
:10BDC0000728C2E900632A9129905ADC38780832A2
:10BDD000002CACBF051B0546002D15DC06440F9B4F
:10BDE000B8F1000FD0D1002B3CD1DDE91235EB18B2
:10BDF0009E421997B346DDF830A0109F90460C463E
:10BE000028BF9B46FFF7DBBA102D29981DDD1024B3
:10BE100004E0103D102D02F1080216DD0130AC4B9C
:10BE200010310728C2E90034CDE92901F1DD28AA43
:10BE30005946504602F0D8FD00287EF437AE103D3A
:10BE4000102DDDE929012BAAE8DC0130A04B55605B
:10BE500029440728CDE9290113602CDC3878083201
:10BE60000644BCE70F9B013B0F9392E728AA594673
:10BE7000504602F0B9FD00287EF418AE2A992BAA8C
:10BE800092E728AA5946504602F0AEFD00287EF4FB
:10BE90000DAE38782A992BAA9AE70799099828AA0B
:10BEA00002F0A2FD00287EF401AE22992A9C0DF139
:10BEB000AC08FFF784BB28AA5946504602F094FD0F
:10BEC00000287EF4F3AD38782A992BAA064486E739
:10BED0000799099828AA02F087FD00287EF4E6ADAC
:10BEE0002A9C0DF1AC08FFF75BBA0799099828AABC
:10BEF00002F07AFD00287EF4D9AD229B2A9C0DF138
:10BF0000AC08FFF771BA0899019126A9049123A9F9
:10BF1000039122A9029103210C9B099800915A4692
:10BF200000F03AFB0378302B054600F09581229B08
:10BF3000089AB94613440F9FEC180C9958460022F2
:10BF40000023F5F7CFFC10B12346FFF7B0BB269BCB
:10BF5000A342BFF4ACAB30215A1C26921970269B29
:10BF60009C42F9D8FFF7A3BB089B9DF883200E9451
:10BF700006930C9308900F9013901090FEF784BED8
:10BF8000229A1092002A40F38181089909F0010356
:10BF90000B4340F05581109B0C93662619F4806F7B
:10BFA00040F01C810C9B23EAE3730693CAE60799D1
:10BFB000099828AA02F018FD00283EF425AEFEF7E5
:10BFC0007BBD00230893FEF7A1BC129B169A9A181A
:10BFD000109B0C92002B40F34D816726DEE726F084
:10BFE00020030693DDE914349B4604F100430C93CF
:10BFF0002D231D93DAE50799099828AA02F0F4FC8D
:10C0000000287EF453AD229D129B2A9C5D1B0DF1EE
:10C01000AC08FFF701BA4E421031DFF8B49034DAC1
:10C020004146DDF824B0A8461024079D03E00831FE
:10C03000103E102E27DD01331032072BC1E900948A
:10C04000CDE92932F3DD28AA2946584602F0CCFC76
:10C0500000287EF42BADDDE929322BA9E8E7089B07
:10C06000EC186AE7079B5B6EDD0707D4079B9B898B
:10C070009C0503D4079B986D01F0E0FC4FF0FF3363
:10C080000B93FEF722BD4546884601333244072B09
:10C09000CDE92932C8F80090C8F804607FF7A4AA57
:10C0A0000799099828AA02F09FFC00287EF4FEACAC
:10C0B000DDE929320DF1AC08B3E40998591C01F00F
:10C0C0002FFD0546002800F00D810D905DE500BFB5
:10C0D000B006010830238DF8843078234AE5129B9E
:10C0E00026930C9B1BF8012CD97B8A425B4609D115
:10C0F000302003F8010C269B5A1E269213F8012CBF
:10C100009142F6D0392A0BBF0C9A0132927AD2B200
:10C1100003F8012CC3E508990C9B09984C1C26A92F
:10C12000049123A9039122A9029102215A46019464
:10C13000009100F031FA0546B9462C440F9FFCE609
:10C14000089B002B08BF0123089347F480730F93CB
:10C15000159B002BC0F2AE80DDF850B01D900C9303
:10C160000D90FFF789BA06230893FFF770BA159B65
:10C17000604D002BB4BF2D229DF883205E4BB8BFCD
:10C180008DF8832027F08007FEF772BD22AA0C9954
:10C19000584602F02BFB00224FF07F53F5F73AF997
:10C1A00002460B46CDE9102300220023F5F79AFB47
:10C1B00008B101232293514B0C9314E5002962D15D
:10C1C00030228DF892200DF19302303302F8013BBA
:10C1D00024ABD31A1A93FFF7C0BA672619990B78C4
:10C1E000FF2B7BD00024109A204603E00130013160
:10C1F000FF2B08D0934206DAD21A4B78002BF5D1E8
:10C200000B780134F4E71991109213900F940F9A60
:10C21000139B1C9913440C9A01FB03230C9323EAF0
:10C22000E3730693FFF7B0BA06F10F02D2B2012111
:10C23000FFF752BA109B0C9378E500230D93D1E6DB
:10C24000169BD31819440C916626A7E619F0010F26
:10C250003FF48EAAFFF788BA0C99584600220023B3
:10C26000F5F740FB00287FF462AE089BC3F10103A1
:10C2700022935DE6C3F101031A4422EAE2730C92B1
:10C28000069367265EE50DF192029EE7089A09F093
:10C29000010959EA020304D10123069366260C938F
:10C2A00050E5169B01331A4422EAE2730C9206937E
:10C2B000662647E50D9095E60E9B9AF8016092463A
:10C2C00053F8042B0E9342EAE2720892FEF71CBB6D
:10C2D00002231A93FFF741BA089C2DE700230F931E
:10C2E000139394E7079A938943F040039381FEF7F1
:10C2F000E3BB00BF64060108680601086C0601087C
:10C30000F0B51F468B89ADF26C4D23F00203ADF8FA
:10C310000C304B6E1993CB89ADF80E30CB69079377
:10C320004B6A09931AAB009304934FF4806315464C
:10C3300006460293059316A800230C46069301F0C7
:10C3400077FB2A463B4669463046FEF76FFA051EE4
:10C3500007DB6946304601F011F9002818BF4FF09D
:10C36000FF35BDF80C305B0603D5A38943F04003CD
:10C37000A381169801F05EFB28460DF26C4DF0BDCE
:10C3800038B5334B1B6805460C460BB19A6B12B39C
:10C39000B4F90C3018079AB225D5216900292DD09F
:10C3A00012F0010007D00020A06060694042A06147
:10C3B00039B1002038BD950758BF6069A0600029D9
:10C3C000F7D1120658BF0846F4D543F04003A381C5
:10C3D0004FF0FF3038BD184601F004F9B4F90C30C5
:10C3E00018079AB2D9D4D1062AD5520714D4216994
:10C3F00043F00803A3819AB20029D1D102F420703E
:10C40000B0F5007FCCD02146284601F019FBB4F9E5
:10C410000C3021699AB2C3E7216B51B104F140029B
:10C42000914204D0284601F0D5F9B4F90C3000222D
:10C43000226321690022C4E9001223F02403D7E714
:10C44000092243F040032A604FF0FF30A38138BD3A
:10C4500014000024024B13B1024800F005B87047E5
:10C460000000000009D70008002301461A461846BC
:10C4700003F0EAB92DE9F04F03690C69A34283B0D8
:10C48000C0F28680013C01F11405A30000F11408FC
:10C49000009355F8243058F8242001338A469A42F4
:10C4A00008EB8401814605EB84070191B2FBF3F6AA
:10C4B00038D30023AE4640469B465EF8041B026814
:10C4C0001FFA81FC06FB0C33090C4FEA134C06FBE8
:10C4D00001CC99B2ABEB01011FFA8CF311FA82F196
:10C4E000C3EB124202EB214289B241EA0241774595
:10C4F00040F8041B4FEA1C434FEA224BDDD2009B5D
:10C5000058F8033073B9019B043B984504D307E006
:10C51000984504F1FF3403D253F80429002AF7D0D8
:10C52000C9F810405146484602F038F800282BDB85
:10C5300001364046002355F8041BD0F800C08AB2EB
:10C540009A1A0B0C12FA8CF2C3EB1C4303EB224336
:10C5500092B242EA0342AF4240F8042B4FEA23432F
:10C56000E9D258F8242008EB84036AB9043B9845C3
:10C5700004D307E0984504F1FF3403D253F80429AB
:10C58000002AF7D0C9F81040304603B0BDE8F08F5C
:10C59000002003B0BDE8F08F2DE9F04F016C99B099
:10C5A00090469946CDE90489259D044641B1426CE7
:10C5B0004A60012393408B6001F094FD00232364C3
:10C5C000B9F1000AB4BF012300232B60764BBCBF36
:10C5D0002AF0004ACDF814A033EA0A0300F0AA803A
:10C5E000DDE904231046194600220023CDE90A01A3
:10C5F000F5F778F9074670B1249A01231360269B5A
:10C60000002B00F0E48269481860431E03930398EE
:10C6100019B0BDE8F08F16AB019317AB009320461D
:10C62000DDE90A2302F080F85FEA1A56054640F079
:10C630009780DDE916763E4406F23240202840F32A
:10C64000B583C0F140000AFA00FA06F2124028FA57
:10C6500000F04AEA0000F4F763FE0123013EA1F175
:10C66000F8710F93524B0022F4F71CFD48A3D3E955
:10C670000023F4F7CFFE48A3D3E90023F4F714FD19
:10C68000804630468946F4F75BFE45A3D3E9002394
:10C69000F4F7C0FE02460B4640464946F4F704FD57
:10C6A00080468946F5F766F9002283460023404616
:10C6B0004946F5F721F9002840F07C82BBF1160FBE
:10C6C00000F26B823B4B03EBCB03D3E90023DDE9A4
:10C6D0000A01F5F711F9002872D00023BE1B0E9352
:10C6E000731E0BF1FF3B069300F15E82002309935A
:10C6F000BBF1000F6BDA099BCDF81CB0A3EB0B0369
:10C700000993CBF100030D93229B092B4FF0000BF3
:10C7100066D8052B40F34883043B22930026229BD6
:10C72000023B032B00F26886DFE813F05C04590437
:10C7300050043304249A42F20F73CAF3130A1360AD
:10C740005AEA08031AD1269B002B00F064861A4B84
:10C7500003930833269A0398136019B0BDE8F08F4D
:10C76000DDE90A12C2F31303084643F07F510F9725
:10C77000A6F2FF36169F41F4401173E7269B002B6B
:10C7800040F0EA830D4B039341E700BFAFF3008015
:10C7900061436F63A787D23FB3C8608B288AC63FC7
:10C7A000FB799F501344D33F0000F07F9D060108A2
:10C7B0000000F83F10090108C8070108C407010874
:10C7C000BE1B731E069300F185840E900990069B94
:10C7D0005B44CDE9063B00230D93229B092B98D99E
:10C7E0000023CDE9223301264FF0FF330C96089346
:10C7F000089B129300216164204601F04DFC0390D8
:10C80000002800F00186039B2364089B0E2B00F296
:10C810001381002E00F010810799002940F35C84F9
:10C82000AE4B01F00F0203EBC2034FEA2118C9051A
:10C83000D3E9006740F11484A94BDDE90A01D3E98B
:10C840000823F4F711FFCDE9100108F00F084FF0AD
:10C85000030AB8F1000F13D0DFF8849218F0010F2B
:10C8600009D030463946D9E90023F4F7D3FD0AF15F
:10C87000010A06460F465FEA680809F10809EDD18A
:10C88000DDE9100132463B46F4F7EEFE804689466C
:10C890000E9B43B1934B002240464946F5F72CF8D6
:10C8A000002840F030855046F4F74AFD42464B469A
:10C8B000F4F7B0FD8C4B0022F4F7F6FBA1F15073B6
:10C8C000CDE910011193089B002B00F09780079B86
:10C8D0001493089B13930C9B002B00F0A584139AD0
:10C8E0007E4B8249039E03EBC20353E902230020DF
:10C8F000F4F7BAFEDDE91023F4F7D4FBCDE910011B
:10C9000049464046F5F736F80746F4F719FD024662
:10C910000B4640464946F4F7C5FB3037DDE91023A6
:10C9200006F8017B80468946F4F7E6FF002840F0D0
:10C930002985CDF854B00027DDE910AB1095139D83
:10C9400013942AE00137AF4280F22C85684B5046A1
:10C9500059460022F4F75EFD654B002282468B4665
:10C9600040464946F4F756FD89468046F5F702F8F9
:10C970000446F4F7E5FC02460B4640464946F4F708
:10C9800091FB303406F8014B52465B46804689469F
:10C99000F4F7B2FF002840F0F38442464B46514979
:10C9A0000020F4F77FFB52465B46F4F7A5FF002812
:10C9B000C8D0DDE91343109D039A079302E0964225
:10C9C00000F0C884B24616F8013D392BF7D0013388
:10C9D000DBB23370079B01330793C8E15046F4F78D
:10C9E000AFFC42464B46F4F715FD3F4B0022F4F7EF
:10C9F0005BFBA1F15073CDE9100111933D4B404613
:10CA000049460022F4F74EFBDDE910894B464246C9
:10CA100006460F46F4F78EFF8146002840F0AA84B0
:10CA2000DDE91001024601F1004330463946F4F7D2
:10CA300063FF002840F04583179B002BC0F28C80D9
:10CA4000079A0E2A00F38880244B03EBC203D3E934
:10CA500000AB239B002B1BDA089B002B18DC40F05B
:10CA60002E83244B002250465946F4F7D3FC02464D
:10CA70000B46DDE90A01F4F749FFDDF820904E4648
:10CA8000002800F0C782239BDDF80C80DF43C9E259
:10CA9000DDE90A7852465B4638464146F4F7E4FD44
:10CAA000F4F768FF81460990F4F74AFC52465B466A
:10CAB000F4F7B0FC039E0B46024641463846F4F7B5
:10CAC000F1FA09F1300306F8013B089B012B00F055
:10CAD0005C830694012704951C462AE0100901088E
:10CAE000E80801080000F03F00001C400000E03FA3
:10CAF000000024400000144052465B464046494630
:10CB0000F4F7B2FDF4F736FF0546F4F719FC524688
:10CB10005B46F4F77FFC01370B4602464946404628
:10CB2000F4F7C0FA05F13003A74206F8013B00F024
:10CB30002983AC4B0022F4F76DFC002200238046D1
:10CB40008946F4F7CFFE0028D6D0049D069C079BAB
:10CB500001330793B2460AE10C9A002A3DD0229A8B
:10CB6000012A40F39C82089B03F1FF380D9B43454B
:10CB7000C0F26D82A3EB0808089B002BC0F23C8337
:10CB8000069A1A440692099A17461A4409920121F4
:10CB9000204601F04FFB064623E00123BE1B0E9307
:10CBA000731E06937FF5A2ADC6F10103099300231E
:10CBB00006939DE55846F4F7C3FB42464B46F4F70F
:10CBC00091FE00287FF47AAD0BF1FF3B76E5864BB2
:10CBD0000393039819B0BDE8F08FDDF83480099F06
:10CBE0000C9E002F0CDD069900290B4608DD099AE2
:10CBF000B942A8BF3B46D21AFF1ACB1A0992069334
:10CC00000D9BDBB10C9B002B00F05D82B8F1000F97
:10CC10000FDD31464246204601F0E8FB2A46014638
:10CC20000646204601F034FB29460546204601F021
:10CC300059FA0D9BB3EB080240F0D882012120463F
:10CC400001F0F8FABBF1000F814600F3B480229B9B
:10CC5000012B40F386814FF0000A0120BBF1000F49
:10CC600040F0B580069A104410F01F0000F0938049
:10CC7000C0F12003042B40F3D283099BC0F11C00B8
:10CC800003440244099307440692099B002B05DDE7
:10CC900029461A46204601F009FC0546069B002B52
:10CCA00005DD49461A46204601F000FC81460E9BF0
:10CCB000002B40F03681089B002B40F31D810C9B1C
:10CCC000002B40F0A080079B01330793DDF80C8018
:10CCD000DDF820A0012707E0294600230A2220468C
:10CCE00001F00AFA0137054649462846FFF7C2FB1C
:10CCF000574500F1300308F8013BEDDB089A002AA4
:10CD0000C8BF9346039AD8BF4FF0010B9344002746
:10CD1000294601222046049301F0C8FB49460546F6
:10CD200001F03CFC002840F3A8811BF8013C039A69
:10CD30000BF1FF3B04E05A4500F0AA811BF8013DCE
:10CD4000392B0BF1010AF6D001338BF8003049463C
:10CD5000204601F0C7F956B12FB1B74203D039468A
:10CD6000204601F0BFF93146204601F0BBF92946C3
:10CD7000204601F0B7F900238AF80030249B079A77
:10CD80001A60269B002B3FF442AC0398C3F800A026
:10CD900019B0BDE8F08F1C20099B03440993069B42
:10CDA00003440744069370E70126B8E4C0F120006D
:10CDB00008FA00F04FE401465A46204601F016FBFF
:10CDC000229B012B814640F3B3814FF0000AD9F832
:10CDD000103009EB8303186901F0DEF9C0F120007F
:10CDE00040E700BF000024409C06010831460023B4
:10CDF0000A22204601F080F9129B002B064640F3E0
:10CE0000E782CDE90783002F00F31A81BAF1000F02
:10CE100040F0D581B046049B039F089903F00102BE
:10CE20007B1E1944229B0C92134309910A93494695
:10CE30002846FFF71FFB31468346284601F0AEFB2C
:10CE4000424649468246204601F0C8FBC268014678
:10CE50000BF13003002A42D106902846089301F0D6
:10CE60009DFB06990490204601F03CF9049A089B2A
:10CE70001AB90A99002900F09B82BAF1000FC0F29A
:10CE8000638122994AEA010A0C9951EA0A0100F0E9
:10CE90005B81002A00F3B481099A3B7007F1010A13
:10CEA0009742D34600F0B281294600230A22204649
:10CEB00001F022F94645054631464FF000034FF098
:10CEC0000A02204612D001F017F941460646002317
:10CED0000A22204601F010F957468046A7E720466F
:10CEE000049301F0FFF8049B0122C6E701F004F966
:10CEF0005746064680469AE7229B022B79DC0C9B1C
:10CF0000002B80D1079B4946013328460793FFF742
:10CF1000B1FADDF80CB000F130030BF8013B00274B
:10CF2000F6E64946284601F039FB0028BFF6C3AEB5
:10CF3000294600230A22204601F0DEF8079B03F170
:10CF4000FF380C9B0546002B7FF450AF129B002B43
:10CF500040F335820893B9E6AF4B03930333FFF7F1
:10CF6000F9BBDDE9041200297FF475AEC2F31303A7
:10CF7000002B7FF470AEA94B1340002B00F0FE8114
:10CF8000099B01330993069B013306934FF0010A75
:10CF900063E601230C93239B079A134412930133F6
:10CFA000012B1F460893B8BF01270021172F61648A
:10CFB0007FF722AC012204235B0003F11400B84286
:10CFC000114602F10102F7D9616415E401230C93C3
:10CFD000239B002B4CDD129308931F46E5E70023AB
:10CFE0000C93D8E700230C93F2E7129BCDF81C803A
:10CFF0000893089B002B7FF446AD49460522204646
:10D0000001F07AF801468146284601F0C7FA002867
:10D010007FF739AD0398079F3123804600F8013B25
:10D02000013703904946204601F05CF87B1CDDF88F
:10D030000CA00793CDF80C80002E7FF494AE96E6FA
:10D0400031463A46204601F031FA0646DEE60D9BAF
:10D05000CDF83480A8EB03039B444FF000088BE528
:10D06000DDE90A234FF0020ACDE91023FFF7F1BBF7
:10D07000012323930893FFF7BBBB03D1049BDB077A
:10D080003FF553AEDA461BF8013D302BFAD05EE691
:10D09000079B039A013307933123137057E60F9AC6
:10D0A000002A00F0268103F23343069ADDF834802B
:10D0B0001A440692099A17461A44099267E54FF0F6
:10D0C00000094E46DFE429460D9A204601F08EF90C
:10D0D0000546B3E50E9067E500F00F81079A504BC7
:10D0E000564206F00F0203EBC203D3E90023DDE949
:10D0F0000A01F4F78FF936118046894600F07181F4
:10D10000484F00234FF0020AF20706D5D7E9002363
:10D11000F4F780F90AF1010A0123761007F10807F4
:10D12000F2D1002B3FF4B4AB80468946FFF7B0BB89
:10D13000049B002B7FF449AEDDE90412C2F3130314
:10D14000002B3FF418AF40E6002A12DD29460122E9
:10D150002046049301F0AAF94946054601F01EFA5B
:10D160000028049B40F31881392B00F0F9800BF163
:10D170003103BA460AF8013B079B01333746079350
:10D180004646E4E50995069C049D02460B46F3F7E6
:10D190008BFF52465B4680468946F4F7CBFB60B96D
:10D1A00052465B4640464946F4F79CFB00283FF454
:10D1B000CEAC099BD9077FF5CAAC039A02E471682B
:10D1C000204600F069FF0746002800F00E81336911
:10D1D00002339A0006F10C010C30F3F791FC39464A
:10D1E0000122204601F062F9804614E629462046D5
:10D1F00001F0FCF8054621E5DDE908239F1AC6E4A5
:10D20000392B00F0AD80BA460133B3E7079A0132FB
:10D210003746079246467BE5C40701080000F07FC9
:10D2200010090108E8080108DDF84CA0844901EB69
:10D23000CA01DDE9102351E90201F4F7EBF8CDE969
:10D24000100149464046F4F795FB0646F4F778F896
:10D250000B46024649464046F3F724FF039F5346D8
:10D260003036012B07F8016B8046894600F0AE800E
:10D27000139E039B1E44734B002240464946F4F71D
:10D28000C9F889468046F4F775FB8246F4F758F8EA
:10D290000AF1300A02460B4640464946F3F702FFC0
:10D2A00007F801ABB74280468946E4D1664B0022BD
:10D2B000DDE91001F3F7F8FE42464B46F4F71CFB9C
:10D2C000002864D1DDE910235F490020F3F7EAFE6E
:10D2D00042464B46F4F72EFB00283FF4ADABB24676
:10D2E000013E1AF8013C302BF9D0149B013307930F
:10D2F0003DE5169BC3F13603D7E6DDE90A894FF019
:10D30000020AFFF7C5BA089B002B3FF467AB129BDC
:10D31000002B7FF791AB079A013ACDE913324046D3
:10D32000484B00224946F4F775F8804689460AF1D1
:10D330000100F4F705F842464B46F4F76BF8434B0F
:10D340000022F3F7B1FEA1F15073CDE91001119362
:10D35000FFF7C1BA079B013307933123FFF739BBAE
:10D36000079BBB4601330793392337460BF8013B34
:10D370004646DCE44FF000094E464BE69A466CE424
:10D38000109D139C149B01330793B246EFE4149B4A
:10D39000039A0793FFF716BB7FF4EBAEDA077FF52E
:10D3A000E8AEE1E6DDF854B0109D139CFFF744BBF6
:10D3B000392BD5D0BAF1000F3FF7D9AED9E6229B71
:10D3C000022B3FF712AECDF81C809BE53E466DE781
:10D3D000229B022B3FF709AE129BCDF81C800893CD
:10D3E00011E54FF0020AFFF753BA194B19483A46B4
:10D3F00040F2EA2102F06EFA0026666431462046C9
:10D4000000F04AFE039078B9114B124800224FF405
:10D41000D57102F05FFA104B0393FFF7F8B83FF4B1
:10D4200034ACC0F13C00B7E4039B236401224FF00D
:10D43000FF33239612930C920893FFF7FDBA00BFB7
:10D4400010090108000024400000E03F00001C40DB
:10D45000D4070108E8070108C8070108B1F90C2042
:10D46000F8B50C461107074642D4636842F40062DF
:10D47000002BA28159DDA56A002D54D000233E68FF
:10D480003B6093B212F4805253D1E16901233846D4
:10D49000A847421C63D0A389A56A5B0705D56368CA
:10D4A000C01A236B0BB1E36BC01AE169024600237B
:10D4B0003846A847411C3ED13B68002B3BD01D2B72
:10D4C00001D0162B52D1A3892269226023F4006374
:10D4D00000216160A381216B3E6021B304F1400310
:10D4E000994202D0384600F075F900202063F8BD5B
:10D4F0002669C6B193B2256826609A070CBF636996
:10D500000023AD1BA3600CE0D4F824C0E1692B46D6
:10D5100032463846E047B0F1000CA5EB0C056644F6
:10D5200016DD002DF0DC0020F8BDE36B002BA2DC43
:10D53000F9E7206DB1E7B4F90C302269226023F4D9
:10D540000063A3810022DB046260C4D52065C2E7CA
:10D55000A38943F040034FF0FF30A381F8BD3B683F
:10D56000002B98D01D2B06D0162B04D0A38943F096
:10D570004003A381F8BD3E60D5E700BF38B50C4637
:10D58000054608B1836BA3B1B4F90C00B8B1636E62
:10D59000DB0701D4810515D528462146FFF75EFF3C
:10D5A000636EDA07054602D4A3899B050ED528468B
:10D5B00038BD00F017F8B4F90C000028E7D1054693
:10D5C000284638BDA06D00F037FAE5E7A06D00F001
:10D5D00035FA284638BD00BF014900F001BA00BF46
:10D5E000B1F900082DE9F0478246394800F024FAE5
:10D5F000DAF83840002C66D1DAF80450354ACAF817
:10D600003C200323CAE9B843DFF8CC90DFF8CC8094
:10D61000334F344E04230AF53B72CAF8E822214600
:10D62000C5E90243C5E90044C5E904446C66082223
:10D63000AC6105F15C00FCF7B3FFC5E90759C5E92A
:10D640000987EE6205F1580000F0F2F9DAF80850A7
:10D65000254BEB602146C5E90044C5E904446C66EE
:10D66000AC60AC61082205F15C00FCF799FFC5E9EC
:10D670000759C5E90987EE6205F1580000F0D8F9AD
:10D68000DAF80C50194BEB602146C5E90044C5E9B6
:10D6900004446C66AC60AC61082205F15C00FCF7E8
:10D6A0007FFF05F15800C5E90759C5E90A76C5F8B5
:10D6B000248000F0BDF90123CAF838300448BDE8E1
:10D6C000F04700F0BBB9BDE8F047014800F0B6B93B
:10D6D000E0290024D9D5000881E80008A5E8000861
:10D6E000E5E8000805E90008090001001200020051
:10D6F000014800F0A1B900BFDC290024014800F076
:10D700009DB900BFDC29002438B5084B084D5B1BD0
:10D710009C1007D0043B1D44013C55F80439984740
:10D72000002CF9D1BDE8384002F068BF680A010852
:10D73000640A0108F8B5244F0C46064600F0A0FC28
:10D74000BA685568C4F57E630F3325F003052B4492
:10D7500023F47F6323F00F03A3F58054B4F5805FB7
:10D7600007DB0021304601F079F8BB682B44984272
:10D7700004D0304600F08AFC0020F8BD61423046FB
:10D7800001F06CF801300DD0104ABB682D1B45F03C
:10D7900001055D60136830461B1B136000F076FCCA
:10D7A0000120F8BD0021304601F058F8BA68831A0C
:10D7B0000F2BDEDD43F001035360054B03491B686B
:10D7C000C01A0860D5E700BF44040024E4290024FF
:10D7D0004C080024002961D0F8B50C46064600F03C
:10D7E0004FFC54F8042C7B4FA4F1080522F00101F2
:10D7F00005EB010CB868DCF80430604523F0030346
:10D8000000F08B80D207CCF8043032D454F8082CC6
:10D81000AD1A1144AA6807F1080082426AD00CEBE5
:10D820000304D4F804E0EC68D4601EF0010FA26099
:10D8300000F0978041F001036B60CCF80010B1F567
:10D84000007F35D27A68CB08480901210133814035
:10D850001143796007EBC30257F83310083AC5E962
:10D86000021247F83350CD603046BDE8F84000F072
:10D870000DBC0CEB03025268D00710D4194407F119
:10D880000800DCF80830834273D0DCF80C20DA6042
:10D89000936041F001036B606950D0E7704741F03D
:10D8A0000103B1F5007F44F8043CCCF80010C9D363
:10D8B000B1F5206F4FEA512348D28B0903F13900AB
:10D8C00003F13802C300F818FB580838984259D0C1
:10D8D0005A6822F003028A4202D99B689842F7D123
:10D8E000D868C5E902308560DD603046BDE8F840A3
:10D8F00000F0CCBB0CEB03025268D20763D40B449C
:10D90000DCE90212CA60916043F001026A603046AD
:10D91000EB50BDE8F84000F0B9BB0B44D10707D489
:10D9200054F8082CAD1A1344D5E90212CA6091606C
:10D9300043F001026A60284ABD6012689A4293D897
:10D94000264B30461968FFF7F5FE8DE7142B0AD9F0
:10D95000542B1FD80B0B03F16F0003F16E02C300B1
:10D96000B1E719448DE703F15C0003F15B02C300EA
:10D97000A9E741F00103C7E90455C5E902006B605E
:10D98000695071E779689210012404FA02F20A439F
:10D990007A60A6E7B3F5AA7F06D8CB0B03F178002F
:10D9A00003F17702C3008EE740F25452934206D847
:10D9B0008B0C03F17D0003F17C02C30083E74FF47D
:10D9C0007E737E227FE741F001036B60CCF800108C
:10D9D0004AE700BF4404002450080024142A00240D
:10D9E0002DE9F8430746884600F538764FF00009E0
:10D9F000D6E90154013D11D4A389012B05F1FF356E
:10DA000008D9B4F90E300133214603D03846C04757
:10DA100049EA00096B1C04F16804EDD13668002E58
:10DA2000E6D14846BDE8F883004870474409002421
:10DA3000704700BF704700BF704700BF704700BF0E
:10DA40002DE9F0418B890C46990796B008D504F171
:10DA500043030122C4E90432236016B0BDE8F0811B
:10DA6000B4F90E100029064627DB6A4602F0A2F838
:10DA7000002821DB019D05F47045A5F50055B5FA98
:10DA800085F54FF480686D094FF4006741463046D4
:10DA900000F046F8B4F90C30F0B1204AF26343F0DC
:10DAA0008003C4F81480A3812060206135BB3B4310
:10DAB000A38116B0BDE8F081A38913F0800519D0C9
:10DAC0004FF040084146304600F02AF80025B4F9EE
:10DAD0000C302F460028E0D19A05BED423F0030372
:10DAE00004F1430243F002030121C4E90421A381AC
:10DAF0002260B2E74FF480682F46C7E7B4F90E10F2
:10DB0000304602F0E1F910B9B4F90C30CFE7A3893F
:10DB100023F0030343F001031BB2C8E7D9D5000883
:10DB20002DE9F04F01F10B06162E83B0044624D8E0
:10DB3000102900F2BA8000F0A3FA10261822022061
:10DB4000B54F3A44A2F1080153688B4200F0BA8005
:10DB50005A68D96822F003021A449D68E9608D6012
:10DB6000516841F001012046516003F1080500F0C1
:10DB70008DFA284603B0BDE8F08F36F0070600F1B5
:10DB80009480B14200F2918000F07AFAB6F5FC7F01
:10DB9000C0F09A81730A00F08F80042B00F26F812D
:10DBA000B30903F1390003F1380CC3009A4F3B4429
:10DBB000A3F108055B689D4206D10CE0002980F2C4
:10DBC0002781DB689D4206D05A6822F00302911B30
:10DBD0000F29F3DD60463D69DFF840C265457CD022
:10DBE0006A6822F00302931B0F2B00F37B81002B4A
:10DBF000C7E904CC80F26C81B2F5007F80F01A8115
:10DC0000D308796801334FEA521E012202FA0EF25C
:10DC10000A4357F833E0C5F808E007EBC3010839B9
:10DC2000E9607A6047F83350CEF80C508310012138
:10DC30009940914257D8114206D120F00300490083
:10DC4000114200F10400FAD007EBC0094D468646A8
:10DC5000D5F80C80454508D11DE1002B80F22481C8
:10DC6000D8F80C80454500F01681D8F8042022F041
:10DC70000302931B0F2BF0DD2046D8E9025408EB7A
:10DC8000060146F00106C8F80460EC60A56043F0A8
:10DC90000104C7E90411C1E902CC4C6048F8023024
:10DCA00000F0F4F908F1080502E00C2323600025D8
:10DCB000284603B0BDE8F08F4FF4007340204FF0CA
:10DCC0003F0C73E7D3689A4208BF02307FF440AF3D
:10DCD0003D69DFF848C1654582D17A68831001212A
:10DCE00099409142A7D9BD686B6823F003094E455E
:10DCF00003D8A9EB06030F2B7ADCDFF824B1494BDC
:10DD0000DBF800201B680132334405EB090A00F000
:10DD1000338103F580530F3323F47F6828F00F0815
:10DD20004146204600F09AFD411C024600F0F38077
:10DD3000824500F2EE803C4B196841441960084668
:10DD400000F04E81DBF80010019301311BBFA2EB04
:10DD50000A0A5044CBF80020186012F0070B00F0BC
:10DD60001781CBF108010A44CBF58051904408316A
:10DD7000A1EB0801C1F30B0A51462046009200F0C6
:10DD80006DFD421CDDE9002300F04F81801A00EB9D
:10DD90000A081968BA6048F001005144BD42506059
:10DDA000196000F02981B9F10F0F40F227816868EE
:10DDB000A9F10C0C2CF0070C00F0010040EA0C005B
:10DDC00068604FF0050E05EB0C00BCF10F0FC0E9C9
:10DDD00001EE00F2328150681546144B1A688A42EF
:10DDE00038BF1960124B1A688A4238BF196094E034
:10DDF000AA1943F0010346F001066E602046BA609E
:10DE0000536000F043F90835284603B0BDE8F08FB1
:10DE1000D9681A44A1E600BF440400244C0400243D
:10DE20004C080024142A0024E42900240C2A00248D
:10DE3000102A0024B2F5206F4FEA522363D3142B2B
:10DE400000F2B78003F15C01C9005B3307EB010E00
:10DE50007958AEF1080E8E4500F091804B6823F0A2
:10DE60000303934202D989688E45F7D1D1F80CE0BB
:10DE70007A68C5E9021ECEF80850CD60D6E6142BAC
:10DE800059D9542B00F29D80330B03F16F0003F13D
:10DE90006E0CC3008AE60EF1010E1EF0030F05F1B1
:10DEA00008057FF4D5AE51E0424445465368D8F8A2
:10DEB0000C1043F00103536055F8083F2046D96029
:10DEC0008B6000F0E3F8F3E6F00806F1080237E6AD
:10DED0002A442046536843F001035360083500F09C
:10DEE000D5F8E5E6A919204646F0010643F00104FD
:10DEF0006E60C7E90411C1E902CC4C60AB5000F080
:10DF0000C5F80835D4E6930903F13901C90038335F
:10DF10009CE7BD425FD0BD68686820F003084645B5
:10DF2000A8EB060302D80F2B3FF762AF204600F0A4
:10DF3000ADF80025BCE603F15C0003F15B0CC30007
:10DF400034E659F808394B4540F0968010F0030F3D
:10DF500000F1FF30F5D17B6823EA01037B604900C3
:10DF600099423FF6C0AE19B9BDE649000EF1040E64
:10DF70001942FAD0704667E603F11008D0E69A100D
:10DF80004FF001087B6808FA02F21A437A6070E7E2
:10DF900002EB08014942C1F30B0A514620460092A8
:10DFA00000F05CFC431CDDE900237FF4EFAEDA46B1
:10DFB000EFE6542B25D8130B03F16F01C9006E3324
:10DFC00044E7B3F5AA7F25D8F30B03F1780003F1FA
:10DFD000770CC300EAE5294B186840441860B1E6A5
:10DFE000CAF30B0CBCF1000F7FF4ACAEBD68C844A3
:10DFF00048F001006860F0E61546EEE60123536044
:10E0000094E7B3F5AA7F23D8D30B03F17801C900B5
:10E0100077331BE740F25452934223D8B30C03F1F9
:10E020007D0003F17C0CC300C0E5ABF1080BD844C4
:10E03000A8EB02084FF0000AABE605F10801204604
:10E040000093FFF7C7FBBD68009B68681968C4E6CA
:10E0500040F254518B420BD8930C03F17D01C9005F
:10E060007C33F3E64FF47E737F204FF07E0C9DE50A
:10E070004FF47E717E23E9E67B6870E7E429002493
:10E080000148FFF7D9BC00BFD82900240148FFF799
:10E09000D5BC00BFD8290024C36C70B505460C461A
:10E0A0004BB153F8240080B1026843F824200023C8
:10E0B000C0E9033370BD2122042101F02BFC03468B
:10E0C000E8640028EDD1002070BD012101FA04F6BA
:10E0D000721D9200284601F01DFC0028F3D0C0E913
:10E0E0000146E4E731B1C36C4A6853F82200086086
:10E0F00043F82210704700BF2DE9F0410D69074633
:10E100000E461C4601F1140E0020DEF800108BB202
:10E1100002FB03434FEA134C090C02FB01CC013014
:10E120009BB203EB0C4385424EF8043B4FEA1C4480
:10E13000EBDC3CB1B368AB4207DD06EB8503013590
:10E140005C6135613046BDE8F08171683846013167
:10E15000FFF7A2FF8046A8B13269023206F10C0136
:10E1600092000C30F2F7CCFCFB6C726853F8221072
:10E17000316043F82260464606EB850301355C6159
:10E180003561DFE7024B03484246B52101F0A2FBAF
:10E19000D407010868080108020C12040346CAB932
:10E1A0000304102013F07F4F04BF1B02083013F04C
:10E1B000704F04BF1B01043013F0404F04BF9B009D
:10E1C0000230002B05DB13F0804F00F1010008BF87
:10E1D000202070470020E5E70368024613F007009F
:10E1E00007D0D9071DD498071FD55B0813600120FD
:10E1F000704799B209B91B0C1020D9B209B908307F
:10E200001B0A190704BF1B090430990704BF9B08A8
:10E210000230D90703D45B0800F1010003D013607A
:10E22000704700207047202070479B081360022031
:10E23000704700BF38B5C36C04460D464BB15868F3
:10E24000B0B102685A6000220123C0E90435C260FF
:10E2500038BD2122042101F05DFB0346E064002863
:10E26000EDD1094B094800224FF4A07101F032FBB7
:10E270001C220121204601F04DFB0028F1D0012293
:10E280000223C0E90123DEE7D4070108680801087A
:10E290002DE9F04F0E691569AE4285B088461446E7
:10E2A00005DB2A46234635460C4616469846A368A3
:10E2B0006168AF19BB42B8BF0131FFF7EDFE0190B5
:10E2C000002800F08780019B03F1140909EB870AFD
:10E2D000D14505D24B46002243F8042B9A45FBD882
:10E2E00008F1140808EB860B04F11403D8451A460C
:10E2F00003EB85055FD22B1B153B23F0030304338F
:10E300001534A54238BF0423CDE902A7AC461F4609
:10E31000924605E0000C29D1C34509F1040948D90A
:10E3200058F8040B85B2002DF4D056464C46002315
:10E3300056F8040B216882B21FFA81FE05FB02EE3B
:10E34000000C0A0C734405FB002202EB13429BB243
:10E3500043EA0243B44544F8043B4FEA1243E7D88A
:10E3600049F8073058F8040C000CD5D0D9F8003023
:10E37000544619464D4600222688090C00FB06111A
:10E380000A449BB243EA024345F8043B54F8046B49
:10E390002968360C8BB200FB063303EB1243A4450D
:10E3A0004FEA1342E8D8C34549F8073009F1040998
:10E3B000B6D8DDE902A7002F02DC05E0013F03D05B
:10E3C0005AF8043D002BF9D0019B18461F6105B097
:10E3D000BDE8F08F034B0448019A40F25D1101F053
:10E3E00079FA00BFD40701086808010812F0030396
:10E3F0002DE9F0411446064632D10D46A41020D036
:10E40000D6F84880B8F1000F33D0E3074FF000078B
:10E4100007D4641015D0D8F80000A8B18046E307EF
:10E42000F7D5424629463046FFF732FFB5B1696855
:10E43000F36C641053F821202A6043F821500546FC
:10E44000E9D12846BDE8F081424641463046FFF713
:10E450001FFFC8F8000007608046E0E70546D8E7E0
:10E46000013B0F4A52F823200023FFF745FE0546E3
:10E47000C4E701213046FFF70FFE804640B101237B
:10E4800040F27122C0E904320023B0640360BCE7AB
:10E49000044B054842464FF4A07101F01BFA00BF3F
:10E4A000D8090108D4070108680801082DE9F047D8
:10E4B0000C4690462669A368496806EB6216751CEF
:10E4C0009D4207464FEA621904DD5B009D4201F15F
:10E4D0000101FADC3846FFF7DFFD8446002851D001
:10E4E000B9F1000F00F114000EDD09F105024FEA49
:10E4F000820E03460CEB8202002143F8041B934278
:10E50000FBD1AEF114031844216904F1140318F08F
:10E510001F0803EB81012DD0C8F1200986464FF07A
:10E52000000A1A6802FA08F242EA0A024EF8042BBC
:10E5300053F8042B994222FA09FAF2D80B1B153B27
:10E5400023F00303043304F11502914238BF04237E
:10E55000BAF1000F18BF2E4640F803A0FB6C6268AA
:10E56000CCF8106053F822102160604643F8224036
:10E57000BDE8F087043853F8042B40F8042F994283
:10E58000F9D8EBE7034B0448624640F2D91101F099
:10E59000A1F900BFD4070108680801080B69844687
:10E5A0000069C01A15D10CF1140C14310CEB830264
:10E5B00010B401EB830301E0944508D252F8044DF6
:10E5C00053F8041D8C42F7D004D24FF0FF3010BC3A
:10E5D00070477047012010BC704700BF2DE9F84F0D
:10E5E0000F691369FF1A002F0E4690467AD101F188
:10E5F0001405143202EB830205EB830301E09D4214
:10E6000073D253F8041D52F8044DA142F7D064D3DD
:10E610007168FFF741FD8146002872D03569D8F84E
:10E620001020C76008F1140E06F1140009F1140A55
:10E6300006F1100C0EEB820200EB85075646002116
:10E640005EF8044B5CF804BFA3B211FA8BF1CB1A4D
:10E65000210CC1EB1B4101EB23419BB243EA014377
:10E66000724546F8043B4FEA2141E9D8A2EB080481
:10E67000153C08F11508424524F0030606F104068E
:10E6800038BF0426304424F0030238BF00228742FA
:10E690005244B24416D95646044654F8043B11FA83
:10E6A00083F10A1402EB134289B241EA0243A74202
:10E6B00046F8043B4FEA2241EFD87A1E101A20F0A8
:10E6C0000302524423B952F8043D013D002BFAD015
:10E6D000C9F810504846BDE8F88F33460127464632
:10E6E000984695E7F9DB002792E70021FFF7D4FC75
:10E6F000814668B101220023C9E904234846BDE8E8
:10E70000F88F074B07484A464FF4107101F0E2F8C2
:10E71000034B04484A4640F2322101F0DBF800BFC7
:10E72000D40701086808010870B5012182B01646B7
:10E730001D46FFF7B1FC044600284BD02B46C5F31D
:10E740000A55C3F313030DB143F48013002E019354
:10E7500022D068460096FFF73FFD002836D0019B87
:10E760000099C0F1200203FA02F20A43C340019368
:10E770006261002B14BF02210121A3612161ADB1AF
:10E78000069AA5F2334303441360079BC0F135009A
:10E790001860204602B070BD01A8FFF71DFD019B67
:10E7A0000121C4E904132030002DE9D104EB8102DA
:10E7B000A0F232431069069A1360FFF7EDFC079B45
:10E7C000C0EB41112046196002B070BDDDE90023A5
:10E7D0006261CEE7034B0448224640F20A3101F061
:10E7E00079F800BFD407010868080108DFF860C0A5
:10E7F000F8B521F000430027634504460D46164650
:10E80000176022DC844653EA0C0C1ED0DFF844C0AB
:10E8100001EA0C0C0A46BCF1000F09D10E4B002294
:10E82000F2F7F8FD6FF0350704460A4621F0004381
:10E8300022F0FF421B1522F4E002A3F2FE3342F065
:10E840007F553B4445F40015336020462946F8BD0A
:10E85000FFFFEF7F0000F07F0000504338B5074D09
:10E860000022044608462A60F3F79EFC431C00D0B1
:10E8700038BD2B68002BFBD0236038BD182A00243C
:10E8800010B50C46B1F90E1001F0DEFB002803DBD9
:10E89000236D0344236510BDA38923F48053A38112
:10E8A00010BD00BF2DE9F0410C46B1F90C101F4618
:10E8B000CB05054616460BD421F48051A1813B4679
:10E8C000B4F90E1032462846BDE8F04100F0A6BF6C
:10E8D000B4F90E100223002201F00EFBB4F90C1063
:10E8E000EAE700BF10B50C46B1F90E1001F004FBC9
:10E8F000A389421C0EBF23F4805343F48053206548
:10E90000A38110BDB1F90E1001F040B830B540EA56
:10E910000104A30701D1032A0FD8844601F1FF3E69
:10E9200007E01EF8011F03F8011B541EC1B19C46ED
:10E9300022466346002AF4D130BD0B468446194670
:10E9400053F8045BA5F1013424EA050414F0803F78
:10E95000E4D1043A032A4CF8045B1946EFD8DDE70A
:10E960006244002CE8D003F8011B9342FBD130BD78
:10E970002DE9F84F4B6E9C0490462DD59368126894
:10E9800043B38B46064602F1080959E9025A5FEA89
:10E990009A0715D0043D002401E0A7420ED055F897
:10E9A000041F5A46304601F0D1F8431C04F101041B
:10E9B000F3D10023C8E90133BDE8F88FD8F8083057
:10E9C0002AF0030AA3EB0A03C8F8083009F1080982
:10E9D000002BDAD10020ECE701F002F90023C8E9AE
:10E9E0000133BDE8F88F00BF10B4946814B110BCB7
:10E9F000FFF7BEBF2046546010BC70472DE9F04FB2
:10EA0000BDB0CDE904301C460191174618B1836BA7
:10EA1000002B00F08682019A536EDE0740F18F8151
:10EA2000B2F90C108AB2900408D441F40052019952
:10EA30004B6E8A8123F4005392B24B66110740F16A
:10EA4000F780019B1B69002B00F0F28002F01A0393
:10EA50000A2B00F0FB8013AB10930023CDE9113398
:10EA6000CDE90A3308930DF14C09099303933B78E0
:10EA7000002B00F051813C4604E014F8013F002BCC
:10EA800000F02C81252BF8D1E51B40F0298123785B
:10EA9000002B00F041814FF0000300258DF83B3042
:10EAA000671C637802954FF0FF3B2B240137A3F1DD
:10EAB00020025A2A00F25281DFE812F09802500137
:10EAC000500194025001500150016A005001500160
:10EAD00036026B0250014102A6025001A2025B0005
:10EAE0005B005B005B005B005B005B005B005B004E
:10EAF000500150015001500150015001500150018E
:10EB00005001230284005001500150015001500176
:10EB100050015001500150015001DD0050015001E1
:10EB20005001070250015902500150011E055001C9
:10EB3000500150015001500150015001500150014D
:10EB40005001230286005001500150014F028600FF
:10EB500080005001450250018102DF006F028000F9
:10EB6000500107027E003E05500150014005500152
:10EB70007E00A3F13002002117F8013B01EB810177
:10EB800002EB4101A3F13002092AF5D902918EE787
:10EB9000DDF814804046FEF747FF43680A931846A5
:10EBA000F2F70EFA0B9006464046FEF73DFF8368EB
:10EBB0000993002E40F07B843B7877E73B7845F063
:10EBC000200573E745F01005AC06049E40F16F8107
:10EBD000073626F007063246736852F8086B04922F
:10EBE0009846002BC0F22D84BBF1FF3F00F010854A
:10EBF00056EA080325F0800A00F008840A2E78F10E
:10EC0000000380F0BD84303601238DF8EF60554657
:10EC100000930DF1EF04DDF800809DF83B30D845FE
:10EC2000B8BFD846002B00F0A88008F10108A4E086
:10EC3000019D05982946FDF7A3FB002840F0888533
:10EC4000AA8902F01A030A2B7FF405AF0199B1F9E2
:10EC50000E30002BFFF6FFAE4B6EDE0702D495059B
:10EC600040F156850199059823463A463DB0BDE8E6
:10EC7000F04F00F093BD45F0100515F0200800F0AE
:10EC80000781049E073626F007063346D6F804802F
:10EC900053F8086B049325F4806A00234FF00002B8
:10ECA0008DF83B20BBF1FF3F00F0C88156EA080217
:10ECB0002AF0800540F0C181BBF1000F40F0AB8429
:10ECC000002B40F0A8831AF00103009300F0D683D4
:10ECD00030238DF8EF300DF1EF049CE7E51B1BD0DE
:10ECE000119B129A01332A44072BC9E9007512922D
:10ECF000119305DC09F10809039B2B440393C6E635
:10ED0000002A00F07F830199059810AAFFF730FED2
:10ED100040B90DF14C09EFE7129B002B40F009853B
:10ED200000231193019A536ED90740F1A68093896D
:10ED30005B0600F1198503983DB0BDE8F08F019B9B
:10ED4000B3F90C108D058AB23FF56DAE1D46986D76
:10ED5000FEF772FEB5F90C108AB264E6002BDBD028
:10ED60008DF88C304FF001084FF000038DF83B30E8
:10ED7000CDF8008023AC4FF0000B15F00203069392
:10ED800018BF08F1020815F08403079305D1029B10
:10ED9000A3EB0806002E00F36C82DDE91121501C64
:10EDA0009DF83B608EB10DF13B020131C9F80020A6
:10EDB00007284FF00102CDE91101C9F8042000F342
:10EDC0003B82024609F108090130069BDBB10FAB1B
:10EDD0000231C9F8003007284FF00203CDE91101D4
:10EDE000C9F8043040F34082002900F006830199FD
:10EDF000059810AAFFF7BCFD002893D1DDE9112189
:10EE00000DF14C09501C079B802B00F05881009B92
:10EE1000ABEB0306002E00F3B681009BC9F800405F
:10EE200019440728CDE91101C9F8043040F34481A1
:10EE3000002900F072820199059810AAFFF798FD49
:10EE400000287FF46FAF12990DF14C09680705D5C2
:10EE5000029BA3EB0804002C00F36982DDE9022386
:10EE60004245ACBF9B1843440393002940F0D58131
:10EE7000002311930DF14C09F9E5019B9B899A053B
:10EE80003FF556AF019CA06DFEF7D8FDA3894FE773
:10EE900015F0100340F0238315F0400200F0EB83DF
:10EEA000049A52F8046B04929846B6B2F3E656F808
:10EEB000043B0496E80600F1ED82690640F1E78222
:10EEC00043F3C0381EB243468BE6049E56F8044B0B
:10EED0004FF000038DF83B30002C00F0B183BBF104
:10EEE000FF3F00F02E835A4600212046F2F718F823
:10EEF000002800F01284031B009304964FF0000BCF
:10EF000089E6049E4FF000038DF83B304FF0010876
:10EF100056F8043B8DF88C300496CDF8008023AC75
:10EF200029E7FEF75FFB76E5049B53F8042B02927A
:10EF3000002A80F29F82029A0493524202923B7806
:10EF400045F00405B2E53B786C2B03BF7B7845F0B8
:10EF50002005013745F01005A8E53B78682B03BF75
:10EF60007B7845F40075013745F040059EE545F096
:10EF7000100A1AF0200800F05582049E073626F089
:10EF800007063346D6F8048053F8086B0493012330
:10EF900084E63B788DF83B4088E5049B53F8046B8E
:10EFA000049330238DF83C3078238DF83D30B94BF5
:10EFB000089345F0020A4FF0000802236EE6AE0601
:10EFC00000F18382EC0600F13383680600F192833E
:10EFD000A90540F12D83049E039A56F8043B04963C
:10EFE0001A7044E53B7845F001055FE59DF83B303C
:10EFF000002B7FF4E1AD20238DF83B303B7855E5C5
:10F000003B7845F0800551E5394611F8013B2A2B44
:10F0100000F0B383A3F13002092A0F464FF0000B32
:10F020003FF645AD17F8013B0BEB8B0B02EB4B0B9F
:10F03000A3F13002092AF5D939E5AA46012B3FF49C
:10F04000DDAD022B3CAC12D1089A06F00F03360955
:10F05000D35C04F8013D46EA08764FEA181856EAF0
:10F060000803F2D13CAB1B1B55460093D3E506F0D9
:10F070000703F60846EA48764FEAD808303356EADE
:10F080000801224604F8013DF1D11AF0010FE9D040
:10F09000302BE7D03023023A04F8013C3CAB9B1AFA
:10F0A000554600931446B6E5009913940123149134
:10F0B000129111930DF14C0909F10809C6E6029B62
:10F0C000A3EB0806002E7FF7A2AE102E40F351836B
:10F0D000DFF8C4A15346CDE906B4BA46DDF814B052
:10F0E000019C2F461D4607E002F1020C09F10809B8
:10F0F0000246103E102E1EDD501C10311023072832
:10F10000CDE91101C9F80050C9F80430ECDD10AAAE
:10F11000002900F08B80214658460DF14C09FFF77D
:10F1200027FC00287FF4FEADDDE91121103E102EF2
:10F1300002F1010CE0DCDDE906B42B463D46574602
:10F140009A463144BCF1070FCDE911C1C9F800A0BE
:10F15000C9F8046040F39581002900F0BB82019951
:10F16000059810AAFFF704FC00287FF4DBAD009B94
:10F17000DDE91121ABEB0306002E02F101000DF1D8
:10F180004C097FF74AAE102EDFF80CA131DD534653
:10F19000CDE90645BA46059C019D4FF0100B1F4670
:10F1A00007E002F1020C09F108090246103E102E98
:10F1B00019DD501C10310728C9E9007BCDE9110188
:10F1C000EFDD10AA19B3294620460DF14C09FFF7CF
:10F1D000CFFB00287FF4A6ADDDE91121103E102EF3
:10F1E00002F1010CE5DCDDE906453B466046574689
:10F1F0009A4631440728CDE91101C9F800A0C9F8A1
:10F20000046000F3E68009F10809013005E64FF0DB
:10F21000010C0A460DF14C09C8E70199059810AA9E
:10F22000FFF7A6FB00283FF423AE7BE54FF0010C6F
:10F230000A460DF14C095CE7002900F0DB800199DA
:10F24000059810AAFFF794FB00287FF46BADDDE969
:10F2500011210DF14C09501CB7E502210FAB14919F
:10F26000139301200DF14C09024609F10809501CC5
:10F27000C9E5102E40F35782DDE911C1DFF81CA06B
:10F28000CDE90CB410235446DDF804B0DDF814A029
:10F2900062460DE06C060108F4090108E409010862
:10F2A00002F1020C09F108090246103E102E1BDD86
:10F2B000501C10310728C9E90043CDE91101EFDDE9
:10F2C00010AA21B3594650460DF14C09FFF750FBE7
:10F2D00000287FF427ADDDE91121103E102E02F148
:10F2E000010C4FF01003E3DCA246DDF830B00D9CBA
:10F2F00062463144072ACDE91121C9F800A0C9F8B6
:10F30000046000F3A78009F10809501C48E50A468B
:10F310004FF0010C0DF14C09C7E76C07119150D566
:10F32000029BA3EB0804002C4BDD0DF14C09102CC3
:10F3300040F30982DFF8ECA2119A059EDDF804B0D3
:10F3400053461025BA461F4606E0901C09F10809ED
:10F350001A46103C102C19DD531C1031072BC9E93B
:10F360000075CDE91131F0DD10AA29B359463046B8
:10F37000FFF7FEFA00287FF4D5ACDDE91121103C3F
:10F38000102C02F101000DF14C09E5DC3B4657461B
:10F390009A4621440728C9E900A4CDE911017FF765
:10F3A0005DAD71B10199059810AAFFF7E1FA002847
:10F3B0007FF4B8AC129951E501200A460DF14C09D1
:10F3C000C7E7DDE902234245ACBF9B1843440393E2
:10F3D0004EE500293FF468AE0199059810AAFFF7A1
:10F3E000C7FA00287FF49EAC1198129901300DF1F4
:10F3F0004C0912E5069B002B77D101200A460DF13E
:10F400004C0900E511920DF14C0975E4BBF1000FB8
:10F410007FF4F9AB55464FF0000BCDF800B03CAC93
:10F42000FFF7F9BB1AF010033AD11AF0400200F0CE
:10F430001381049A52F8046B04929846B6B20123E1
:10F440002CE42D2376428DF83B3068EB4808AA4621
:10F45000012327E400297DD00199059810AAFFF720
:10F4600087FA00287FF45EACDDE911210DF14C092B
:10F47000501C95E404933B78FFF718BB3CACFFF7B6
:10F48000CABB09F108090CF101006246BFE4AA05F4
:10F4900000F138814FEAE3781E464346FFF7A1BBEF
:10F4A000049B53F8046B04930123FFF7F7BB099BFC
:10F4B000002B3FF481AB099B1B78002B3FF47CAB06
:10F4C0003B7845F48065FFF7F1BADDE9031656F89D
:10F4D000042B0496CB17C2E90013FFF7C8BA049BAC
:10F4E00053F8046B0493FFF7D6BB02210FAB1491C2
:10F4F00013930DF14C09B8E64B4A089215F0200819
:10F5000036D0049E073626F007063246D6F8048029
:10F5100052F8086B0492EA0709D556EA080206D0A9
:10F520008DF83D30302345F002058DF83C3025F450
:10F53000806A0223FFF7B2BBAA461AE53B4A08924B
:10F54000DCE720460496F1F73BFD4FF0000B0090FE
:10F55000FFF761BB9DF83B20002A00F0C18001202D
:10F560000DF13B02149013920DF14C09014628E471
:10F5700015F0100242D0049A52F8046B0492CAE7C4
:10F580000AF48063CDF800B0CDF81890BB46DDF8E2
:10F59000249000253CAC1F4609E030464146F1F777
:10F5A0002DF90A2E78F100031BD306468846304613
:10F5B00041460A220023F1F721F91146303104F8BF
:10F5C000011C0A220023013C0135002FE5D099F8E7
:10F5D0000010A942E1D1FF2DDFD00A2E78F10003FF
:10F5E00064D23CAB1B1BCDF824905F46DDF818902D
:10F5F000DDF800B000935546FFF70DBB15F0400154
:10F6000047D0049951F8046B04919046B6B282E752
:10F61000AA46FFF7F3BA012BAA467FF412ADFFF713
:10F62000F2BA00BFE4090108800601086C0601086F
:10F63000049E039A56F8043B1A600496FFF717BA23
:10F64000BBF1060FD84628BF4FF00608504CCDF846
:10F6500000800496FFF78FBB049B1AF4007814BF58
:10F6600053F8046B53F8046B04931CBF9046F6B236
:10F670000123FFF713BB049B15F4007814BF53F864
:10F68000046B53F8046B04931CBF9046F6B2FFF76B
:10F6900002BB049A15F4007814BF52F8046B52F8B8
:10F6A000046B04921CBF8846F6B234E70B9B0A99A0
:10F6B000E41A1A462046FFF729F999F801300BB1F0
:10F6C00009F10109304641460A2200230025F1F7DD
:10F6D00095F86AE701200A460DF14C09FFF797BB40
:10F6E000069B002B7FF4B9AD0A4601200DF14C09B1
:10F6F000FFF78DBB049E039A56F8043B04961A80CC
:10F70000FFF7B5B943F3C0185EB24346FFF769BAD5
:10F71000886DFEF793F9FFF7A5BACDF800B004960F
:10F720008346FFF778BA119A1299DFF868A0013280
:10F73000DFE50199059810AAFFF71AF900283FF4B0
:10F74000EFAAFFF7EFBA1198DFF848A0013020E6E2
:10F75000019B5B6EDB0707D4019B9B899F0503D44C
:10F76000019B986DFEF76AF94FF0FF330393FFF7A3
:10F77000E2BADFF824A08446E3E4049A7B780F46DB
:10F7800052F8041B049241EAE17BFFF78FB900BFF6
:10F7900094060108E4090108F4090108F0B51F46C0
:10F7A0008B89ADF26C4D23F00203ADF80C304B6E3B
:10F7B0001993CB89ADF80E30CB6907934B6A099347
:10F7C0001AAB009304934FF48063154606460293E8
:10F7D000059316A800230C460693FEF729F92A463E
:10F7E0003B4669463046FFF709F9051E07DB6946C7
:10F7F0003046FDF7C3FE002818BF4FF0FF35BDF8B7
:10F800000C305B0603D5A38943F04003A38116980F
:10F81000FEF710F928460DF26C4DF0BD38B50C46D8
:10F82000084D8446114620461A4600232B60644644
:10F83000F2F700FC431C00D038BD2B68002BFBD036
:10F84000236038BD182A00242DE9F047DFF87CA09A
:10F850000646DAF8000098460F469146FEF7ECF8A7
:10F860001B4B1B68D3F8484124B365681F2D26DC69
:10F870005EB96B1C0235DAF80000636044F825704D
:10F88000FEF7DCF80020BDE8F08704EB85010123DA
:10F89000C1F88890D4F88821AB401A43022EC4F8EE
:10F8A0008821C1F80881E4D1D4F88C211343C4F82D
:10F8B0008C31DEE703F5A674C3F84841D5E7DAF8E2
:10F8C0000000FEF7BBF84FF0FF30DCE740040024F7
:10F8D0005806010800B50B4C25681446EE681A4618
:10F8E00085B003460D464CB107490095CDE901149A
:10F8F0003046064900F0C2F800F02CFE04490C46E0
:10F90000F3E700BF14000024040A0108140A0108E8
:10F91000100A010838B5A1FB02148CBBFEF700F9F0
:10F920000546E0B150F8042C22F00302043A242AE0
:10F9300017D8132A1AD91B2AC0E900441DD9242A32
:10F9400014BF00F1100200F118024FF00003C0E9EB
:10F95000024404BF04614461C2E900339360284655
:10F9600038BD2146FAF71CFE284638BD0246002362
:10F97000C2E900339360284638BD00F10802F6E77B
:10F98000FAF7E4FD0C2300250360E8E738B5074DDE
:10F990000022044608462A60F2F766FB431C00D0AA
:10F9A00038BD2B68002BFBD0236038BD182A0024FB
:10F9B00070B500294BD006460C4610B1836B002B66
:10F9C00048D0636ED80734D5B4F90C30002B3ED044
:10F9D00021463046FDF742FDE36A054633B1E16951
:10F9E000304698470028B8BF4FF0FF35A3891A0664
:10F9F0003BD4216B41B104F14003994202D030461F
:10FA0000FDF7E8FE00232363616C21B13046FDF76A
:10FA1000E1FE00236364FDF76BFE636E0022DB07EB
:10FA2000A28127D5A06DFEF705F8FDF767FE2846F1
:10FA300070BDA3899905CBD4A06DFDF7FDFFB4F986
:10FA40000C30002BC4D1656E15F0010508D00025DF
:10FA5000284670BDFDF7C6FD636ED807B4D4E8E74D
:10FA6000A06DFDF7EBFF284670BD21693046FDF71C
:10FA7000B1FEBEE7A06DFDF7E1FFD3E70EB410B510
:10FA800083B005AB064C53F8042B01930146206864
:10FA9000FEF7B4FF03B0BDE8104003B0704700BFED
:10FAA000140000242DE9F04383B00746884614462D
:10FAB00000F01CFA012803D108F1FF33FE2B37D9DF
:10FAC000424604F15C0301A9384600F017FD421CD0
:10FAD000064633D038B39DF804C00DF10509002562
:10FAE00009E023685A1C226083F800C00135B54242
:10FAF00019D219F801CBA368013B002BA360F0DAFF
:10FB0000D4F818E0734561462246384602DBBCF162
:10FB10000A0FE6D100F09AFC431CE7D106463046B6
:10FB200003B0BDE8F0834646304603B0BDE8F0833D
:10FB30005FFA88FC8DF804C00646CEE7A3893046FC
:10FB400043F04003A38103B0BDE8F08330B5536EAA
:10FB500013F0010FB2F90C30144683B005469AB287
:10FB600001D198051CD5900406D4626E43F400536D
:10FB700042F40052A381626622462846FFF792FFB4
:10FB8000636EDA07054602D4A3899B0502D5284691
:10FB900003B030BDA06DFDF751FF284603B030BD66
:10FBA000A06D0191FDF748FFB4F90C3001999AB2AC
:10FBB000D9E700BF70B50C46084D03460026204625
:10FBC00011461C462E60F2F77BFA431C00D070BD34
:10FBD0002B68002BFBD0236070BD00BF182A0024C7
:10FBE0009368002B00F081802DE9F04FB1F90C30C3
:10FBF0000C461907804683B0174698B223D523696F
:10FC00000BB310F002033D682BD04FF0000ADFF871
:10FC1000B4B256465E453346524628BF5B46404620
:10FC2000002E4FD0E169D4F824C0E047002852DD0F
:10FC3000BB681B1A8244361ABB60002BEAD1002035
:10FC400003B0BDE8F08F21464046FCF799FB002841
:10FC500040F03481B4F90C303D6898B210F00203E2
:10FC6000D3D110F0010942D14E463EB38205D4F8FB
:10FC700008B040F18180B3455A4600F2B18010F4DB
:10FC8000906F40F0BE8020680192494600F060F914
:10FC9000A3682168019AA3EB0B030A44B246A36050
:10FCA00022600026B868A0EB0A00D144B8600028A2
:10FCB000C5D0B4F90C0080B2002ED7D1D5E900969A
:10FCC0000835D2E7D5E900A60835A3E72146404626
:10FCD000FDF754FC80B3B4F90C3043F040034FF00F
:10FCE000FF30A38103B0BDE8F08F002070471E46AF
:10FCF000AA46994618461D4656B388B34A46D4E9E3
:10FD000004132068B24228BF3246884205D9A16850
:10FD100003EB010B5A4500F3A780934264DCE169D1
:10FD2000D4F824C02A464046E047B0F1000BD2DDAB
:10FD3000B9EB0B09CAD00120BB68A3EB0B035D44F0
:10FD4000A6EB0B06BB60002B3FF479AF002ED4D19D
:10FD50000AF1080353E902569A460833002EF9D0F7
:10FD600032460A212846F1F7DBF8002800F09D8092
:10FD70000130A0EB0509C1E720682369984217D834
:10FD80006369B34214D86FF00042B24228BF3246D2
:10FD9000E16992FBF3F2D4F824C002FB03F340467E
:10FDA0004A46E047B0F1000A95DDA6EB0A0679E77E
:10FDB000B345DA4628BFB2465246494600F0C8F875
:10FDC000A3682268A3EB0A035244A3602260002BBD
:10FDD000EBD121464046FDF7D1FB0028E5D07AE77C
:10FDE0002068B34632464FE72946019200F0B0F84A
:10FDF000019AA3689B1AA360236813442360934667
:10FE000096E723682169A3EB010B636903EB430ABF
:10FE10000AEBDA7A0BF101034FEA6A0A33445345DD
:10FE2000524684BF9A46524643052CD51146404659
:10FE3000FDF776FE00283BD05A4621690190F0F785
:10FE40005FFEA289019B22F4906242F08002A281AF
:10FE500003EB0B002361AAEB0B03C4F814A0A3600F
:10FE60002060B34632460FE729465A4600F070F844
:10FE700023685B44236021464046FDF77FFB002852
:10FE80003FF456AF27E7404600F0F4F80346002859
:10FE9000DED121694046FDF79DFCB4F90C300C22FF
:10FEA00023F08003C8F8002017E7721C914626E76C
:10FEB0000C22B4F90C30C8F800200EE74FF0FF30E8
:10FEC000BEE600BF00FCFF7F38B5074D00220446A8
:10FED00008462A60F2F7A2F8431C00D038BD2B6810
:10FEE000002BFBD0236038BD182A0024014B93F867
:10FEF000280170475408002438B50C46084D844644
:10FF0000114620461A4600232B606446F2F7B8F8E3
:10FF1000431C00D038BD2B68002BFBD0236038BDBC
:10FF2000182A002482B049B15AB16BB113780B6022
:10FF30001278101E18BF012002B0704701A9002AD4
:10FF4000F3D1104602B070476FF00100F4E700BF34
:10FF500088420DD98B1883420AD900EB020CBAB142
:10FF6000624613F801CD02F801CD9942F9D17047EC
:10FF70000F2A0ED8034602F1FF3C4AB10CF1010CE6
:10FF8000013B8C4411F8012B03F8012F6145F9D195
:10FF9000704740EA01039B0750D1A2F1100370B5EE
:10FFA00001F1200C23F00F0501F1100E00F11004F7
:10FFB000AC441B095EF8105C44F8105C5EF80C5C05
:10FFC00044F80C5C5EF8085C44F8085C5EF8045C7D
:10FFD00044F8045C0EF1100EE64504F11004E9D17A
:10FFE000013312F00C0F01EB031102F00F0400EBD0
:10FFF000031327D0043C24F003064FEA940C1E445C
:020000040801F1
:100000001C1F8E465EF8045B44F8045FB442F9D1CD
:100010000CF1010402F0030203EB840301EB840101
:1000200002F1FF3C4AB10CF1010C013B8C4411F888
:10003000012B03F8012F6145F9D170BD02F1FF3C9E
:1000400003469BE72246EBE738B50C46084D84464D
:10005000114620461A4600232B606446F2F718F832
:10006000431C00D038BD2B68002BFBD0236038BD6B
:10007000182A00242DE9F84F1746002900F098802F
:1000800007F10B0580460C46FDF7FAFF162D5DD8EB
:1000900010252A46AF425ED854F8041C21F003060E
:1000A0009642A4F1080962DABC4BD3F808C009EB08
:1000B0000600844500F09780D0F804C02CF00103BE
:1000C00003445B68DB0768D42CF0030C06EB0C03DD
:1000D000934247DACB0710D454F8083CA9EB030A43
:1000E000DAF8043023F003018C44B444944580F2E0
:1000F00011817318934280F2E88039464046FDF73B
:100100000FFD0746E0B154F8043C23F001034B44D3
:10011000A0F10802934200F0D280321F242A00F29C
:10012000F580132A00F2AC8003462246116819605C
:100130005168596092689A6021464046FDF74AFB33
:100140004046FDF7A3FF3846BDE8F88F25F00705C8
:10015000002D2A469EDA0C23C8F8003000273846C6
:10016000BDE8F88F1E46D0E90223D3609A60731B66
:100170000F2B22D8D9F8043003F0010333434E4447
:10018000C9F80430736843F00103736040462746A2
:10019000FDF77CFF3846BDE8F88FC907ADD454F8A9
:1001A000083CA9EB030ADAF8041021F00301A0E7E8
:1001B000BDE8F84F1146FDF7B3BCD9F8041001F0C3
:1001C00001012943C9F8041009EB05014E4443F02D
:1001D00001034B60736843F00103083173604046CC
:1001E000FDF7F8FAD2E7DCF8040020F0030B06EB89
:1001F0000B0C05F1100084454DDAC9073FF57DAFC2
:1002000054F8081CA9EB010ADAF8041021F00301E4
:100210008B44B34458453FF76CAF5746DAF80C109F
:1002200057F8080F321F242AC160886000F2DB8073
:10023000132A40F2D6802168CAF808106168CAF80B
:100240000C101B2A00F2DF8008340AF1100221682A
:10025000116061685160A16891600AEB0501ABEB28
:10026000050242F0010299604A60DAF8043003F0B6
:1002700001031D434046CAF80450FDF707FF6EE72F
:1002800023680360636843601B2A68D804F108028E
:1002900000F108034AE709EB05029A60ACEB05039D
:1002A00043F00103536054F8043C03F001031D4381
:1002B000404644F8045CFDF7E9FE27464FE750F856
:1002C000043C23F003031E4451E75746DAF80C10B0
:1002D00057F8080F321F242AC16088604CD8132AAF
:1002E00048D92168CAF808106168CAF80C101B2A9E
:1002F00056D808340AF110021E462368136063685A
:100300005360A3689360D1463C4630E72146FFF72F
:100310001FFE11E7D0E902135746CB60996057F8EA
:10032000081FDAF80C30CB60321F242A99602DD8D0
:10033000132A29D92368CAF808306368CAF80C3030
:100340001B2A42D808340AF1100322681A60626836
:100350005A60A2689A606646D1463C4607E7A368A1
:100360008360E368C360242A26D004F1100200F100
:100370001003DBE63A46BFE7214638461E46D14623
:10038000FFF7E6FD3C46F2E63B46DEE7214638460F
:100390006646D146FFF7DCFD3C46E8E6440400240F
:1003A000A168CAF81010E168CAF81410242A20D0F5
:1003B00010340AF118029FE7236903616169416102
:1003C00004F1180200F11803B0E6A368CAF810306F
:1003D000E368CAF81430242A21D010340AF1180333
:1003E000B3E73A4633E721463846FFF7B1FD164BEF
:1003F00033E72269CAF818206269CAF81C20183449
:100400000AF1200278E7A168CAF81010E168CAF87A
:100410001410242A0DD010340AF1180217E72369AA
:10042000CAF818306369CAF81C3018340AF120037E
:100430008BE72269CAF818206269CAF81C201834B0
:100440000AF1200203E700BF44040024F8B50D467A
:100450001446064610B1836B002B43D0B4F90C2030
:10046000A369A360170790B21BD52369CBB1EDB286
:1004700081042F4622D522686169D31A994229DD69
:100480000133A1680139A160511C216015706269B6
:100490009A422AD0A389DB0701D50A2D25D03846F8
:1004A000F8BD21463046FBF76BFF20BBB4F90C20AA
:1004B000236990B2EDB281042F46DCD442F400529D
:1004C000A281626E616922F4005262662268D31AC8
:1004D0009942D5DC21463046FDF750F858B92268DC
:1004E0000123CEE7FDF77EF8B8E721463046FDF759
:1004F00045F80028D3D04FF0FF37D0E770B5054658
:1005000084B01C4639B10B4ED6F8E060B047431CAE
:1005100009D004B070BD0A460649D1F8E06001A9CF
:10052000B047431CF5D100228A2322602B6004B01F
:1005300070BD00BF5408002449B1FF2A02D80A70D8
:10054000012070478A2303604FF0FF307047084650
:10055000704700BF08B5062000F004F80120F1F74D
:100560001DFE00BF38B5154B1F281D6820D8D5F8D3
:10057000DC22044662B152F820304BB1012B15D079
:10058000591C0FD0002542F820509847284638BD06
:10059000284600F02BF8224601462846BDE83840A0
:1005A00000F00EB816232B60012038BD002038BDA6
:1005B00016232B604FF0FF3038BD00BF140000241D
:1005C00070B50C46084D03460026204611461C46D1
:1005D0002E60F1F7DBFD431C00D070BD2B68002BB3
:1005E000FBD0236070BD00BF182A0024F1F7CCBDFA
:1005F000F8B500BFF8BC08BC9E467047F8B500BF10
:08060000F8BC08BC9E467047DF
:1006080023000000534554004D554C006D756C0097
:1006180000000000010203040102030406070809A0
:10062800000610160006101601000200040006005D
:1006380008000A000C0010002000400080000001A3
:100648000804020408010101010101030701000077
:1006580018000024494E4600696E66004E414E005F
:100668006E616E0030313233343536373839616275
:100678006364656600000000303132333435363744
:10068800383941424344454600000000286E756CE5
:100698006C2900003000000020202020202020208D
:1006A80020202020202020203030303030303030C2
:1006B80030303030303030300020202020202020D2
:1006C80020202828282828202020202020202020FA
:1006D800202020202020202020881010101010100A
:1006E8001010101010101010100404040404040456
:1006F80004040410101010101010414141414141F0
:1007080001010101010101010101010101010101D1
:1007180001010101101010101010424242424242E1
:1007280002020202020202020202020202020202A1
:100738000202020210101010200000000000000049
:1007480000000000000000000000000000000000A1
:100758000000000000000000000000000000000091
:100768000000000000000000000000000000000081
:100778000000000000000000000000000000000071
:100788000000000000000000000000000000000061
:100798000000000000000000000000000000000051
:1007A8000000000000000000000000000000000041
:1007B8000000000000000000000000004E614E0034
:1007C800496E66696E6974790000000042616C6C5C
:1007D8006F6320737563636565646564000000007A
:1007E8002F6D6E742F776F726B73706163652F77DF
:1007F8006F726B73706163652F4743432D31302DE2
:10080800706970656C696E652F6A656E6B696E7369
:100818002D4743432D31302D706970656C696E65C5
:100828002D3333385F32303231313031385F313641
:1008380033343531363230332F7372632F6E657728
:100848006C69622F6E65776C69622F6C6962632FC1
:100858007374646C69622F64746F612E63000000A6
:100868002F6D6E742F776F726B73706163652F775E
:100878006F726B73706163652F4743432D31302D61
:10088800706970656C696E652F6A656E6B696E73E9
:100898002D4743432D31302D706970656C696E6545
:1008A8002D3333385F32303231313031385F3136C1
:1008B80033343531363230332F7372632F6E6577A8
:1008C8006C69622F6E65776C69622F6C6962632F41
:1008D8007374646C69622F6D707265632E630000B7
:1008E8000080E03779C34143176E05B5B5B8934624
:1008F800F5F93FE9034F384D321D30F94877825AF0
:100908003CBF737FDD4F1575000000000000F03F0D
:1009180000000000000024400000000000005940D2
:100928000000000000408F40000000000088C34025
:1009380000000000006AF8400000000080842E419A
:1009480000000000D01263410000000084D79741E6
:100958000000000065CDCD41000000205FA00242EC
:10096800000000E876483742000000A2941A6D4261
:10097800000040E59C30A2420000901EC4BCD64254
:1009880000003426F56B0C430080E03779C34143FF
:1009980000A0D8855734764300C84E676DC1AB4375
:1009A800003D9160E458E143408CB5781DAF154493
:1009B80050EFE2D6E41A4B4492D54D06CFF080446E
:1009C800F64AE1C7022DB544B49DD9794378EA4483
:1009D80005000000190000007D00000020202020F4
:1009E80020202020202020202020202030303030BF
:1009F8003030303030303030303030302C20667588
:100A08006E6374696F6E3A2000000000617373654D
:100A18007274696F6E2022257322206661696C6585
:100A2800643A2066696C6520222573222C206C6943
:100A38006E65202564257325730A000043000000B5
:0C0A4800504F5349580000002E000000E1
:080A5400D8FDFE7F0100000047
:080A5C0055C40008E502000882
:040A6400C1020008C3
:100A6800320000000090D0030090D0030100000085
:100A780010000000180000240000000004030024F7
:100A88006C030024D40300240000000000000000D0
:100A9800000000000000000000000000000000004E
:100AA800000000000000000000000000000000003E
:100AB800000000000000000000000000000000002E
:100AC800000000000000000000000000000000001E
:100AD800000000000000000000000000000000000E
:100AE80000000000000000000000000000000000FE
:100AF80000000000000000000000000000000000EE
:100B080000000000000000000000000000000000DD
:100B180000000000000000000000000000000000CD
:100B280001000000000000000E33CDAB34126DE66A
:100B3800ECDE05000B0000000000000000000000D3
:100B4800000000000000000000000000000000009D
:100B5800000000000000000000000000000000008D
:100B6800000000000000000000000000000000007D
:100B7800000000000000000000000000000000006D
:100EA800D4290024000000000000000044040024AD
:100EB800440400244C0400244C040024540400245A
:100EC800540400245C0400245C040024640400240A
:100ED800640400246C0400246C04002474040024BA
:100EE800740400247C0400247C040024840400246A
:100EF800840400248C0400248C040024940400241A
:100F0800940400249C0400249C040024A4040024C9
:100F1800A4040024AC040024AC040024B404002479
:100F2800B4040024BC040024BC040024C404002429
:100F3800C4040024CC040024CC040024D4040024D9
:100F4800D4040024DC040024DC040024E404002489
:100F5800E4040024EC040024EC040024F404002439
:100F6800F4040024FC040024FC04002404050024E8
:100F7800040500240C0500240C0500241405002495
:100F8800140500241C0500241C0500242405002445
:100F9800240500242C0500242C05002434050024F5
:100FA800340500243C0500243C05002444050024A5
:100FB800440500244C0500244C0500245405002455
:100FC800540500245C0500245C0500246405002405
:100FD800640500246C0500246C05002474050024B5
:100FE800740500247C0500247C0500248405002465
:100FF800840500248C0500248C0500249405002415
:10100800940500249C0500249C050024A4050024C4
:10101800A4050024AC050024AC050024B405002474
:10102800B4050024BC050024BC050024C405002424
:10103800C4050024CC050024CC050024D4050024D4
:10104800D4050024DC050024DC050024E405002484
:10105800E4050024EC050024EC050024F405002434
:10106800F4050024FC050024FC05002404060024E3
:10107800040600240C0600240C0600241406002490
:10108800140600241C0600241C0600242406002440
:10109800240600242C0600242C06002434060024F0
:1010A800340600243C0600243C06002444060024A0
:1010B800440600244C0600244C0600245406002450
:1010C800540600245C0600245C0600246406002400
:1010D800640600246C0600246C06002474060024B0
:1010E800740600247C0600247C0600248406002460
:1010F800840600248C0600248C0600249406002410
:10110800940600249C0600249C060024A4060024BF
:10111800A4060024AC060024AC060024B40600246F
:10112800B4060024BC060024BC060024C40600241F
:10113800C4060024CC060024CC060024D4060024CF
:10114800D4060024DC060024DC060024E40600247F
:10115800E4060024EC060024EC060024F40600242F
:10116800F4060024FC060024FC06002404070024DE
:10117800040700240C0700240C070024140700248B
:10118800140700241C0700241C070024240700243B
:10119800240700242C0700242C07002434070024EB
:1011A800340700243C0700243C070024440700249B
:1011B800440700244C0700244C070024540700244B
:1011C800540700245C0700245C07002464070024FB
:1011D800640700246C0700246C07002474070024AB
:1011E800740700247C0700247C070024840700245B
:1011F800840700248C0700248C070024940700240B
:10120800940700249C0700249C070024A4070024BA
:10121800A4070024AC070024AC070024B40700246A
:10122800B4070024BC070024BC070024C40700241A
:10123800C4070024CC070024CC070024D4070024CA
:10124800D4070024DC070024DC070024E40700247A
:10125800E4070024EC070024EC070024F40700242A
:10126800F4070024FC070024FC07002404080024D9
:10127800040800240C0800240C0800241408002486
:10128800140800241C0800241C0800242408002436
:10129800240800242C0800242C08002434080024E6
:1012A800340800243C0800243C080024FFFFFFFF0A
:1012B80000000200430000000000000000000000E1
:1012C8000000000000000000000000000000000016
:1012D80000000000430000000000000000000000C3
:1012E80000000000000000000000000000000000F6
:1012F80000000000430000000000000000000000A3
:1013080000000000000000000000000000000000D5
:101318000000000043000000000000000000000082
:1013280000000000000000000000000000000000B5
:101338000000000043000000000000000000000062
:101348000000000000000000000000000000000095
:101358000000000043000000000000000000000042
:101368000000000000000000000000000000000075
:101378000000000043000000000000000000000022
:101388000000000000000000000000000000000055
:10139800000000003905010825FF000800000000D2
:1013A800C0060108500A0108100A0108100A0108BD
:1013B800100A0108100A0108100A0108100A010899
:1013C800100A0108100A0108100A0108FFFFFFFFB0
:1013D800FFFFFFFFFFFFFFFFFFFF0000010041537A
:1013E8004349490000000000000000000000000020
:1013F8000000000000000000000000000000415351
:1014080043494900000000000000000000000000FF
:1014180000000000000000000000000000000000C4
:0400000508002A695C
:00000001FF
